:020000040800F2
:1000000000000220E903010839A700083BA7000807
:100010003DA700083FA7000841A700080000000016
:1000200000000000000000000000000043A70008DE
:1000300045A700080000000047A7000849A70008DE
:100040002D0401082D0401082D0401082D040108C8
:100050002D0401082D0401082D0401082D040108B8
:100060002D0401082D0401082D040108656800080D
:100070002D0401082D0401082D0401082D04010898
:100080002D0401082D0401082D0401082D04010888
:100090002D0401082D0401082D040108E9A9000818
:1000A0002D0401082D0401082D0401082D04010868
:1000B00045A900082D0401082D0401082D0401089C
:1000C0002D0401082D0401082D0401082D04010848
:1000D0002D0401082D040108FDAA00082D040108C3
:1000E0002D0401082D0401084DA700082D04010866
:1000F0002D0401082D0401082D0401082D04010818
:100100002D0401082D0401082D0401082D04010807
:100110002D0401082D0401082D0401082D040108F7
:100120002D0401082D0401082D0401082D040108E7
:100130002D0401082D0401082D0401082D040108D7
:100140002D0401082D0401082D0401087DA70008D5
:100150002D0401082D0401082D0401082D040108B7
:100160002D0401082D0401082D0401082D040108A7
:100170002D0401082D0401082D0401082D04010897
:080180002D0401082D04010803
:1001880084B0050800000020FC0C0020000D0020B1
:10019800FC52002008B5074B186807F0ABFF0AF0BF
:1001A80071FA054B054801221A70BDE8084001F0B4
:1001B8006CBA00BFA83E0020443E00206C0F00200F
:1001C80008B5034801F061FA024B00221A7008BD15
:1001D80044130020443E002008B5054B01220020AE
:1001E8001A7004F05DFE0348BDE8084001F04DBAFE
:1001F800C0440020E81300202DE9F041144C2046AB
:1002080002F0ADFF00201349134A02F05FFD1349C5
:10021800134A0746002002F059FD1249124A0646C1
:10022800002002F053FDD22105463A4623460A2013
:1002380002F064FED22132462346FA2002F05EFE26
:100248005A20D2212A462346BDE8F04102F056BE84
:10025800FC1100206E9F0508C9010008779F05085A
:10026800E10100087F9F05089D01000808B5054BBE
:10027800012200201A7004F013FE0348BDE808406C
:1002880001F003BAC0440020E813002008B5034871
:1002980001F0FBF9024B00221A7008BD441300203C
:1002A800443E002008B5054B02221A700AF0EAF90C
:1002B8000348BDE8084001F0E8B900BF443E00200B
:1002C800FC1100202DE9F041144C204602F047FFB4
:1002D80000201349134A02F0F9FC1349134A074650
:1002E800002002F0F3FC1249124A0646002002F0F0
:1002F800EDFCD22105463A4623460A2002F0FEFDCF
:10030800D221324623465A2002F0F8FDAA20D221F3
:100318002A462346BDE8F04102F0F0BD6C0F0020EC
:100328006E9F050895020008889F0508AD02000821
:10033800919F050875020008014801F0A6B900BFA1
:100348001010002010B5094C204602F008FF0020CC
:100358000749084A02F0BAFCD221024623464FF464
:100368008270BDE8104002F0C9BD00BF3015002002
:100378009A9F05084103000810B5074C4FF6E07135
:10038800206801F0E7FF2068044901F091FFBDE80B
:10039800104003F01DB900BF000D0020A19F050803
:1003A80010B5074C4FF6E071206801F0D3FF2068C4
:1003B800044901F07DFFBDE8104003F009B900BF12
:1003C800000D0020B69F050810B5074C4FF6E071E8
:1003D800206801F0BFFF2068044901F069FFBDE80B
:1003E800104003F0F5B800BF000D0020CB9F0508B2
:1003F80010B5074C4FF6E071206801F0ABFF20689C
:10040800044901F055FFBDE8104003F0E1B800BF12
:10041800000D0020E09F050810B51E4CFFF7C0FF37
:10042800002004F03DFD23790BB9FFF7CDFF637978
:100438000BB9FFF7DDFFA3790BB9FFF79DFF154B4C
:100448005A79E2B11A79D2B1997900221A715A719E
:1004580001B19A71104B0F4C1A7008F03FFF2068D9
:100468004FF6E07101F076FF20680C4901F020FF9B
:1004780008F053F803F0ACF8094803F0EDF8FFF77B
:100488008FFF002008F00CF80648BDE8104001F086
:10049800FCB800BF000D0020443E0020F59F050871
:1004A800809698004413002008B5002007F0F8FF54
:1004B8000248BDE8084001F0E8B800BF4413002036
:1004C80010B586B04FF07E5302930023039308F0D3
:1004D800B4FD8DED000ACDED010A9DE8030006ABE1
:1004E80003E903009DED020ADDED030A9DED041A00
:1004F800DDED051A08F053FD104C002084ED040AC8
:10050800C4ED050A07F0DAFF20644FF6E07004F046
:100518009BFC3C215E220023B72004F0B1FD0120A2
:1005280007F0BEFF064B02224FF0804001211A70EF
:1005380006B0BDE810400EF08AB900BF3848002068
:100548001D0E00201FB508F078FD8DED000ACDEDD9
:10055800010A9DE803000E4A02AB83E8030082E823
:1005680003004FF6E07004F06FFC6E210023B72003
:100578005E2204F085FD012007F092FF054B012162
:100588004FF08040197005B05DF804EB0EF05FB9CC
:10059800384800201D0E002010B5214B2148224C60
:1005A80086B002930023039303F056F808F045FD44
:1005B8002046012184ED080AC4ED090A08F0A9FDC6
:1005C8008DED000ACDED010A9DE8030006AB03E9B5
:1005D80003009DED020ADDED030A9DED041ADDED31
:1005E800051A08F0DCFC4FF6E07084ED0C0AC4ED47
:1005F8000D0A04F029FCA0215E220023B72004F094
:100608003FFD012007F04CFF084B03224FF08040CC
:1006180001211A7006B0BDE810400EF018B900BFED
:1006280000004842A0860100384800201D0E002026
:100638002DE9F04F434D444E85B000244FF6FF7826
:10064800284602F08CFD4146224623463F48009446
:10065800019401F043FE0427B060224623464FF67A
:10066800E0713B480097019401F038FE2346306062
:100678004146224637480097019401F02FFE36493B
:10068800F060364A204602F021FB3549354A0746D4
:10069800204602F01BFB3449344A8046204602F0CB
:1006A80015FB3349334A8146204602F00FFB324995
:1006B800324A8246204602F009FB3149314A8446D3
:1006C8002046CDF80CC002F001FB21468346B268F3
:1006D8002B46204602F012FC214632682B467D202C
:1006E80002F00CFC2321F2682B46B42002F006FC31
:1006F8009B213A462B46FA2002F000FC692142462B
:100708002B46FA2002F0FAFB37214A462B46FA20FC
:1007180002F0F4FBC82152462B466E2002F0EEFB95
:10072800C8215A462B46AA2002F0E8FBDDF80CC087
:10073800F0206246C8212B4605B0BDE8F04F02F014
:10074800DDBB00BFA0120020000D002009A0050895
:1007580011A0050822A005082AA00508A10500087F
:1007680032A005084D0500083AA00508C90400088C
:1007780042A00508210B000849A00508B10400089B
:1007880050A00508210400081FB5134802F064FFB3
:1007980008F053FC8DED000ACDED010A9DE8030039
:1007A8000E4A02AB83E8030082E803004FF6E070CC
:1007B80004F04AFBFFF71CFEDF205E2200236E21B7
:1007C80004F05EFC064B012200201A7105B05DF8AA
:1007D80004EB07F065BE00BFA0860100404800207A
:1007E800000D002010B586B04FF07E530293002311
:1007F800039308F022FC8DED000ACDED010A9DE877
:10080800030006AB03E903009DED020ADDED030AD0
:100818009DED041ADDED051A08F0C1FB0E4C002011
:1008280084ED060AC4ED070A07F054FE60644FF62B
:10083800E07004F009FBDF203C215E22002304F075
:100848001FFC064B01229A71FFF7BEFD002006B07F
:10085800BDE8104007F024BE38480020000D0020F5
:1008680008B5FFF789FDBDE8084002F0B1BE70B5D4
:100878002DED028B9FED238A88B00A26F0EE488A78
:1008880003E0B0EE608AF0EE418A08F0D6FB8DED09
:10089800000ACDED010A9DE8030004AB83E80300DC
:1008A800F0EE680AB0EE480A9DED041ADDED051A6F
:1008B8008DED028ACDED038A08F056FBCDED010AD5
:1008C8008DED000A9DE8030002AD85E80300013EB6
:1008D8006C46DDED020A9DED031AD2D19FED0A0A9E
:1008E80008F0A2FB8DED000ACDED010A9DE803009A
:1008F80085E80300DDED030A9DED020A08B0BDECB2
:10090800028B70BD00000000CDCCCC3D2DE9F74F27
:10091800564D574CDFF86491DFF864814FF6E0706C
:1009280004F092FA28680EF0E3FE064668680F465F
:100938000EF0DEFE3246CDE900013B464946204630
:1009480013F03CFC224600230520372104F0B6FBB7
:100958002869484F484E0EF0CBFE824668698B46A0
:100968000EF0C6FE5246CDE900015B4639462046E8
:1009780013F024FC224600230520692104F09EFB85
:10098800286B0EF0B5FE8246686B8B460EF0B0FE03
:100998005246CDE900015B464146204613F00EFC65
:1009A800002305209B21224604F088FB31462A6C4F
:1009B800204613F003FC224600239B21A22004F0CA
:1009C8007DFB4FF4FC6004F03FFAA8680EF090FE3F
:1009D8008246E8688B460EF08BFE5246CDE9000150
:1009E8005B464946204613F0E9FB22460520502184
:1009F800002304F063FBA8690EF07AFE8246E869DA
:100A08008B460EF075FE5246CDE900015B4639462D
:100A1800204613F0D3FB224600230520822104F050
:100A28004DFBA86B0EF064FE8246E86B8B460EF019
:100A38005FFE5246CDE900015B464146204613F071
:100A4800BDFB00230520B421224604F037FB3146C4
:100A58006A6C204613F0B2FBA220B4212246002380
:100A680003B0BDE8F04F04F029BB00BF38480020B0
:100A7800100D002069A005088CA0050857A00508DE
:100A88007BA0050810B5204B2048214C86B0029366
:100A98000023039302F0E0FD08F0CFFA204602217C
:100AA80084ED0A0AC4ED0B0A08F033FB8DED000A49
:100AB800CDED010A9DE8030006AB03E903009DEDB7
:100AC800020ADDED030A9DED041ADDED051A08F0B2
:100AD80066FA4FF6E07084ED0E0AC4ED0F0A04F0D2
:100AE800B3F9DF20A0215E22002304F0C9FAFFF742
:100AF80057FC084B01225A71FFF708FF002006B087
:100B0800BDE8104007F0CCBC00004842A0860100B8
:100B180038480020000D002008B5FFF741FCBDE86B
:100B28000840F3E6002008B504F0BAF9064B0022A5
:100B38001A70064B1B78022B0CBF05480548BDE808
:100B4800084000F0A2BD00BFC0440020443E002081
:100B5800FC1100206C0F00202DE9F14F2D4C204690
:100B680002F0FDFA00202C492C4A02F0AFF82C497B
:100B78002C4A8146002002F0A9F82B492B4A074647
:100B8800002002F0A3F82A492A4A0646002002F06B
:100B98009DF82949294A0546002002F097F8284976
:100BA800284A8046002002F091F82749274A8246C1
:100BB800002002F08BF8D22183464A462346E620DD
:100BC80002F09CF928203A462346014602F096F99D
:100BD800462132462346282002F090F964212A460D
:100BE8002346282002F08AF98221424623462820FB
:100BF80002F084F9524623462820A02102F07EF90B
:100C080028205A46BE21234601B0BDE8F04F02F025
:100C180075B900BFE813002091A005082D0B000846
:100C28009AA0050841110008A5A005081D11000893
:100C3800AFA00508F9100008BAA00508D5100008EB
:100C4800C5A00508B1100008CFA005088D10000840
:100C5800023810B5052800F2CE81DFE810F0060052
:100C68000A005F00C90081011701BDE8104007F0C4
:100C7800C1BC00204FF6E07107F0C4FD63204FF6B9
:100C8800E07107F0BFFDB3204FF4F06107F0BAFD43
:100C9800C7204FF6E07107F0B5FD4FF6FF7004F07E
:100CA800D3F8DC2100237D20D34A04F007FA4EF262
:100CB8009C7004F0C9F8052001210023CF4A04F0F4
:100CC800FDF9052052210023CD4A04F0F7F9B62199
:100CD80000230520CB4A04F0F1F94FF4F06004F04A
:100CE800B3F80121002340F21310C44A04F0E6F9D6
:100CF800002340F213105221C24A04F0DFF9B62152
:100D0800C14A40F21310002304F0D8F94EF29C7047
:100D180004F09AF80520A221BC4A67E100204FF6AA
:100D2800E07107F06FFD31204FF6E07107F06AFDC2
:100D380063204FF6E07107F065FD95204FF6E071EE
:100D480007F060FDC7204FF6E07107F05BFD4EF23B
:100D58009C7004F079F8052001210023AC4A04F0C6
:100D6800ADF9052020210023AA4A04F0A7F905209F
:100D780052210023A84A04F0A1F905208421002368
:100D8800A64A04F09BF9B62105209E4A002304F0E8
:100D980095F94FF4F06004F057F8012140F2131070
:100DA80000239B4A04F08AF940F2131020219C4A40
:100DB800002304F083F940F213105221914A0023D2
:100DC80004F07CF940F213108421964A002304F0C1
:100DD80075F9B621944A40F21310002304F06EF915
:100DE8004FF6FF7004F030F87D20DC218F4AFDE0DB
:100DF80000204FF6E07107F005FD27204FF6E0715F
:100E080007F000FD4F204FF6E07107F0FBFC77205C
:100E18004FF6E07107F0F6FC9F204FF6E07107F0FF
:100E2800F1FCC7204FF6E07107F0ECFC4EF29C7025
:100E380004F00AF8052001210023724A04F03EF963
:100E48000520162100237A4A04F038F905203E21AE
:100E58000023784A04F032F9052066210023764AF7
:100E680004F02CF98E2100230520744A04F026F999
:100E78000520734AB621002304F020F94FF6FF70CD
:100E880003F0E2FF7D20DC216E4AAFE000204FF640
:100E9800E07107F0B7FC31204FF6E07107F0B2FCC3
:100EA80063204FF6E07107F0ADFC95204FF6E07136
:100EB80007F0A8FCC7204FF6E07107F0A3FC4EF23C
:100EC8009C7003F0C1FF0520012100235E4A04F055
:100ED800F5F80520202100235C4A04F0EFF80520EE
:100EE800522100235A4A04F0E9F8052084210023FE
:100EF800584A04F0E3F8B6210520424A002304F0DA
:100F0800DDF84FF4F06003F09FFF012140F2131069
:100F18000023514A04F0D2F840F2131020214F4A1E
:100F2800002304F0CBF840F213105221354A002375
:100F380004F0C4F840F213108421494A002304F055
:100F4800BDF8B621474A40F21310002304F0B6F862
:100F58004FF6FF7003F078FF7D20DC21424A45E020
:100F680000204FF6E07107F04DFC31204FF6E0719C
:100F780007F048FC63204FF6E07107F043FC95202A
:100F88004FF6E07107F03EFCC7204FF4FC6107F014
:100F980039FC4EF29C7003F057FF05200121002315
:100FA800324A04F08BF8052020210023304A04F04F
:100FB80085F80520522100232E4A04F07FF8842169
:100FC800002305202C4A04F079F84FF4F06003F070
:100FD8003BFFB6210520294A002304F06FF84FF69D
:100FE800FF7003F031FF264A8720DC210023BDE88B
:100FF800104004F063B810BDA5A00508D9A00508E5
:10100800D4A00508B3A50508D8A0050806A10508B9
:10101800F2A00508DDA00508EDA00508E2A0050876
:10102800E7A00508ECA00508F1A00508AFA0050891
:10103800F5A00508F9A00508FDA0050801A1050807
:1010480005A1050809A1050815A1050819A10508A4
:101058001DA1050820A1050829A1050825A1050845
:1010680024A1050828A105082DA1050838A105080F
:10107800FEA00508F6A005083CA10508CAA60508B3
:10108800CFA0050810B5064C06480623237000F0CB
:10109800FCFA2078FFF7DCFDBDE8104007F038BF08
:1010A800C04400207816002010B5064C06480723D7
:1010B800237000F0EAFA2078FFF7CAFDBDE8104077
:1010C80007F026BFC04400207816002010B5064C53
:1010D80006480523237000F0D8FA2078FFF7B8FDFA
:1010E800BDE8104007F014BFC04400207816002067
:1010F80010B5064C06480423237000F0C6FA207881
:10110800FFF7A6FDBDE8104007F002BFC04400206D
:101118007816002010B5064C06480323237000F00B
:10112800B4FA2078FFF794FDBDE8104007F0F0BE50
:10113800C04400207816002010B5064C064802234B
:10114800237000F0A2FA2078FFF782FDBDE8104076
:1011580007F0DEBEC0440020781600200E4A0123A6
:1011680010B513700D4A002414700D4A20461370F0
:1011780007F096F9204603F093FE0A4B04221A70F2
:1011880007F012FE07F0B0FE074B08481C70BDE8D8
:10119800104000F07ABA00BFC0440020140E0020AE
:1011A800110E0020443E002044460020B4100020C8
:1011B8000E4A012310B513700D4A002414700D4A0D
:1011C8002046137007F06CF9204603F069FE0A4BBD
:1011D80002241C7007F0E8FD07F086FE074B08485C
:1011E8001C70BDE8104000F050BA00BF1C0E002073
:1011F800140E0020C0440020443E00204446002035
:10120800E8130020034B01224FF4FC601A7003F02E
:101218001BBE00BF140E002070B5264C264E206859
:101228008EB04FF4784101F095F82068234901F019
:101238003FF809F04FFA22490246684612F0BEFF0D
:10124800204B21491A884FF6E07507A812F0B6FF1F
:101258006068294601F07EF86068694601F028F860
:10126800A068294601F076F807A9A06801F020F8DF
:1012780002F0AEF94FF47A6006F0EAFF20682946DA
:1012880001F068F82068314601F012F860682946D4
:1012980001F060F86068314601F00AF8A068294654
:1012A80001F058F8A068314601F002F802F090F910
:1012B8000EB070BD2C0D0020BA9F05083EA1050890
:1012C80052A10508AC3E002060A105080C4B10B5E2
:1012D80000220C4C1A7007F0F5FA04F079FD07F0BB
:1012E80022F907F0E9FA20684FF6E07101F032F8C8
:1012F8002068054900F0DCFFBDE8104002F068B93D
:10130800140E00202C0D00206AA105080E4B0022A7
:1013180010B51A700088C83880B2042805D90B485F
:101328000B4A0C4B992102F07BFB0B4CC0B204F02A
:10133800D9FD20684FF6E07101F00CF820680749E4
:10134800BDE8104000F0B4BF140E00207EA10508CF
:101358008CE003089EA105082C0D0020CFA10508EC
:101368000F4B002210B51A7009F0D2F9044628B1C3
:10137800FFF752FFBDE8104002F02AB903F090FDD4
:1013880007F0A0FA06F00AFF064B1C70064B012274
:101398001A7007F091FA0548BDE8104000F075B9D9
:1013A800140E0020C0440020443E00206C0F002092
:1013B8000E4B002210B51A7009F0AAF9044628B19C
:1013C800FFF72AFFBDE8104002F002B903F068FDFC
:1013D80007F078FA064B1C70064B02221A7007F0C9
:1013E8006BFA0548BDE8104000F04FB9140E002014
:1013F800C0440020443E0020FC1100200E4B002277
:1014080010B51A7009F084F9044628B1FFF704FFF3
:10141800BDE8104002F0DCB809F034F9204603F0CA
:101428003FFD064B064803221A7000F02EF9BDE86E
:101438001040FFF715BA00BF140E0020443E0020EC
:10144800A01200202DE9F04F6C486D4D89B00024A2
:1014580001F085FE4FF6FF71224623466948009445
:10146800019400F03BFF042607464FF6E071224640
:10147800234665480096019400F030FF4FF6E0716E
:1014880080462246234661480096019400F026FFD4
:101498004FF6FF718146224623465D480096019427
:1014A80000F01CFF4FF6FF7128602246234659487A
:1014B8000096019400F012FF234668604FF6FF7112
:1014C800224654480096019400F008FF5249A8604B
:1014D800524A204601F0FAFB5149524A82462046B8
:1014E80001F0F4FB5049514A8346204601F0EEFBD7
:1014F8004F4903904F4A204601F0E8FB4E490490BB
:101508004E4A204601F0E2FB4D4905904D4A2046DF
:1015180001F0DCFB4C4906904C4A204601F0D6FB12
:101528003A4607902146354B204601F0E7FCC82093
:1015380021464246314B01F0E1FC0A21C8204A46C7
:101548002E4B01F0DBFC55212A682C4B782001F04A
:10155800D5FC69216A68294B782001F0CFFC7820F6
:101568007D21AA68254B01F0C9FCC825052623273B
:10157800E0B204F0E7FB364A0146284601F0A6FB34
:1015880094FBF6F106FB114179431E31024689B2FC
:1015980000201A4B0134013501F0B0FC042CADB227
:1015A800E6D1D22152460520144B01F0A7FCD221E6
:1015B8005A464C20114B01F0A1FCD221039A0F4B43
:1015C8009C2001F09BFCD221049A0C4BEC2001F0EA
:1015D80095FCB421059A094BEC2001F08FFCB4214D
:1015E800069A064B9C2001F089FC079A034B4C2075
:1015F800B42109B0BDE8F04F01F080BC44130020CD
:101608002C0D0020DFA10508E9A10508F6A10508B1
:1016180001A20508B79F050815A20508D5120008FC
:101628001DA205080514000826A20508B91300081C
:101638002FA205086913000838A205080D12000832
:1016480041A20508B91100084AA205086511000859
:101658001513000808B500F04FFBFEF7CDFD00F0AC
:1016680083F8FEF7E5FFFEF72DFEFFF775FA00F0A9
:1016780001FDFFF7E7FEFEF765FE00F0EFFB00F067
:1016880047FABDE8084000F015BB10B5044628B974
:101698000F48104A104B492102F0C2F90F4B186845
:1016A800844213D010B1C36900219847002003F089
:1016B800F7FB002003F0DEFB4FF6FF7003F0C4FBDE
:1016C800E369204601219847044B1C6010BD00BF08
:1016D80053A205089BE003086FA20508380D0020F7
:1016E8000048D2E74413002008B5124B124A1B7871
:1016F8000D2B8CBF00210121117014225A430F4970
:1017080088588B184FF47A720D495043086059680D
:101718004A430C490A609A680B4B1A6006F07EFE31
:1017280007F0CAF8094B0A4800221A70BDE80840B9
:10173800FFF7ABBFAE3E0020280F002000000020BE
:10174800B03E0020CC440020A4440020443E0020A9
:1017580044130020024B034800221A70FFF795BF7C
:10176800443E0020441300202DE9F347384DDFF8AC
:10177800FC80384E0024284601F0F1FC224623461E
:1017880047F6FF7134480094019400F0A7FD4FF626
:10179800FF79042782464946224623464046009759
:1017A800019400F09BFD494630602246234640469E
:1017B8000097019400F092FD494670602246234646
:1017C80040460097019400F089FD2346B0604946E1
:1017D800224640460097019400F080FD1F49F060C2
:1017E8001F4A204601F072FA1E491F4A0746204642
:1017F80001F06CFA2146804652462B46204601F0FD
:101808007DFB3C2132682B465A2001F077FB5A2099
:1018180072682B46014601F071FB7821B2682B46AD
:101828005A2001F06BFB9621F2682B465A2001F0F2
:1018380065FBD2213A462B46EC2001F05FFB9C2049
:10184800D22142462B4602B0BDE8F04701F056BB14
:10185800B41000203C0D00207FA205088CA20508CA
:101868005D17000895A20508F1160008B79F05083E
:1018780070B5474E474C327847492DED028B1425F9
:1018880092B005FB02420C320FA812F097FC337895
:101898000D2B05FB03F504EB050332D8D3ED016AE4
:1018A8009B6807EE103A6359B8EEE68A06EE903A5E
:1018B800DFED3A7AF8EEC78AB8EEE67A88EE278A3C
:1018C800C8EEA78AC7EE277A17EE900A0DF010FF28
:1018D80002460B466846324912F070FC18EE100AB0
:1018E8000DF006FF02460B4605A82E4912F066FCCD
:1018F80018EE900A0DF0FCFE02460B460AA82A498B
:1019080029E093ED017A9B6807EE903A635906EE59
:10191800903AF8EEE78AF8EEE67AB8EEC78A17EE5C
:10192800900A0DF0E5FE02460B4668461F4912F084
:1019380045FC18EE100A0DF0DBFE02460B4605A822
:101948001B4912F03BFC18EE900A0DF0D1FE0B4635
:10195800184902460AA8184C12F030FC20681749AA
:1019680000F0A6FC20680FA900F0A2FC6068694698
:1019780000F09EFCA06805A900F09AFCE0680AA99E
:1019880000F096FC01F024FE12B0BDEC028B70BD95
:10199800AE3E0020000000209EA2050800007A4408
:1019A800A9A20508BAA20508CBA20508DCA2050869
:1019B800EDA20508FEA205083C0D0020C09F050801
:1019C8004FF6FF7070474FF6FF7070471FB500293C
:1019D80047D04FF2DE7003F063FA002003F036FBC5
:1019E8000F2003F031FA1F4C1F4A412101230A201E
:1019F80003F064FB042003F029FB236828209621C8
:101A0800042B24DC0123194A03F058FB03A90DF128
:101A18000E02206803F0D8FD0F2003F015FABDF878
:101A28000C00BDF80E1014380F242822002380B2B1
:101A3800009403F039FABDF80E10BDF80C000094BC
:101A4800143989B22822012303F02EFA09E0084A42
:101A5800012303F033FB1E20A521064A012303F0CE
:101A68002DFB1FBD4C0D00200FA3050822A3050860
:101A78003EA3050854A3050837B51E4C2368042B5C
:101A880005462BDC01A80DF1060103F09BFDBDF80E
:101A98000630BDF80420184904200AF0DDFE23684A
:101AA800002B04DA1548164A164B592105E0042B79
:101AB80005DD1248124A144B5A2101F0B1FF04EB1C
:101AC8008302BDF8041001339180BDF8061023602D
:101AD800052BD18008D1201D03F0F6FD00230B480B
:101AE8002360FFF7D2FD03E028460121FFF76EFFD0
:101AF8003EBD00BF4C0D00206BA30508B0A3050830
:101B0800ADE00308D2A30508E9A305088C1400205A
:101B180037B50B4C204601F022FB0A4B0A490093CB
:101B280000250120094A0A4B019501F0C0F9294610
:101B380002462346284603B0BDE8304001F0DEB92E
:101B480058110020D5190008C9190008CF19000834
:101B5800811A00084FF6FF7070474FF6FF70704704
:101B680030B54FF6E07087B003F09AF9002003F023
:101B78006DFA0F2003F068F900212C4A2C4C012340
:101B88000A2003F09BFA002003F05EF9042003F01A
:101B98005DFA0A201921274A012303F08FFA25212B
:101BA800254A01230A2003F089FA1F2003F04CF983
:101BB80001230A203721214A03F080FA2378002BD9
:101BC80031D001231E2096211D4A03F077FA62883E
:101BD8001C4902A812F0F2FA01231E20A22102AA2F
:101BE80003F06CFAA288184902A812F0E7FAAE21AD
:101BF80002AA01231E2003F061FA0F2003F024F942
:101C08006088A188143880B20F2528220023009507
:101C180003F04AF9A18860880095143989B228220E
:101C2800012303F041F907B030BD00BF17A4050830
:101C3800640D002029A4050849A4050869A405081D
:101C48008CA405089EA40508ABA4050801B187E784
:101C5800704713B50DF1060101A803F067FC144B9A
:101C680001221A705988BDF80420891A0E311C29DE
:101C780019460AD89C88BDF80600201A0E301C2880
:101C880003D899680131996001E000238B60084B03
:101C98009968012905DD00229A601A70FFF720FD76
:101CA80005E05A80BDF806209A80FFF759FF1CBD51
:101CB800640D002037B50B4C204601F050FA0A4B52
:101CC8000A49009300250120094A0A4B019501F0B1
:101CD800EEF8294602462346284603B0BDE83040C0
:101CE80001F00CB98C140020551C00085D1B00087D
:101CF800631B00085B1C000810B50B4C204601F064
:101D08002EFA00200146224600F048FB0020074931
:101D1800074A00F0DBFFD221024623464FF48270C7
:101D2800BDE8104001F0EAB878160020B8A405080C
:101D3800611D000870B5C9240AE0A8B20022314626
:101D4800013502F00BFAF02DF7D10134EF2C02D057
:101D58000025A6B2F1E770BD08B5FFF7EBFF064B0B
:101D6800186806F0C7F9054B054800221A70BDE847
:101D78000840FFF78ABC00BFA83E00201C0E0020C8
:101D88001010002010B5064C4FF6FF71206800F0C7
:101D9800E1FA044B20681968BDE8104000F088BAE1
:101DA800700D0020EC02002008B5002003F078F840
:101DB800054B1868054B196800F07AFA0448BDE825
:101DC8000840FFF762BC00BF700D0020E802002049
:101DD800441300200088A0F5C87080B2092808B50F
:101DE80005D90848084A094B8C2101F019FE084B0F
:101DF8001880084BFF21197006F032FABDE8084038
:101E0800C0E700BFBDA40508BFE00308E0A40508BB
:101E18001C1700201E1700200088A0F5967080B2BD
:101E2800092808B505D90848084A094B802101F056
:101E3800F7FD084B1880084B0121197006F010FABD
:101E4800BDE808409EE700BFBDA40508D4E003082C
:101E5800E0A405081C1700201E170020F7B5002471
:101E68003348344D01F07BF9224623464FF6FF7183
:101E780031480094019400F031FA042622462346A2
:101E880007464FF6FF712D480096019400F026FA98
:101E98002346286022464FF6FF7128480096019491
:101EA80000F01CFA26496860264A204600F00EFF1A
:101EB800214606463A4620461D4B01F01FF82A687F
:101EC8001B4B2046282101F019F83246AA20D221BE
:101ED800174B01F013F80F254FF4967440F235169E
:101EE80020461949194A00F0F1FE013402467821CA
:101EF80028460F4BA4B2233501F000F8B442ADB226
:101F0800EED10F254FF4C87440F2991620461049B7
:101F1800104A00F0DBFE013402469B212846044BA0
:101F2800A4B2233500F0EAFFB442ADB2EED1FEBD53
:101F3800D4150020700D002011A50508C89F0508BC
:101F48001DA50508B11D000826A50508211E0008C5
:101F580028A50508DD1D000808B5FFF713FF0020B8
:101F6800014606F07DF9BDE8084001F031BB00BF2D
:101F780010B506F021FF194B194A00241C700220E5
:101F88002346CA2103F09AF8204606F089FA154B31
:101F98001C80154B1C70154B1B78023B052B1CD85D
:101FA800DFE803F003070B13170FBDE81040FFF736
:101FB800C3B8BDE81040FFF7ADB8BDE81040FFF763
:101FC80097B8BDE81040FFF76FB8BDE81040FFF7BD
:101FD8007DB8BDE81040FFF755B810BD1C0E0020B5
:101FE800B69F05082445002044460020C044002030
:101FF80008B5084B01221A70074B186806F07AF8E2
:10200800002002F04DFF06F0CFFE0448BDE808406E
:10201800FFF73BBB1C0E0020A83E0020E813002061
:1020280038B50D4B0D4D00241C700D4B1C700D4B1D
:10203800186806F05FF8204602F032FF0A4B1B785A
:10204800022B0CBF09480A48FFF71FFB2C70BDE89C
:10205800384006F0A9BE00BF1C0E002044460020F0
:10206800C0440020A83E0020443E0020FC1100206F
:102078006C0F00202DE9F041144C204601F06FF858
:1020880000201349134A00F021FE1349134A07465A
:10209800002000F01BFE1249124A0646002000F0FC
:1020A80015FED22105463A462346E62000F026FFD3
:1020B8004B2132462346642000F020FF642069212A
:1020C8002A462346BDE8F04100F018BF1010002052
:1020D80091A00508292000082AA50508F91F00086D
:1020E80036A50508791F000808B508B143682BB95B
:1020F8000348044A044B9B2101F092FC586908BD2F
:1021080043A50508E8E0030865A5050808B5FFF735
:10211800EBFF8068123080B208BD08B5FFF7E4FF16
:102128004068063080B208BD2DE9F84F044688465D
:10213800FFF7DAFF6689E589074606F1030905F125
:102148000F0AB8F1000F1FD01F2002F07DFE2046B5
:10215800FFF7DCFF83462046FFF7DFFF29460346EB
:102168005FFA8BF2F0B202F0AFFE042002F06EFFCD
:102178000B364FF6FF70033502F066FEB0B2A9B217
:102188003A68012302F09AFF3D69204641464A46D3
:102198005346A847BDE8F88F13B504460DF106016C
:1021A80001A803F0C3F92046FFF79EFF6389BDF835
:1021B8000410BDF80620C91AE389D21A0339C36886
:1021C8000F3A204698471CBDF7B5044614200D4623
:1021D80016461F4611F080FC089BC7600361064B3A
:1021E8000649074A80E8700000930190054B0020DB
:1021F80000F05DFEFEBD00BF31210008232100086C
:1022080015210008A1210008704708B508B14368E6
:102218002BB90448044A054BAD2101F001FC58696B
:1022280008BD00BF84A5050800E1030865A50508E9
:10223800F8B505460E46FFF7E8FF836B04461BB169
:1022480028463146984700E018466F8994F83C3094
:10225800ED890EB9034310D0208E02F0F5FD608E93
:1022680002F008FE94F8350002F0F0FE94F83430DD
:1022780038462946224602F021FF002384F83C30E4
:10228800F8BD08B5FFF7C1FF90F83500BDE8084074
:1022980002F0F1BE38B5FFF7B8FF044612F014F8A3
:1022A800054694F8350002F0E1FE684380B238BD77
:1022B80038B50D46FFF7A9FF29462E22044612F02D
:1022C80033F850B1204629462E2212F07FF8002319
:1022D80084F82E30012384F83C3038BD2DE9F743CB
:1022E800074640200E461546984611F0F5FB044671
:1022F80028B91148114A124B4E2101F091FB114B9C
:10230800114A12498DE818000020114B00F0CFFD4A
:1023180039468146FFF7CCFF9DF82830268684F899
:1023280035300B9B6586A363002384F8348084F8DA
:102338003C304846BDE8FE8384A5050818E103083B
:10234800A2A50508392200088B2200089D22000852
:102358001122000810B50C46FFF757FF0123048629
:1023680080F83C3010BD00BF4FF4A0707047C82003
:1023780070477047074B1B78022B07B508D1064BEF
:102388001B78022B04D001A80DF1060103F0CEF84A
:102398000EBD00BF44460020C044002073B50A4B60
:1023A80006460D461446009300200849084A094B82
:1023B800019000F07CFD294602462346304602B0D3
:1023C800BDE8704000F09ABD7B2300087123000827
:1023D800772300087D23000813B502AB03E9060044
:1023E800436843B1027C0124082A9C7004D11B690C
:1023F8002146984700E01C4620461CBD30B5002801
:102408002BD0058B002425E0036A1A7C012A05D10C
:102418005B681A888A421BD1187F30BD052A06D10D
:102428005B681A888A4213D193F82C0030BD032ABE
:1024380006D15B681A888A420AD193F8250030BD14
:10244800062A05D15B681A888A4201D1D87A30BD3C
:1024580001340430AC42D7D3002030BD08B18175B7
:1024680001207047F8B504460D46D0B1E175D0F8A3
:1024780098309847012D0DD12746002606E0F869C7
:1024880000F10802436906CA98470136238B0437CE
:102498009E42F4D3D4F89830204629469847012024
:1024A800F8BDF8BDF8B50546084617460E4611F0C2
:1024B8000BFF013FB84234BF04463C463CB12846B6
:1024C8003146224611F082FF00232B55F8BD2C70AF
:1024D800F8BDF7B5044600200090019000296CD0A3
:1024E8000E8B68E000F1080351F823301D7C042DA1
:1024F80004D15D682D88954247D0013000F108036A
:1025080051F823301D7C012D04D15D682D8895423A
:102518003BD0013000F1080351F823301D7C052D14
:1025280004D15D682D8895422FD0013000F1080351
:1025380051F823301D7C032D04D15D682D88954208
:1025480023D0013000F1080351F823301D7C022DFF
:1025580004D15D682D88954217D0013000F1080339
:1025680051F823301D7C072D04D15D682D8A9542D2
:102578000BD0013000F1080351F823301D7C062DE3
:1025880008D15D682D88954203D103F108012046E2
:1025980015E0013000F1080351F823502B7C082B7B
:1025A80009D16F683F88974204D105F10801204698
:1025B8001A4605E00130B04294D320466946082205
:1025C80011F03AFD2046FEBDF8B505460F46164601
:1025D800002830D04388032B2FD0202011F07CFA1C
:1025E800044600282BD040F80C5B39460C22FFF734
:1025F80059FF1820E66111F06FFA0646B8B10223B8
:102608000374012363760F4B446063600E4BA36031
:10261800002323766B8805EB830201339BB2012BE1
:1026280050606B800CD16A685268137608E02046C7
:1026380011F05AFA04E0064602E0002600E00646D9
:102648003046F8BD64600408025D040837B5456883
:1026580002AB03E906003DB3037C0124042B85F893
:10266800314022D1688E02F0EFFB95F8300002F07D
:10267800EDFC95F8343043B9BDF80200BDF80610FA
:10268800AA1C234602F01AFD0FE0012B03D10848CB
:1026980040F2395104E0022B07D1054840F241517C
:1026A800044A054B01F0BCF92C4620463EBD00BF4C
:1026B800B5A50508D82B0408B3A50508F8B5044640
:1026C8000F46164610B3838A0A2B20D0202011F01B
:1026D80003FA0546E8B14460102200F108003946C3
:1026E800FFF7E0FE4FF6FF73A08A2B801F236B8055
:1026F80000232B76831D013080B20128EE6144F857
:102708002350A08207D1A3691876F8BDF8BD002030
:10271800F8BD0120F8BD0120F8BD2DE9F3471D469D
:102728004B1C984282460C461746BDF828600DDDC2
:1027380095420BDC01320AF101035B1A521BC8B245
:10274800D2B29BB22946009602F0B6FBAAF1020A61
:102758003046C4EB0A0A02F077FB4FF000084FF04E
:1027680001091FFA8AFA0BE0601C08EB050180B228
:1027780089B252460023009602F096FB09F101093E
:102788007B1B08F1010899451FFA88F8ECD3BDE8CE
:10279800FC87F8B5C7B2144638461E460D4602F007
:1027A80095FB621E92B23846294602F08FFB3046EE
:1027B80002F04AFB022606E0A21B92B238462946DE
:1027C80002F084FB0136A642F6D3F8BD73B5044681
:1027D8000E4600F11E001546009200233C2280B2EE
:1027E8001E3E02F061FBB1B220463C220123009557
:1027F80002F05AFB7CBD73B504460E4601381546F7
:1028080000920023032280B2013E02F04DFBB1B2D8
:10281800204603220123009502F046FB7CBDF7B554
:10282800089D2E7BEF7A1C463604AB7A06EB07260A
:10283800F618431A687B06EB00602D1800200190FB
:10284800121B08462146009501F026FFFEBD30B553
:10285800456885B004AB03E906007DB101242C73FB
:102868006D68BDF80800BDF80A109DF80C209DF8A9
:102878000E300095FFF7D3FF204600E0284605B04C
:1028880030BD2DE9F04385B004AB03E90600446888
:10289800BDF80860BDF80C70002C41D0012384F805
:1028A800263094F825300BB9A26800E06268FFB2C0
:1028B800BDF80A109DF80E30009230463A46FFF7F0
:1028C800AEFF04F10C08022002F0C0FB404611F0F4
:1028D800FBFC054600B1451E0F3F0024153E1FFABC
:1028E80087F90DE002F0BCFB02F0C0FB04FB1061AD
:1028F80089B248462022002302F0FAFB0134E4B2F0
:10290800AC42EFD3002002F09FFAB8B2B1B242460F
:10291800012302F0EDFB002002F098FB012000E00B
:10292800204605B0BDE8F0832DE9F04385B004AB3F
:1029380003E906004568BDF80860BDF80C70002D75
:102948003CD001236B762B7EBDF80A10012B0CBFFF
:102958006A68AA689DF80E300092FFB23A4630467F
:10296800FFF75DFF0C35022002F070FB284611F0DE
:10297800ABFC0E3F81460024163E1FFA87F80DE097
:1029880002F06EFB02F072FB04FB106189B2404654
:102998002022002302F0ACFB0134E4B24C45EFD90D
:1029A800002002F051FAB8B2B1B22A46012302F06F
:1029B8009FFB002002F04AFB012000E0284605B0FA
:1029C800BDE8F0832DE9F04F85B00546DDF840906D
:1029D800029148469046039311F076FCDDF838A042
:1029E800DDF83CB00646294600242F4611E024B104
:1029F800B4420CBF5B46534600E0039B01F1080557
:102A0800ADB200932846029A4346FFF708FF013407
:102A18002946B442EBDD002002F016FA022002F04B
:102A280015FB7D1D08F10508A8B21FFA88F14A4672
:102A3800012305B0BDE8F04F02F040BB70B5406817
:102A480086B006AB03E9060000282ED0012380F8E3
:102A58002D308668164BF21A534243EB020390F866
:102A68002C205AB1002B134D134B144A08BF1D4696
:102A7800134B00F11C0418BF13460AE0002B0D4D40
:102A88000D4B0E4A18BF1D460D4B00F10C0408BF34
:102A98001346BDF81200BDF81410BDF816200096B4
:102AA80001950294FFF78EFF012006B070BD00BFAC
:102AB80048350408843104082A37040866330408B2
:102AC8000C39040870B5446886B006AB03E9060003
:102AD80004B301236377A668104B227FF11A4B4297
:102AE80043EB01030AB10BB904E01BB966680C4D4E
:102AF8000C4B01E00C4D0D4BBDF81200BDF8141045
:102B0800BDF8162000960C3401950294FFF75AFF81
:102B1800012000E0204606B070BD00BF94400408C4
:102B2800D03C0408B23E04086A4204084044040841
:102B38002DE9F04385B004AB03E906004468BDF80D
:102B48000860BDF80A90BDF80C50BDF80E80002C46
:102B580000F08C800123A3740220676802F076FAE3
:102B68004FF6FF7002F086F9002002F06DF9EDB221
:102B78005FFA88F8A6F1160189B230462A4643461C
:102B88000097FFF74CFE277A002F2ED1A28A234602
:102B980000E00137974204D29969097E043300297D
:102BA800F7D002F05DFA02F061FAA9F116091FFAEE
:102BB80089F90E2101FB10914FF6FF7208F1010807
:102BC8005FFA88F389B2009248462A46FFF7A5FDC6
:102BD800022002F03BFA1F2002F036F9A38A002BEC
:102BE80038D0103DE8B2303E2CE0E3685C68A28A39
:102BF8002346013A002700E00137974204D2996939
:102C0800097E04330029F7D002F02AFA02F02EFADE
:102C18000E2101FB10914FF6FF7208F101085FFACF
:102C280088F389B2009248462A46FFF776FD0220CB
:102C380002F00CFA1F2002F007F9A38A53B1103DE5
:102C4800E8B21A3E0637B1B254F8272001230832F9
:102C580002F04EFA002002F0F9F94FF6FF7002F088
:102C680009F91F2002F0F0F8012000E0204605B025
:102C7800BDE8F0832DE9F041054636208846144624
:102C88001F4610F029FF0646E0B120F8025B4146D6
:102C98002E22FFF707FCBDF8183086F834407386FB
:102CA8001820012386F8307086F8313010F014FFB0
:102CB800044618B104234660037404E0304610F05B
:102CC80013FF00E004462046BDE8F081F8B506464B
:102CD80024200F46154610F0FFFE0446D8B10F4BCE
:102CE800068083600E4B39464360102200F10C00C9
:102CF800FFF7D8FB01260023182025622377667783
:102D080010F0EAFE054610B14460067404E020465F
:102D180010F0EAFE00E005462846F8BD9440040895
:102D2800EE3A0408F8B506462C200F46154610F072
:102D3800D3FE0446E8B120F80C6B39461922FFF798
:102D4800B1FB0D4BA562A3600C4B6360002384F8B4
:102D580025301820012384F8263010F0BDFE0546E2
:102D680018B103234460037404E0204610F0BCFE4D
:102D780000E005462846F8BDA05904083E56040858
:102D880010B50446142010F0A7FE20B1002343809C
:102D9800014B0480036110BDD125000838B50546F4
:102DA800442010F099FE0446C0B10E4B05824360E2
:102DB8000D4B0360012383740023037283820B4B42
:102DC8000364182010F088FE054618B107234460F4
:102DD800037404E0204610F087FE00E0054628460C
:102DE80038BD00BF345204082A4E0408C52600081E
:102DF8002DE9F04105463420884614461F4610F058
:102E08006BFE064620B3144B05808360134B414686
:102E18004360102200F10C00FFF744FB214606F145
:102E28001C001022FFF73EFB002386F82C301820E8
:102E38000123376386F82D3010F04EFE044618B192
:102E480005234660037404E0304610F04DFE00E0B0
:102E580004462046BDE8F08148350408A22F04083E
:102E68002DE9F041044614200D461646984610F008
:102E780033FE0746B8B1069B048003610023C37282
:102E880001234560068180F80A800373182010F03A
:102E980023FE044618B106234760037404E038464D
:102EA80010F022FE00E004462046BDE8F0812DE93E
:102EB800F041044618200D461646984610F00CFEC0
:102EC8000746B8B101238370069B04800361079B02
:102ED80045608660C0F80C804361182010F0FCFD46
:102EE800044618B108234760037404E0384610F01C
:102EF800FBFD00E004462046BDE8F0812DE9F341E2
:102F080098461B8B1D2B05460C4617464FF00000B4
:102F180000F2B480B5F5A07F0090019000F2AE8079
:102F2800F02900F2AB80127CADF80610511EADF806
:102F38000250072900F28A80DFE801F045595E0453
:102F4800456A14767B684E4A7A611A8893F8343059
:102F58003A80013BDBB2012B7FD8ADF80240ADF8D7
:102F680006507AE005F11602ADF8002004F11602C9
:102F7800ADF8042002AE434A16E903007A6107F16E
:102F8800080282E8030003F10802013348F82270BE
:102F9800A8F818307B681A8A187A3A8000286CD109
:102FA800FFF7FCFE3849436859603849DF6001265D
:102FB800163D196002461E72A8B2E1B24346FFF7F9
:102FC8009DFF30465AE0012A0CBF314B314B7868DF
:102FD8007B6130F80C3B3B8011F076F9431CDB0039
:102FE8001A34ED18ADF80440ADF8005035E07B68B0
:102FF800294A1B687A6102E0284A7B687A611B8843
:1030080014353B80ADF800501434ADF8044024E08A
:103018007B68234A7A611A883A801A899B7AAD18A4
:10302800ADF80050E418F0E77E681E4B7B613388EA
:1030380038463B8073689847013D4519ADF8005004
:10304800B36838469847013C0419DEE71648174A22
:10305800174B40F21A3100F0E3FC02AA12E9030010
:1030680007F1080383E80300B8F8183003F10802F1
:10307800013348F82270A8F818300120BDE8FC8117
:1030880055260008392B0008204A0408164604086B
:10309800CD2A0008452A0008312900088B28000895
:1030A80057280008E1230008B5A50508E82B0408FF
:1030B800B3A50508F8B51646002834D01378002BB8
:1030C8002ED0028B002327E0046A257C042D21D111
:1030D80065682F888F421DD195F8313053B16F8EB6
:1030E80001F0D8FE04F1080268866369204606CA22
:1030F80098476F86A81C31462E22FFF7D3F995F81A
:1031080031307BB104F108026369204606CA98474A
:103118000120F8BD013304309342D5D30020F8BD17
:103128001846F8BD0120F8BD70B5B8B1068B044645
:10313800002310E0256A287C04280AD16D682888B5
:10314800884206D11046A91C2E22FFF7ABF90120B0
:1031580070BD01330434B342ECD3002070BD38B5E0
:10316800044620B3134BC361134BC0F89830134B7C
:10317800C0F89C30124B00257822C0F8A030857525
:10318800C5750583294600F1200010F097FFD4F893
:1031980098302046294698470A4A1388312B07D881
:1031A800094941F8234001331380012038BD38BD57
:1031B800284638BD6D240008652400080524000849
:1031C800DB240008780D0020201700202DE9F041AD
:1031D8000446002800F0B380078B02460025A8E0CB
:1031E800136A1E7C042E00F08780012E23D15868B4
:1031F80003888B4240F09B8005F1080710F074FCAF
:1032080054F827004FF00008C0F8048010F06CFC58
:10321800228B531E9D4208D00732238354F8221074
:1032280044F8271044F8228002E044F827802583D8
:103238003046BDE8F081052E5ED0032E5CD0022E0C
:1032480013D15B68186803888B4270D14388013BAF
:103258009BB243800BB910F047FC05F1080654F8FF
:103268002630586810F040FC4EE0072E21D15E68E9
:10327800338A8B425BD1002706E0BB1D013756F825
:10328800230010F031FCFFB2B38ABB42F5D8002707
:10329800B78205F1080654F82630586810F024FC67
:1032A80054F8260033E044F8267025830120BDE851
:1032B800F081062E1ED1586803888B4237D105F15C
:1032C800080610F011FC54F826000027476010F09B
:1032D8000BFC228B531E9D4209D00833013A54F847
:1032E8002310228344F8261044F82370DEE744F8BC
:1032F80026701AE0082E1AD1586803888B4216D116
:1033080010F0F2FB05F1080654F826000027476084
:1033180010F0EAFB228B531E9D42C4D0073254F8AA
:10332800221044F8261044F822702383BEE70135A2
:103338000432BD42FFF454AF0020BDE8F081BDE87F
:10334800F08170B5044600282AD0068B751E083611
:1033580000EB86061EE056F8043D1A7C042A13D0BA
:10336800012A11D0052A0FD0032A0DD0022A02D132
:103378005B681B6809E0072A02D15B68198A05E0C7
:10338800062A01D0082A04D15B6819882046FFF76D
:103398001DFF013D681CDED100232383012070BD81
:1033A80070BDF0B528B30023068B1A461EE0046AE8
:1033B800257C072D18D16468258A8D4214D1A78AE7
:1033C800002504EB83040DE004EB050C0435DCF860
:1033D80018C09CF818C0BCF1010F03F1010301D11A
:1033E800D8B2F0BDBB42EFD301320430B242DED3D3
:1033F8000020F0BD70B508B3048B00231BE0026AFF
:10340800157C072D15D15268158A8D4211D10023DC
:10341800958A11461C46012007E013B99669307653
:1034280001E08E69347601330431AB42F5D30120D3
:1034380070BD01330430A342E1D3002070BD2DE9F3
:10344800F04128B30023078B1A461EE0046A257C46
:10345800072D18D16468258A8D4214D1B4F814C098
:10346800002504EB83040CE066190435B66996F868
:103478001880B8F1010F03D106F10800BDE8F0810A
:1034880001336345F0D301320430BA42DED3002061
:10349800BDE8F0812DE9F04700282FD00023B0F8CF
:1034A80018C01D4627E0046A267C072E21D16468CF
:1034B800268A8E421DD1B4F81480002604EB8309B5
:1034C80015E009EB0604A7693C7E012C0DD192F8A2
:1034D80000A0BAF1000F08D007F108001146102229
:1034E800FEF7E0FF2046BDE8F08701330436434588
:1034F800E7D3013504306545D5D30020BDE8F08712
:10350800F0B5B0B1068B002510E0046A277C062FC1
:103518000AD1646827888F4206D123819DF8143028
:103528006260A3720120F0BD01350430B542ECD3CE
:103538000020F0BD10B500210446FEF793FF204699
:103548000121BDE81040FEF78DBF38B598B1048B56
:10355800024600230CE0106A058804328D4206D129
:1035680000F10802436906CA9847012038BD0133B3
:10357800A342F0D3002038BD10B50C460021FEF759
:1035880071FF20460121BDE81040FEF76BBF13B55F
:1035980002AC04E90C00BDF80230834206D8BDF83D
:1035A8000030834234BF0020012000E00020BDF835
:1035B80006308B4206D8BDF804308B4234BF002158
:1035C800012100E00021002818BF0846C0B21CBD38
:1035D80038B5114B114A1988002319E052F8045FD5
:1035E800A87D012812D100240CE004F1080355F845
:1035F8002300037C082B03D1436800211B699847EB
:103608000134A4B22B8BA342EFD838BD01339BB24F
:103618008B42E3D138BD00BF780D00201C17002075
:10362800704770B5094CA5787DB9094B1E78012EF5
:103638000BD16368013363606268064B9A4204D910
:10364800284601F0C5FCA670656070BD780D0020A5
:103658008401002040420F00054A9060134602E0B2
:1036680099680139996091680029F9D1704700BFBC
:10367800780D0020F0B585B001F056FF002800F065
:103688004981002502A80DF10A01ADF80850ADF8EE
:103698000A5001F04BFF03A80DF10E01ADF80C50D4
:1036A800ADF80E5001F08EFFBDF80C10BDF80820E3
:1036B8000091BDF80E10BDF80A3001912C46964DC8
:1036C8009649082009F0C8F8A878012803D101F024
:1036D8007FFCAC7019E1924B5B78012B40F01581AF
:1036E800AB78002B40F011816B6029888D4A09E185
:1036F80052F8046FB07D012840F002810025FAE0FD
:1037080005F10803BDF8080056F82340BDF80A1073
:1037180004F108030CCBFFF73AFF002800F0E9801A
:10372800237C013B062B00F29F80DFE803F004298D
:10373800159D1F9D4C006668012304F10805337729
:1037480095E80600636920469847002333772046AA
:10375800636995E8060086E0636893F8252012F10E
:10376800FF3218BF012283F8252077E0636893F8B9
:103778002C2012F1FF3218BF012283F82C206DE0B3
:103788006268137E1568002B6ED16E882F46294615
:10379800184606E051F804EFDEF804E001338EF82D
:1037A8001800B342F6D301231376002607E057F832
:1037B800040F00F10802436906CA984701366B886E
:1037C8009E42F4D350E0656820892E68A37B227B53
:1037D8000096A0F1160189B2FFF721F81420FFF72F
:1037E8003BFF2B7AC3B9AF8A29461A461E4609E021
:1037F800886990F818E00676BEF1010F08BF1346F5
:1038080004310132BA42F3D301220BB9AB6924E087
:10381800053355F8233020E06368DB685A680023D5
:10382800908A154619461F4609E0AE6996F818E0D1
:103838003776BEF1010F08BF0B46043501318142CE
:10384800F3D3411E8B4203D1053052F8203003E0F8
:1038580004D2073352F8233001221A7604F1080201
:1038680006CA636920469847237C013B072B4CD83E
:10387800DFE803F00410074B0A0D123A63681B6A6D
:1038880034E063689B6A2DE063681B6B2AE0636819
:103898001B6927E0636824E063681A7A7AB9988A12
:1038A8001946013800E00132824204D28C69247E34
:1038B8000431002CF7D0063253F8223011E0DB68CF
:1038C8005A68908A11460138002300E00133834288
:1038D80004D28C69247E0431002CF7D0063352F8C8
:1038E8002330DB69984710E06368DB682046984717
:1038F8000BE00135ADB2338BAB423FF601AF04E0CC
:1039080001339BB28B427FF4F3AE01F053FE0F20DC
:10391800FFF7A2FE05B0F0BD780D0020DBA5050875
:10392800840100201C170020034B9A6812B19A6882
:10393800013A9A60704700BF780D00202DE9F347DF
:103948000120DFF8D080DFF8D09001460AF01EFB96
:10395800012400254FF480760227404669460096E8
:103968008DF804708DF805408DF806508DF80740E5
:1039780009F064FF40460821224609F0DFFF244B86
:10398800DFF898801A6844F2A243B2FBF3FA0AF10E
:10399800FF3A204621461FFA8AFA0AF027FBC8F8A0
:1039A80004A048464146A8F80050A8F80250A8F8D4
:1039B800085088F80A500AF0B5FE7023A8F80C30B1
:1039C8000423A8F810300AF1FF3A6323642203FBAA
:1039D8000AF3B3FBF2F39BB2C8F8143008F10C01F8
:1039E8004846A8F80E40A8F81870A8F81A50A8F881
:1039F8001C60A8F81E500AF0B3FF484621460AF09A
:103A080026FF484621460BF02CFABDE8FC8700BF8C
:103A1800F00200200000024000000140880D002054
:103A280083B50E460746154910201C46154608F072
:103A380013FF1020124908F00FFF1020114908F059
:103A48000BFF10200E4908F007FF002310200E4935
:103A5800019308F001FF334610200C493A4608F05C
:103A6800FBFE10200A492A4608F0F6FE10200949F4
:103A7800224608F0F1FE019B0133E7E715A6050889
:103A88001AA605083AA605084AA605085AA605086A
:103A98006FA6050880A6050808B5164B1A6A0132F4
:103AA8001A621A6A012A1A4603D0134840F21D21E5
:103AB8000FE05862194602E04B6A013B4B62506ABC
:103AC8000C4B0028F8D11A6A012A06D00A484FF48C
:103AD8000A710A4A0A4BFFF7A3FF1A6A013A1A62E7
:103AE8001B6A2BB10448054A064B40F22A21F2E72B
:103AF80008BD00BF880D002091A60508C66304080C
:103B0800BBA60508CCA6050810B5084C0221002262
:103B1800204609F008FF44F6FF70FFF7BDFF204676
:103B280002210122BDE8104009F0FDBE0004024058
:103B38000C4B0D491A6844F2A2436428B2FBF3F314
:103B4800D4BF20EAE0706420013B9BB24B60013B8C
:103B580058436422B0FBF2F080B2486103480C314C
:103B68000AF081BEF0020020880D0020000001400C
:103B780010B5134B93F828202AB11248124A134B58
:103B88004FF442710EE0012283F8282066234FF09B
:103B9800C042013BDBB2108033B90A480A4A0C4BD9
:103BA80040F21231FFF73CFF1488A4B28442F0D1EE
:103BB800084B1980024B002283F8282010BD00BF53
:103BC800880D002091A60508D0630408DDA6050825
:103BD800B3A505080000026010B5FFF7AFFE64202A
:103BE800FFF7A6FF21210720FFF7C2FF3220FFF7CA
:103BF80053FF01210020FFF7BBFF3220FFF74CFFE6
:103C080023210720FFF7B4FF3220FFF745FF0021EB
:103C18001020FFF7ADFF41F28830FFF73DFF332159
:103C28000720FFF7A5FF3220FFF736FF112046F6E1
:103C38003001FFF79DFF3220FFF72EFF4FF4C061E0
:103C48000220FFF795FF3220FFF726FF122046F6E5
:103C5800EB41FFF78DFF3220FFF71EFF03204AF6E6
:103C6800A401FFF785FF3220FFF716FF00210C2083
:103C7800FFF77EFF3220FFF70FFF0D2040F60C0103
:103C8800FFF776FF3220FFF707FF0E204FF42C5185
:103C9800FFF76EFF3220FFF7FFFEB0211E20FFF76F
:103CA80067FF3220FFF7F8FE012042F63F31FFF7A9
:103CB8005FFF3220FFF7F0FE05200021FFF758FFD5
:103CC8003220FFF7E9FE00210620FFF751FF3220DE
:103CD800FFF7E2FE16204EF61C71FFF749FF32206F
:103CE800FFF7DAFE172040F20311FFF741FF3220F9
:103CF800FFF7D2FE00210B20FFF73AFF3220FFF733
:103D0800CBFE00210F20FFF733FF3220FFF7C4FE60
:103D180041200021FFF72CFF3220FFF7BDFE422093
:103D28000021FFF725FF3220FFF7B6FE00214820CB
:103D3800FFF71EFF40F23F143220FFF7ADFE214689
:103D48004920FFF715FF3220FFF7A6FE00214A2081
:103D5800FFF70EFF3220FFF79FFE00214B20FFF7F1
:103D680007FF3220FFF798FE44204FF46F41FFF71A
:103D7800FFFE3220FFF790FE00214520FFF7F8FEF6
:103D88003220FFF789FE21464620FFF7F1FE322058
:103D9800FFF782FE302040F20771FFF7E9FE32207C
:103DA800FFF77AFE31204FF40171FFF7E1FE322070
:103DB800FFF772FE32204FF40171FFF7D9FE40F28F
:103DC80002543220FFF768FE21463320FFF7D0FE69
:103DD8003220FFF761FE342040F20751FFF7C8FE9A
:103DE8003220FFF759FE35204FF40171FFF7C0FE6E
:103DF8003220FFF751FE36204FF40171FFF7B8FE6D
:103E08003220FFF749FE21463720FFF7B1FEA4F51F
:103E180000743220FFF740FE21463A20FFF7A8FE43
:103E28003220FFF739FE2F2041F2BE21FFF7A0FE16
:103E38003220FFF731FE21463B20FFF799FE322062
:103E4800FFF72AFE00212320FFF792FE3220FFF71A
:103E580023FE00212420FFF78BFE3220FFF71CFEF3
:103E680025204FF40041FFF783FE3220FFF714FEB0
:103E780000214F20FFF77CFE3220FFF70DFE4E2079
:103E88000021FFF775FE3220BDE8104004E608B5B2
:103E9800124B93F829202AB11148124A124B40F2CA
:103EA80022310FE0012283F82920222166234FF0D6
:103EB800C042013BDBB2118033B90948094A0B4BB8
:103EC80040F23B31FFF7ACFD108880B22228F0D1D8
:103ED800024B002283F8292008BD00BF880D00206E
:103EE80091A60508DD630408DDA60508B3A5050845
:103EF80010B51E4B032826D8DFE800F0021A080E7A
:103F08001C8841F2280246F628000AE01C8841F283
:103F1800080246F6080004E01C8841F2300246F622
:103F2800300049F241318C4214BF014611460BE082
:103F3800188846F6200249F24131884214BF1146DA
:103F48004FF4815100E000211B8848F68912934202
:103F580005D049F22032934204D1032000E0112019
:103F6800FFF706FEBDE8104091E700BF860100207C
:103F7800014B18800A208FE5000002604FF0C04313
:103F8800188003F500331A881A88188880B2704799
:103F98004FF0C04322221A8003F5003382B01A88FA
:103FA80092B2ADF806201B889BB2ADF80630BDF87A
:103FB800060080B202B07047072040F27311D7E5BF
:103FC80007200021D4E582B0044BADF80600BDF807
:103FD800062092B25A8502B0704700BF880D0020B3
:103FE80082B0044BADF80600BDF8062092B25A80A4
:103FF80002B0704786010020014B80B218807047DC
:10400800000002604FF0C04380B218807047024B36
:1040180080B21880704700BF000002604FF0C043B4
:1040280080B218807047024B80B21880704700BF7A
:104038000000026082B0044B0190019ADA62DA6AE9
:10404800002AFCD102B07047880D002070B54FF0EF
:10405800C0452A242C800A4C060AC0B2268020803B
:10406800100AD2B2208022802B222A800A0A2280BB
:10407800C9B21A0ADBB221802280238070BD00BF3A
:104088000000026010B50B4614460246FFF7DEFF3B
:104098004FF0C0432C22A0B21A80BDE8104067E759
:1040A800114B1B8848F68912934210B504460BD071
:1040B80049F22032934212D1C1F1EF01202089B296
:1040C800FFF756FD212006E0C1F1EF014E2089B22D
:1040D800FFF74EFD4F202146BDE8104048E5024657
:1040E8000B46BDE81040B1E78601002008B5FFF790
:1040F800D7FF0F4B1B78012B4FF0C0420D4B0FD150
:104108002E2111801A881A881B8892B202F0FC00AE
:1041180002F4784242EAC000C3F3C423184308BD3E
:10412800222111801A881A88188880B208BD00BF19
:10413800F01700200000026070B5074D0646012404
:1041480021463046FFF7D2FF0134A4B2C82C25F827
:10415800020FF5D170BD00BF4646002010B5084BD0
:104168001B78012B144602D1BDE810408AE7FFF7FF
:1041780097FFFFF78CFE2046BDE81040F8E600BF29
:10418800F017002070B5074D06460124214601347A
:1041980035F8022F3046A4B2FFF7E0FFC82CF5D15E
:1041A80070BD00BF4646002070B505460E46FFF7B5
:1041B800C3FF01242146013428463246A4B2FFF742
:1041C800CDFFC82CF6D170BD2DE9F04104460D464F
:1041D8001646BDF81880032B39D8DFE803F00B35F5
:1041E8001927381980B2294642460137FFF7B6FF2A
:1041F800BFB200E00027B742F3D1BDE8F081E01B71
:1042080080B2294642460137FFF7A8FFBFB200E057
:104218000027B742F3D1BDE8F081E91B89B22046F7
:1042280042460137FFF79AFFBFB200E00027B742C6
:10423800F3D1BDE8F081791989B2204642460137A9
:10424800FFF78CFFBFB200E00027B742F3D1BDE80B
:10425800F08170B5194B1A4A598E92F900406418CA
:104268000025A4B28AB0AC4208BF0124C62C28BFDE
:10427800C62415700F264FF6FF721E865C865A8577
:1042880019202B46009221460A22FFF79DFF21465E
:104298003046FFF72BFF224603460A4902A80FF0D3
:1042A8008DFF02AA06A808490FF088FF3220D22104
:1042B80006AA2B4600F002FF0AB070BD880D002048
:1042C800E22D0020F2A60508FAA605082DE9F3411B
:1042D800BDF820500C4690461F461A460023064655
:1042E8000095FFF771FF611E414430463A460023AE
:1042F80089B20095FFF768FF304621464246012300
:104308000095013EFFF760FFBF19B8B2214642464B
:104318000123089502B0BDE8F04155E72DE9F041C9
:104328000D46C5F1F008411E5E18C2EB0802C5F142
:10433800EF039BB292B2B6B29A422CBF904698460F
:104348009A4234BF11461946864234BF374607465B
:1043580040F23F13864238BF06469E4228BF1E469B
:10436800174B1B8848F68912B8F1EF0F28BF4FF09A
:10437800EF089342044610D049F2203293421AD1F2
:104388005020FFF7F5FB51204146FFF7F1FB522083
:104398003946FFF7EDFB53200AE041EA082189B2CC
:1043A8004420FFF7E5FB45203946FFF7E1FB4620AF
:1043B8003146FFF7DDFB20462946BDE8F0416FE6B0
:1043C8008601002000200146F0224FF4A073A5E7E3
:1043D80070B580B202FB03F489B292B29BB2FFF7C8
:1043E8009DFF0020FFF784FD0025064E04E0708D38
:1043F80080B2FFF7BDFD0135A542F8DBBDE870408E
:10440800E0E700BF880D002070B54FF0C0452A24B2
:104418002C80094C060A26802080080A20802180EA
:104428002B212980110A218022801A0A22802380C8
:104438002C232B8070BD00BF0000026070B5114BAB
:104448001B78012B044607D1002040F23F11024699
:10445800EF23FFF7D9FF04E0FFF7B4FF0020FFF7D1
:1044680047FDF02509E0013E2046B6B2FFF780FD82
:10447800002EF8D1013DADB215B14FF4A076F2E7A8
:1044880070BD00BFF01700202DE9F04F1C463E4BD1
:1044980087B01B78039183469DF8441010980591C6
:1044A800012B039B049092461FFA8BF09AB208D115
:1044B800411E531E0919534489B29BB2FFF7A4FF4A
:1044C80009E01FFA8AF51146A3B22A46FFF726FF2C
:1044D8000020FFF70DFD0027DDF80C803E4640F276
:1044E8003F1CA14639E0BBF1000F2EDB65452CDCF3
:1044F8000398002829DBB8F1EF0F26DC220702D148
:10450800002CC8BF013621492140002903DA0139AE
:1045180061F00F010131059A0AB1C1F10F01049848
:1045280030F8162003FA01F10A4012B26AB11849AC
:104538004A8D029392B2A8B21FFA88F1CDF804C04E
:10454800FFF70CFEDDF804C0029B013401354C4531
:10455800C9DB0136013708F10108574503DA5D4622
:1045680000240123F3E7084B1B78012B08D1002016
:1045780040F23F110246EF2307B0BDE8F04F43E792
:1045880007B0BDE8F04F1DE7F01700200F000080CE
:10459800880D00202DE9F74F1F463B4BDDF8308092
:1045A8001B7816469DF83420012B044601920D46CF
:1045B80080B28AB208D1411E531EC9199B1989B20B
:1045C8009BB2FFF721FF09E01FFA86FE1146BBB236
:1045D8007246FFF7A3FE0020FFF78AFC4FF0000B9E
:1045E800DA463DE0002C30DB09EB040340F23F12D1
:1045F80093422ADC002D28DB0BEB0503EF2B24DC90
:1046080019F00F0F04D1B9F1000FC8BF0AF1010A60
:104618001E4B09EA0303002B03DA013B63F00F0387
:104628000133019A0AB1C3F10F03012202FA03F31D
:1046380038F81A2013401BB213B1154B588D01E0FE
:10464800144A508880B2FFF793FC09F1010901E090
:104658004FF00009B945C5DB0AF1010A0BF1010B5E
:10466800B345F5DB084B1B78012B08D1002040F23D
:104678003F110246EF2303B0BDE8F04FC4E603B094
:10468800BDE8F04F9EE600BFF01700200F00008045
:10469800880D0020860100202DE9F0411C4F069C62
:1046A8003F789DF81C60012F02FB03F580B28FB2A2
:1046B80009D1411ECB1899B27B1E9A1893B23A467B
:1046C800FFF7A2FE07E092B29BB23946FFF726FE3B
:1046D8000020FFF70DFC002709E034F8020B1EB19B
:1046E800030A43EA002080B2FFF742FC0137AF42D9
:1046F800F3DB074B1B78012B07D1002040F23F1159
:104708000246EF23BDE8F0417EE6BDE8F04159E6F8
:10471800F01700202DE9F0431F2093B0FFF78EFE1D
:104728004FF47840FFF78AFE4FF6E0754FF4FC60CF
:10473800FFF784FE2846FFF781FE0020514CFFF763
:104748007DFE00204FF6FF79014664220346A4F857
:104758002A90CDF80090FFF737FD00200A21642247
:104768000346CDF80090FFF72FFD00200146642294
:1047780001234FF4784765850095FFF725FD7720DD
:10478800EF21C82200234FF4FC6667850097FFF7E6
:104798001BFDBD213222012340F23F1066850096A1
:1047A800FFF712FDA02032220023782167850097A9
:1047B800FFF70AFDA0207821322201234FF01F08BD
:1047C80066850096FFF700FDA0207821322202239B
:1047D800A4F82A80CDF80080FFF7F6FCA020782105
:1047E8003222032365850095FFF7EEFC264B274907
:1047F800A3F8028002AD3C2228460FF01DFCEB20F6
:10480800C3210522302300950025A4F82A9001959C
:10481800FFF7C0FE32210A2096220B4667850097D3
:10482800FFF754FD32213C2096220B466685009600
:10483800FFF74CFD32210B4696226E20A4F82A8001
:10484800CDF80080FFF742FDFFF7BAFBFFF7B4FB96
:104858003220FFF76DF92846FFF76AF96420FFF761
:1048680067F90B4B03F110028DE8240028465A68BB
:104878001B682946FFF710FF1195119B013311930F
:10488800FBE700BF880D002086010020F2630408C2
:10489800788801082DE9F14FFFF750F84FF0C0452F
:1048A8006420FFF745F90127FFF72EF94FF0280993
:1048B8006D48FFF7F1F82F800520A5F8009002F069
:1048C80031FECF232B80694B002683221E801A805D
:1048D80030221A80ED222A804FF064080322A3F8C0
:1048E80000801A8012221A8081221A80E8222A80E7
:1048F80085221A8079221F801A80CB222A803922A9
:104908001A804FF0340C02242C21F72219801E80C3
:10491800A3F800C01C802A8020221A80EA222A805C
:10492800C0221E80C1211E802A8026221A8029804A
:1049380011211980C5212980352119803E2119802E
:10494800C7212980BE211980362129803A20552186
:10495800A3F8009028801980B12129804FF0100B0E
:10496800F2211E80A3F800B02980082119802A802E
:10497800E0221F804FF01F092A801A22A3F8009016
:104988004FF0180A1A800F210A22A3F800A01A80F3
:104998001980062119804521198087211980322123
:1049A800198007211A804FF0E10E19801C80052418
:1049B80019801C801E80A5F800E04FF0250E1E808F
:1049C800A3F800E04FF0270EA3F800E01C80A3F83E
:1049D80000B04FF0090BA3F800B04FF0780B188027
:1049E800A3F800B04FF04D0BA3F800B01C800D24C5
:1049F800A3F800A01C8038241C8018802A20A3F863
:104A08000090EF2428802B201E801E801E801C8092
:104A180028803F201E801E801F801880B720A5F8A0
:104A280000C028801980B62129801A8082221A8025
:104A38001122A3F800E040461E8029272A8002F0B0
:104A480071FD40462F8002F06DFD0948FFF724F8FC
:104A58002C232F8030462B8040F23F1132462346CC
:104A680001B0BDE8F04FCFE4400D03000000026044
:104A780040420F002DE9F041022098B001210024A6
:104A880009F084FA012502268048169616A98DF8A1
:104A98005D408DF85E408DF85F408DF85C5008F001
:104AA800CDFE1820294609F071FA2846294609F052
:104AB80085FA21460C22764808F040FF0C227448FB
:104AC800294608F03BFF04210C22714808F036FF04
:104AD80005210C226E4808F031FF07210C226C4892
:104AE80008F02CFF08210C22694808F027FF09214B
:104AF8000C22674808F022FF0A2165480C2208F0BA
:104B08001DFF0B2162480C2208F018FF0E210C2211
:104B18005F4808F013FF0F210C225D4808F00EFFD4
:104B280007210C225B4808F009FF08210C2259488C
:104B380008F004FF09210C22564808F0FFFE0A215C
:104B48000C22544808F0FAFE0B210C22514808F0B8
:104B5800F5FE0C210A464F4808F0F0FE0D210C2204
:104B68004C4808F0EBFE0E210C224A4808F0E6FEFD
:104B78000C2248480F2108F0E1FE4CF6B373444874
:104B8800169316A98DF85C608DF85E408DF85F402D
:104B98008DF85D5008F052FE16A94FF680733D4817
:104BA80016938DF85C608DF85E408DF85F408DF847
:104BB8005D5008F043FE40F6B830FEF76DFFFEF793
:104BC800A3FF40F6B830FEF767FF0F2311934FF4A9
:104BD800805310270DF13C08099368464FF40023D1
:104BE80010941294149415940094019402940397C9
:104BF80004940694079408940A9405940B940C93CF
:104C0800CDF834800F95139508F091FB052368467D
:104C180011930F961094129414941594CDF838802B
:104C2800139508F084FB2946204608F000FC40F65E
:104C3800B830FEF731FF2046FFF7A0F904461649C1
:104C4800164E3846224607F007FE41F289239C4259
:104C580048F68918124F01D044450ED1FEF7BCFF23
:104C680000233B70A6F8008010200E4948F68912F0
:104C780041F2892307F0F0FD05E0FFF70BFE49F24A
:104C880041333D70338018B0BDE8F0810004024024
:104C9800000C024000100240FFA605088601002013
:104CA800F017002016A705084FF0C04336221A80D7
:104CB80003F50033012814BF682048201880704786
:104CC80070B5244B01228CB01A7000240AE0A9B2F6
:104CD8001F2230460135FFF741FA642DF7D1013420
:104CE800642C02D00025A6B2F1E732200146024624
:104CF8000346FFF7ABF94FF0C0432E221A8003F5A5
:104D0800003300201A881C881D88A4B200F09CF883
:104D1800ADB20023224600930F492B4603A80FF09B
:104D28004DFA00230A20C82103AA00F0C7F904F0AD
:104D3800FC0204F4784444EAC20242EAD522074954
:104D480003A80FF03BFA0A20DC2103AA002300F095
:104D5800B5F9FEE7F017002055A705086DA7050867
:104D68002DE9F04F40F23F19484534BF04464C4600
:104D7800EF2B34BF98464FF0EF084A4538BF9146AD
:104D8800EF2934BF0D46EF25C4EB090AC5EB080728
:104D980085B0BAF1000FB8BFCAF1000A002FB8BF3A
:104DA8007F424FF6FF734C452CBF1A4601221FFA6B
:104DB8008AFA454538BF0123BFB202930FFA8AF633
:104DC8003BB29E42BDF838B0019202DDC6F34F06F1
:104DD80007E0022693FBF6F67642B6B201E01E46DD
:104DE80003E00FFA8AF35B420393144A1378022B09
:104DF800204629465A4602D1FDF7FDFC01E0FFF79F
:104E0800ADF94C4501D1454514D0039A33B29342CC
:104E180005DD019AF31BA4189BB2A4B200E0334647
:104E280036B23AB29642DADA029A5344AD189BB2D5
:104E3800ADB2D4E705B0BDE8F08F00BFC044002094
:104E480000487047F817002082B0064BADF80600FE
:104E5800BDF8062092B21A80188880B202B0FFF717
:104E6800B2B800BFF4170020014B188880B2704711
:104E7800F417002082B0064BADF80600BDF80620F6
:104E880092B21A80188880B202B0FFF7A9B800BFA2
:104E9800F6170020014B188880B27047F6170020DB
:104EA800FFF7CCBAFFF73ABA10B5BDF8084002943C
:104EB800BDE81040FFF788B910B5BDF80840029466
:104EC800BDE81040FFF702BAFFF782BA2DE9F04FAC
:104ED8004FEA420800253D4C85B082468B46C8F112
:104EE800030817462E461FFA87F909EB0B0C228890
:104EF80005EB0A031FFA8CFC9BB26146184692B276
:104F0800CDF804C00293FFF729F9C9EB0B0292B25E
:104F18000392029B22880399184692B2FFF71EF962
:104F2800DDF804C02288C5EB0A039BB26146184627
:104F380092B20293FFF712F9029B2288039918464E
:104F480092B2FFF70BF905EB0B0292B2039209EB51
:104F58000A03228803999BB2184692B20293FFF77C
:104F6800FDF8029B2288C5EB0B0C1FFA8CFC184637
:104F7800614692B2CDF804C0C9EB0A09FFF7EEF812
:104F8800228803991FFA89F992B24846FFF7E6F892
:104F98002288DDF804C092B248466146FFF7DEF881
:104FA800B8F1000F04DA08EB860808F1060805E0F6
:104FB800F31B08F10A0808EB8308013F01360135A5
:104FC800BE42ADB28FD905B0BDE8F08FF41700200E
:104FD80008B9FEF7F5BF012801D1FEF7EDBF70470C
:104FE800704700200146F0224FF4A073FFF796B9EE
:104FF800704708B505280CD8DFE800F0121403053F
:105008000709094808BD094808BD094808BD0948F5
:1050180008BD0948094A0A4B40F24111FEF700FD54
:10502800084808BD084808BD740100206401002034
:105038005C0100205401002078A705082E640408AC
:10504800B3A505087C0100206C01002010B50446BA
:10505800FFF7CFFF014B18601C7110BD8C010020B9
:10506800014B1879704700BF8C01002008B5FFF785
:10507800C0FF808808BD08B5FFF7BBFFC08808BD22
:10508800F7B51F460B4B0C4E1D681446EA882B6873
:10509800203C5443A4B2AE1B03EB440418BF0126C2
:1050A800AB888DE8500017B1FFF7EEF901E0FFF784
:1050B80071FAFEBD8C0100207C0100202DE9F04131
:1050C8000F46984615460446084E08E020464346D3
:1050D8003946FFF7D5FF33689B88E418A4B215F862
:1050E800012B002AF2D1BDE8F08100BF8C0100201D
:1050F80010B5044608462146BDE81040DEE7094BD6
:1051080070B5044618790E461546FFF7B4FFC6F188
:10511800F001091A89B220462A460023BDE87040EA
:10512800CCE700BF8C010020704700BF044B1A6811
:105138000AB9044A1A601A681018186010467047AD
:10514800BC0D0020FC5200204FF0FF30704708B51E
:105158000248034A034B3721FEF762FC97A705086C
:1051680044640408B3A505080120704710B5044637
:105178000A48022109F090F90028F9D00748214689
:1051880009F053F90548012109F086F90028F9D0FA
:105198000248BDE8104009F045B900BF003800409A
:1051A80010B51948022109F077F90028F9D01648F6
:1051B800002109F03AF91448012109F06DF9002895
:1051C800F9D0114809F02EF90402A4B2002301E035
:1051D80001339BB2002BFBD00B48022109F05CF98C
:1051E8000028F9D00848002109F01FF906480121D4
:1051F80009F052F90028F9D0034809F013F92043BF
:10520800C0F3CB0010BD00BF003800402DE9F047C7
:105218008AB00AAF0A20012108F0B8FE4FF46043B3
:1052280047F8143D474EDFF824A1012400254FF02C
:105238000208304639468DF81A508DF818808DF8D6
:1052480019808DF81B4008F0F9FA30460D21052227
:1052580008F074FB30460E21052208F06FFB05228A
:1052680030460F2108F06AFB21464FF4804008F0D1
:10527800B1FE504608F08CFF4FF48273ADF802304F
:105288004FF40073ADF80A303823ADF80C305046AF
:1052980007236946ADF81030ADF80050ADF804505A
:1052A800ADF80650ADF80850ADF80E5008F0A2FF62
:1052B8005046214609F039F8A9468DF81A5030466B
:1052C8004FF48055394605958DF818408DF81980AA
:1052D8008DF81B4008F0B2FA3046294608F01FFB4B
:1052E8004025394618488DF818908DF819808DF8A2
:1052F8001A908DF81B40059508F0A0FA21464FF446
:10530800804008F073FE0621032009F0FDF80C2305
:1053180007A88DF8213007958DF820908DF8224048
:1053280007F080FF17238DF8243009A80F238DF884
:1053380025308DF826308DF8274002F073FB0AB02F
:10534800BDE8F08700040240000C0240003800402D
:10535800014B1878704700BFC00D0020024B5A88D7
:105368009B8802800B807047C00D0020014B0022F3
:105378001A707047C00D0020F0B593B06846002140
:1053880048220EF09BFE6D46002464484FF480517D
:1053980008F0C7FA002301E001339BB2002BFBD0D1
:1053A8009020FFF7E3FE002301E001339BB2002BBE
:1053B800FBD0FFF7F5FE4FF480510746574808F039
:1053C800AEFA002301E001339BB2002BFBD0534817
:1053D8004FF4805108F0A5FA002301E001339BB295
:1053E800002BFBD0D020FFF7C1FE002301E00133E2
:1053F8009BB2002BFBD0FFF7D3FE4FF4805106463B
:10540800464808F08CFA45F8047B01342E6244487B
:105418004021E4B208F071FA10B9092CB5D101E0C5
:10542800092C78D19DE80C00D218029B03980699A4
:10543800D218049BC018059BC018079BCB18089965
:10544800032490FBF4F092FBF4F25B1893FBF4F363
:10545800151AC11A9C1A002DB8BF6D420029B8BF91
:105468004942002CB8BF6442502D03DD502909DDA4
:10547800502C50DC8D4205DAAC424FF0020405DBBB
:10548800111806E08C424FF0020401DAD11800E04E
:10549800C1180A9B099A0C980F9DD2180B9BD21819
:1054A8000D9BC0180E9BC018109BEB18119D91FB0B
:1054B800F4F1032492FBF4F290FBF4F05B1993FBF4
:1054C800F4F3161AC41A9D1A002EB8BF7642002C9F
:1054D800B8BF6442002DB8BF6D42502E89B203DDBB
:1054E800502C09DD502D16DCA64205DAB5424FF0E6
:1054F800020405DB131806E0A5424FF0020401DAA6
:10550800D31800E0C318074A93FBF4F39BB29380C7
:1055180001235180137013B0F0BD00BF0004024096
:10552800000C0240C00D0020FFF712BFF7B505467A
:105538000C4601A80DF10601FFF710FF1B4BBDF843
:105548000660BDF8040093E80600724301FB0022E0
:1055580099685218164992FBF1F207EE102AF8EEF4
:10556800C77A40F23F17FCEEE77A17EE902A92B21C
:10557800B2F5207F28BF3A462A801D69DA685B6940
:105588006E4302FB0060C01890FBF1F107EE101AA1
:10559800F8EEC77AFCEEE77A17EE903A9BB2B3F5CD
:1055A800F07F28BFEF232380FEBD00BFC80D002079
:1055B80040420F00FFF7DABE014B187E704700BF6C
:1055C800C80D0020FFF7CABE042808B505D907484A
:1055D800074A084B7D21FEF723FA054B03EB8000B1
:1055E800038B0B80438B138008BD00BFB8A7050849
:1055F8004A640408D6A7050808B5082001F094F9FC
:1056080042F69643C31A584240EB030008BD10B552
:105618000A2001F0B1F90C4C20600E2001F0ACF921
:105628006060122001F0A8F9A060162001F0A4F92A
:10563800E0601A2001F0A0F920611E2001F09CF919
:1056480001236061237610BDC80D002010B5FFF757
:10565800DDFD01F033FA044601F03CFA0749034640
:105668002246202007F0F8F8FFF7C6FF28B101F01E
:105678003FFA10B9BDE81040C9E710BD12A80508E7
:1056880010B5104C0A20216801F05DF961680E2000
:1056980001F059F9A168122001F055F9E1681620C6
:1056A80001F051F921691A2001F04DF961691E20B4
:1056B80001F049F9082042F69641BDE8104001F092
:1056C80025B900BFC80D00202DE9F04F0346A7B04B
:1056D800B0F800C01C898688DF885D89CDF810C0C5
:1056E800B249B0F802C0B3F80C90B3F80E80CDF808
:1056F80024C00FFA84FB30B201220FFA87FE0BEBAD
:10570800000C0A7629B20FFA89FACDF888C001EBA5
:105718000E0C0FFA88F2CDF890C00AEB0B0CCDF8FE
:1057280030C002EB010CCDF858C0B3F810C05B8A4A
:10573800CDF800C00FFA8CFC06910CEB00010A9121
:1057480002930CEB0A011BB2239103EB0E010E919D
:1057580099182591049900FA81F0584450446044FE
:10576800DDF824C006990EFA8CFEDDF810C01FFA89
:1057780080FB1CFB0CF08E4416FB0600964414FBC1
:105788000400009A19FB09009E4412FB02001FFA4C
:105798008EFA09F08BFFDDF824C0029ACDE91201D8
:1057A8001CFB0CF017FB070015FB050018FB080095
:1057B80012FB020009F07AFFDDF824C0029ACDE955
:1057C800140104991CFB01F317FB063615FB04664C
:1057D800009B18FB096612FB036009F067FFDDE90F
:1057E8001423CDE90001DDE9120109F0D5FF0446D3
:1057F8000D46DDE9000102460B4609F0CDFF0246E1
:105808000B462046294609F013FECDE918015846F3
:1058180009F05CFFCDE91001DDE91023DDE90001A5
:1058280009F0BAFFCDE90601504609F04FFF80465E
:1058380089464246DDE912014B4609F0ADFFDDE934
:105848001023CDE91C01DDE9140109F0A5FF0022B0
:1058580006460F46564BDDE9180109F09DFF424602
:1058680004460D464B46DDE9060109F095FF024660
:105878000B4609F0DFFD02460B462046294609F093
:10588800D9FD424604460D464B46DDE91C0109F0A8
:1058980083FF02460B462046294609F0C9FDDDE98B
:1058A800102304460D463046394609F075FF024676
:1058B8000B462046294609F0BBFDDDF828C0CDE996
:1058C80002014FEA8C10DDF830C000EB0C20DDF847
:1058D80010C0A0241CFB040009F0E8FEDDF838C065
:1058E800CDE90A014FEA8C10DDF858C000EB0C2016
:1058F800DDF824C01CFB040009F0D8FECDE90C013A
:10590800504609F0D3FEDDE91023CDE91601DDE9A3
:105918000C0109F041FF4246CDE91E014B46DDE985
:105928000A0109F039FF4246CDE920014B46DDE97D
:10593800000109F031FF32463B4609F079FDCDE917
:105948000E01584609F0B2FEDDE91C23CDE91A0123
:10595800DDE9060109F06CFDDDF88CC0C024CDE955
:10596800060104FB0CF0DDF888C0302505FB0C00AF
:10597800DDF810C078261CFB060009F097FEDDF85C
:1059880094C0824604FB0CF0DDF890C005FB0C00C7
:10599800DDF824C01CFB06008B4609F087FEDDE914
:1059A800102306460F4609F0F7FE03E0C80D002055
:1059B800000014404246CDE904014B465046594682
:1059C80009F0EAFEDDE9142380468946DDE90A018B
:1059D80009F0E2FEDDE9002304460D46DDE90C018D
:1059E80009F0DAFE02460B462046294609F020FD5A
:1059F8000022A14B09F0D0FEDDE9202304460D4624
:105A0800DDE91E0109F014FD02460B46DDE9160129
:105A180009F0C2FE02460B462046294609F00AFD57
:105A2800002204460D46954BDDE90E0109F0B4FE4F
:105A380002460B462046294609F0FCFCDDE9022314
:105A480009F0D4FF88A3D3E9002309F0A5FE0AF0E2
:105A58003DF98B490860DDE91223DDE90C0109F005
:105A68009BFEDDE9002304460D46DDE90A0109F045
:105A780093FE02460B462046294609F0D9FC00222F
:105A88007D4B09F089FEDDE91E2304460D46DDE95C
:105A9800200109F0CDFC02460B46DDE91A0109F0A8
:105AA8007BFE02460B462046294609F0C3FC00222D
:105AB80004460D46714BDDE9060109F06DFE02460C
:105AC8000B462046294609F0B5FCDDE9022309F01A
:105AD8008DFF65A3D3E9002309F05EFE0AF0F6F80E
:105AE800674A5060DDE90E23DDE90A0109F054FE3A
:105AF800DDE9062304460D46DDE90C0109F04CFEFC
:105B080002460B462046294609F094FC002204462A
:105B18000D465A4BDDE9180109F03EFE02460B46D8
:105B28002046294609F086FCDDE9022309F05EFFDC
:105B38004DA3D3E9002309F02FFE0AF0C7F8504B14
:105B480059469860DDE91423504609F025FEDDE941
:105B5800002304460D463046394609F01DFE02462C
:105B68000B462046294609F063FC0022424B09F007
:105B780013FE424604460D464B46DDE9040109F092
:105B880057FC02460B46DDE9160109F005FE024600
:105B98000B462046294609F04DFC35A3D3E90023DE
:105BA80004460D46DDE90E0109F0F6FD02460B46F6
:105BB8002046294609F03EFCDDE9022309F016FFDC
:105BC80029A3D3E9002309F0E7FD0AF07FF8DFF8FD
:105BD800B0C0DDE91223CCF80C003946304609F094
:105BE800DBFDDDE9002304460D465046594609F021
:105BF800D3FD02460B462046294609F019FC00222F
:105C08001D4B09F0C9FDDDE9042304460D46404655
:105C1800494609F00DFC02460B46DDE91A0109F078
:105C2800BBFD02460B462046294609F003FC10A39B
:105C3800D3E9002304460D46DDE9060109F0ACFD71
:105C480002460B462046294609F0F4FBDDE902230B
:105C580009F0CCFE04A3D3E9002309F09DFD0AF066
:105C680035F8074908610DE00000000080842E41E6
:105C78000000000000C0824000001440000089407D
:105C8800C80D0020DDE90E235046594609F084FD71
:105C9800DDE9062304460D463046394609F07CFD09
:105CA80002460B462046294609F0C4FB11A3D3E956
:105CB800002304460D46DDE9180109F06DFD024692
:105CC8000B462046294609F0B5FBDDE9022309F019
:105CD8008DFE0AA3D3E9002309F05EFD09F0F6FF63
:105CE800034A506127B0BDE8F04FC9E4AFF3008024
:105CF800C80D00200000000000C082400000000025
:105D080080842E41AFF30080064B074A5968116022
:105D18001969064A1160D969054A11609A6A054BE2
:105D28001A60704794010020B03E0020CC44002047
:105D3800A4440020643E0020014B1878704700BF3F
:105D4800E40D0020032808B505D90548054A064B87
:105D58007321FDF765FE0C235843044B185808BD02
:105D68004DA805087664040867A805089401002072
:105D7800032808B505D90648064A074B7821FDF7D8
:105D88004FFE064B0C2202FB0030406808BD00BFE6
:105D98004DA805088664040867A805089401002032
:105DA800034B044A1B780C2101FB032398687047B6
:105DB800E40D002094010020034B044A1B780C20BA
:105DC80000FB032399607047E40D00209401002034
:105DD800144B1B78012B10B5134B144C0ED11968BA
:105DE800C82000F0B0FD2168CC2000F0ACFD104BBD
:105DF800D020196800F0A7FDD4200DE01968D8203C
:105E080000F0A1FD2168DC2000F09DFD084BE0209A
:105E1800196800F098FDE420064B1968BDE81040A9
:105E280000F091BD280F0020B03E0020CC44002097
:105E3800A4440020643E0020144B1B78012B10B5AD
:105E4800134C0FD1C82000F097FD2060CC2000F043
:105E580093FD104B1860D02000F08EFD0E4B18609B
:105E6800D4200EE0D82000F087FD2060DC2000F070
:105E780083FD084B1860E02000F07EFD064B18609B
:105E8800E42000F079FD054B186010BD280F0020B4
:105E9800B03E0020CC440020A4440020643E0020F2
:105EA80008B502F02FFB10B1BDE80840C4E7BDE813
:105EB800084029E70148FBF7E8BB00BFD4150020DC
:105EC8000148FBF7E2BB00BFD41500200148FBF7EF
:105ED800DCBB00BFD41500200148FBF7D6BB00BFD0
:105EE800D4150020032808B505D91648164A174BBB
:105EF8004F21FDF795FD164B1870164B1870164B71
:105F0800012202281A70154B0FD0032813D0904293
:105F180005D0134A12681A60BDE80840CAE7114A5A
:105F280012681A60BDE80840CAE70F4A12681A608A
:105F3800BDE80840CAE70D4A12681A60BDE8084083
:105F4800CAE700BF4DA805089764040891A805088A
:105F5800E40D0020A63E0020100E0020EC020020D8
:105F6800E4020020E0020020DC020020D802002029
:105F7800064B07495960C021002219721E211A7068
:105F8800D9601A745A611A76DA61704724180020A9
:105F980040787D0110B50321FF22C02001F0A4F84C
:105FA8001F4C102120608022C02001F09DF8112193
:105FB80020608022C02001F097F812212060802202
:105FC800C02001F091F8132120608022C02001F048
:105FD8008BF8142120608022C02001F085F815215B
:105FE80020608022C02001F07FF8802220601621E6
:105FF800C02001F079F82060C0201721802201F02C
:1060080073F82060074CC020227AB72101F06CF8A1
:106018000023237463612376E3610123237010BD99
:10602800883E00202418002038B5C0200321FF2214
:1060380001F05AF80B4D00242B19615D5A78C020E5
:10604800023401F051F8C82CF6D1B121AC22C0209D
:1060580001F04AF8C0200321002201F045F8002091
:1060680038BD00BFAB6404082DE9F34706460F4668
:1060780092461D461AB90C1FE401914635E005EE1B
:10608800902A06EE903AB8EE657AF8EE667AFC0148
:10609800C7EE277AA4F500749FED5C7A67EE877ADD
:1060A80017EE900A09F024FB41EC100B0BF07CFB77
:1060B80059EC108B4946404609F030FE24184FEA47
:1060C800CA1009F0F3FACDE90001284609F0EEFA02
:1060D8004B46424609F060FB02460B46DDE90001EB
:1060E80009F0A6F909F01AFE8146002E14BF4FF0F8
:1060F80022084FF01A08C5F307224146C02000F0D5
:10610800F3FF08F10101EAB2C02000F0EDFFC4F38B
:10611800014208F10201C02000F0E6FFC4F30722A3
:1061280008F10301C02000F0DFFFE2B208F104012A
:10613800C02000F0D9FFC9F3034305F4702243EAF5
:10614800123208F10501C02000F0CEFF08F1060167
:10615800C9F30722C02000F0C7FF08F107015FFA62
:1061680089F2C02000F0C0FFC020B121A02200F0B9
:10617800BBFF07EE107A264CF8EEC77A0EBBD4EDBB
:10618800015A06EE90AAB8EE657A05EE905AB8EE76
:10619800666AF8EE656A0123C6EE266A237477EE0E
:1061A800A67A67EE277A17EE900A09F0A1FA41EC71
:1061B800100B0BF0F9FA51EC100B09F0AFFD606110
:1061C80020E005EE90AAD4ED016AB8EE656A05EE06
:1061D800905AB8EE667AF8EE656A0123C6EE266A2A
:1061E800237677EEA67A67EE277A17EE900A09F0FB
:1061F8007FFA41EC100B0BF0D7FA51EC100B09F0B9
:106208008DFDE0610020BDE8FC8700BF0000004371
:10621800241800200022012326E7012838B50D465E
:1062280004D002280CBF3C242C2400E0342421464E
:10623800C02000F0D3FF05F0070200F00F0040EA8D
:1062480002122146C020BDE8384000F04DBF2DE9BC
:10625800F3470A9C1D4607468A461646524B01E0FC
:106268006D0864089C42FBD82DB906F10076043EFF
:10627800F601A94634E006EE905AB8EE667A06EEC4
:10628800904AF8EE667AF601C7EE277AA6F5007608
:106298009FED467A67EE877A17EE900A09F028FA9A
:1062A80041EC100B0BF080FA59EC108B4946404634
:1062B80009F034FD3618E80109F0F8F9CDE90001D4
:1062C800204609F0F3F94B46424609F065FA0246C2
:1062D8000B46DDE9000109F0ABF809F01FFD814626
:1062E800022F9BBF324BDB194FF0000893F8C88090
:1062F800C4F307224146C02000F0F6FE08F1010170
:10630800E2B2C9B2C02000F0EFFE08F10201C9B242
:10631800C6F30142C02000F0E7FE08F10301C9B24C
:10632800C6F30722C02000F0DFFE08F10401C9B25D
:10633800F2B2C02000F0D8FE04F47024C9F303437D
:1063480008F1050143EA1432C9B2C02000F0CCFEBE
:1063580008F10601C9B2C9F30722C02008F10708ED
:1063680000F0C2FE5FFA89F25FFA88F1C02000F0FF
:10637800BBFEBAF1010F0CBF2F220F220DB942F05C
:106388004002012F06D002D3022F0AD105E0C02017
:10639800102104E0C020112101E0C020122100F0EA
:1063A800A3FE0020BDE8FC87FFFF0F0000000043AC
:1063B800AB64040807B5012300930023FFF747FFE8
:1063C8000EBD00280CBFFF22002208B5C020032103
:1063D80000F08AFE002008BD08B5C020B121AC221B
:1063E80000F082FE002008BD08B50420012107F056
:1063F800CDFD4FF480700121BDE8084007F0F6BDDF
:1064080007B50223009303238DF8043003480023C3
:1064180069468DF8073007F011FA0EBD00080240F2
:1064280030B5124D8BB0002406A806940794089442
:10643800099406F0D1FB00948DF804408DF80540CE
:106448000294039404942846012469468DF8144064
:1064580006F093FB28460B212246062306F008FC8B
:106468002846214606F0D2FB0BB030BD0020014083
:1064780010B5002104460122302000F035FEC0B9D5
:10648800012001F04FF8002CB8BF4034E4B21021CD
:106498002246302000F028FE012001F043F8302089
:1064A8001121224600F020FE0120BDE8104001F035
:1064B80039B810BD10B5002104460122302000F083
:1064C80013FEC0B9012001F02DF8002CB8BF4034EC
:1064D800E4B212212246302000F006FE012001F02D
:1064E80021F830201321224600F0FEFD0120BDE8EE
:1064F800104001F017B810BD38B5012205460C460A
:106508003020002100F0F0FDF0B9012001F00AF878
:1065180025EAE5725F2AA8BF5F223B21D2B230206C
:1065280000F0E2FD012000F0FDFF24EAE4725F2A9A
:10653800A8BF5F22D2B230203C2100F0D5FD012057
:10654800BDE8384000F0EEBF38BD302810B504462D
:106558000ADC10F17F0F02DB002802DB05E06FF098
:106568007E0404F5807400E03024002130200A46BF
:1065780000F0BAFDA8B90120E4B200F0D3FF412130
:106588002246302000F0B0FD012000F0CBFF302083
:106598004221224600F0A8FD0120BDE8104000F08D
:1065A800C1BF10BD282810B5044609DC10F1180F2A
:1065B80002DB002802DB04E06FF017047F3400E000
:1065C8002824002130200A4600F08EFDA8B90120B9
:1065D800E4B200F0A7FF53212246302000F084FDEA
:1065E800012000F09FFF30205421224600F07CFD5E
:1065F8000120BDE8104000F095BF10BD08B530205F
:106608000021012200F070FD60B9012000F08AFF2E
:1066180030203321402200F067FD0120BDE808400A
:1066280000F080BF08BD10B530200021012200F025
:106638005BFD044660B9012000F074FF302033216F
:10664800224600F051FD0120BDE8104000F06ABF6D
:1066580010BD10B530200021012200F045FD044690
:10666800A0B9012000F05EFF34212246302000F05E
:106678003BFD012000F056FF30203721224600F074
:1066880033FD0120BDE8104000F04CBF10BD402094
:10669800EEE640200EE708B500210122302000F088
:1066A80023FD012000F03EFF30203421024600F097
:1066B8001BFD012000F036FF30203721024600F094
:1066C80013FD0120BDE8084000F02CBF08B50021EB
:1066D8000122302000F008FD012000F023FF3020C7
:1066E80034210C2200F000FD0120BDE8084000F034
:1066F80019BF000000000000184B1949D3ED006ACB
:1067080093ED017A00231A469FED166A03E0F0EE36
:10671800476AB0EE677A505E05EE900AF8EEE57AC1
:106728000133C7EE867A9BB218B204327F2877EE1F
:10673800E67AECDD27EE077A07EEA77A0A49074AD8
:106748000B80BDEEC77A002313605360C2ED027A56
:1067580017EE102A054B92001A607047E80D0020CA
:10676800E02900200000FA45103E0020AC1A002065
:106778002DE9F84F2E4B2F4A19682F4B19B92F497D
:1067880011602F4A02E02F4911602F4A1A602F4BDF
:10679800DFF8BCA0DFF8BC90DFF8BCB000221A809C
:1067A800244A9846176830E007EB84036500B3F97C
:1067B800023007EE103AF8EEC77A013617EE900A63
:1067C80008F096FF18A3D3E9002308F0E5FF09F0C5
:1067D8007DFA29F815002AF8140037F9243007EE55
:1067E800103AF8EEC77A013517EE900A08F080FFE4
:1067F8000DA3D3E9002308F0CFFF09F067FA2BF8BF
:10680800140029F81500A8F80060B8F8006034B240
:10681800FF2CC9DD00F05EF800F06AF801F0A4F979
:10682800BDE8F84F68E700BF9A9999999999E93FA7
:10683800A01A0020941A0020CC180020E43100206F
:10684800E42D0020E4390020E4350020103E00202B
:10685800E0250020E0290020E027002010B50B4C9F
:10686800204606F038FC0A4B18600A4806F033FC4C
:10687800094B1860FFF77CFF084B094901222046A5
:106888009A81BDE8104006F0A7BC00BF1060024026
:10689800A01A002088600240BC1A0020E80D0020E1
:1068A80020800010014B1868704700BFAC1A002008
:1068B80008B5054B054819880022012309F064FF33
:1068C800034B187008BD00BFC4010020C825002074
:1068D800E420002003480449044A4FF4807309F077
:1068E800CBBF00BFC8010020E0250020C623002040
:1068F80003480449044A4FF4807309F0BDBF00BF40
:10690800D4010020E0270020001C002038B50546EF
:106918000C460135C1F3072100F012FEA8B2E1B21E
:1069280000F00EFE00B238BD38B5044600F01EFD7A
:1069380001340546A0B200F019FDEDB2C0B240EA3C
:10694800052000B238BD37B50B0E8DF804300B0C9E
:106958008DF805300B0A8DF806308DF807100024E5
:1069680000E0284601AB451CE15C013400F0E8FD7D
:10697800042CADB2F5D13EBD37B5002400E0284661
:10698800451C00F0F3FC01ABADB2E0540134042C1B
:10699800F5D19DF805009DF80430000440EA036035
:1069A8009DF8073018439DF8063040EA03203EBDA5
:1069B80038B50446642000F0B5FD25786068AD0060
:1069C800EDB2257006F09FFF237A40FA03F000F03D
:1069D80003000543104B257005F00F055A5D6378D9
:1069E800D218D2B2D3B20132D2B2022A637001D81D
:1069F8000022A2705BB2012B03DD0123A3700023E8
:106A0800637094F90130013303DAFF23A370002384
:106A1800637094F9020038BD76650408F7B5042060
:106A28000121234F07F0B2FA02AD01214FF4804053
:106A3800012407F0DBFA00264FF4B07338466946A4
:106A480045F8083D8DF804608DF8074006F0F6FE1D
:106A58001020214607F09AFA7823694615480093D2
:106A68008DF804608DF8074006F0E8FE0420214602
:106A780007F08CFA21464FF4804007F0B7FA1C2340
:106A88003846694600938DF804608DF8074006F093
:106A9800D5FE0220214607F079FAB02306488DF882
:106AA800046069468DF80740009306F0C7FEFEBDF6
:106AB800000802400010024000040240802108B58E
:106AC800034806F01AFFD0F1010038BF002008BDC6
:106AD8000004024008B54FF48071044806F00DFF29
:106AE800D0F1010038BF002008BD00BF00080240F7
:106AF80008B5FFF7E3FF08B1FFF7ECFFC0B208BD28
:106B080010B5642000F00EFD2348FFF751FF04463E
:106B180038B9224B01221A70214B1870214B18707A
:106B28000FE0FFF7D7FF60B9002C1E4A1C4C1B4B27
:106B3800C8BF10704FF00101CEBF217020701170D6
:106B480018701948FFF734FF184B1B78042B16D11F
:106B580000281FD0164B1A7806DD0132D2B20F2A50
:106B68001A7008D9102205E0013AD2B2102A1A7018
:106B780001D900221A70BDE81040FAF779BE002842
:106B88000C4B01D1187010BD02DD01221A7010BD26
:106B9800FF221A7010BD00BF14020020E12D002052
:106BA800E02D0020E32D002020020020443E00209C
:106BB800AE3E0020E22D002007B50220012107F09B
:106BC800E5F9012300938DF8043002238DF8053090
:106BD8000448002369468DF806308DF8073006F022
:106BE8002DFE0EBD0004024010B5084C0121002204
:106BF800204606F098FE40F2FF4000F093FC012189
:106C080020460A46BDE8104006F08DBE000402404A
:106C180008B5FFF7E9FF00210A46302000F064FAC2
:106C2800012000F07FFC01210A46302000F05CFAC8
:106C3800012000F077FC00210122302000F054FAF6
:106C4800012000F06FFC01210822302000F04CFAEE
:106C5800012000F067FC02210122302000F044FAF4
:106C6800012000F05FFC00210A46302000F03CFAC9
:106C7800012000F057FC1B21CD22302000F034FA0F
:106C8800012000F04FFC04210322302000F02CFAF0
:106C9800012000F047FC06210822302000F024FAE9
:106CA800012000F03FFC07210A46302000F01CFAC2
:106CB800012000F037FC08218022302000F014FA6F
:106CC800012000F02FFC1E21B022302000F00CFA29
:106CD800012000F027FC05219122302000F004FA61
:106CE800012000F01FFC0D210322302000F0FCF9E8
:106CF800012000F017FC0E210022302000F0F4F9EA
:106D0800012000F00FFC14218022302000F0ECF963
:106D1800012000F007FC0B218822302000F0E4F964
:106D2800012000F0FFFB30200C21822200F0DCF96A
:106D3800012000F0F7FB12218822302000F0D4F95E
:106D4800012000F0EFFB13218C22302000F0CCF959
:106D5800012000F0E7FB00210122302000F0C4F9F7
:106D6800012000F0DFFB0C210822302000F0BCF9E4
:106D7800012000F0D7FB0D210822302000F0B4F9E3
:106D8800012000F0CFFB0E210822302000F0ACF9E2
:106D9800012000F0C7FB0F210822302000F0A4F9E1
:106DA800012000F0BFFB00210A46302000F09CF9CA
:106DB800012000F0B7FB40210222302000F094F9B6
:106DC800012000F0AFFB00224121302000F08CF9B7
:106DD800012000F0A7FB30203F21D42200F084F9E5
:106DE800012000F09FFB00210122302000F07CF9F7
:106DF800012000F097FB10210F22302000F074F9D9
:106E0800012000F08FFB11210F22302000F06CF9D7
:106E1800012000F087FB12210022302000F064F9E5
:106E2800012000F07FFB13210022302000F05CF9E4
:106E3800012000F077FB09213C22302000F054F9B2
:106E4800012000F06FFB00210122302000F04CF9F6
:106E5800012000F067FB30203421024600F044F99D
:106E6800012000F05FFB30203721024600F03CF99A
:106E7800012000F057FB36210322302000F034F9BE
:106E8800012000F04FFB39210322302000F02CF9BB
:106E9800012000F047FB3B213C22302000F024F980
:106EA800012000F03FFB3C210A46302000F01CF98D
:106EB800012000F037FB00210A46302000F014F9C9
:106EC800012000F02FFB5121C022302000F00CF9E6
:106ED800012000F027FB30205221002200F004F9A5
:106EE8000120BDE8084000F01DBB00BF2DE9F04FB0
:106EF800454E464D93B001214FF4001007F046F877
:106F0800304605F0E9FF4FF0C0630293404B03930E
:106F1800404B002404934FF400794FF400334FF4AE
:106F280080684FF400674FF4005A4FF4807B304676
:106F380002A90C9301930997CDF81890059407942A
:106F4800CDF82080CDF828A0CDF82CB00D9406F00F
:106F58004FF822463046304906F0A5F83046012160
:106F680006F0ABF801210A464FF0402007F07CFA02
:106F7800284605F0B1FF294A019B0392284A0C9341
:106F880004922846402202A9059209970294CDF856
:106F980018900794CDF82080CDF828A0CDF82CB013
:106FA8000D9406F025F8224628461E4906F07BF87F
:106FB8002846012106F081F842F2107701220221C9
:106FC800194807F051FA384600F0ACFA304601216A
:106FD80006F049F80121284606F045F8384600F041
:106FE800A1FA0B238DF8443011A801238DF84540F0
:106FF8008DF846408DF8473000F014FD384600F013
:1070080091FA13B0BDE8F08F10600240886002402A
:107018000C400040E4390020E43100200C3C0040E2
:10702800E4350020E42D0020003C004002481021F7
:10703800012206F08FB800BF1060024013B502208D
:10704800012106F0A3FF4FF410730E4C00930223A6
:107058008DF804308DF8053001238DF80630204670
:10706800002369468DF8073006F0E8FB2046062124
:10707800042206F063FC20460921042206F05EFC87
:107088001CBD00BF0004024030B5154D85B001217C
:107098004FF4001006F09EFF284606F065FC00231A
:1070A800ADF804304BF6FF73ADF806303323ADF876
:1070B80008304FF48063ADF80A304FF48043ADF8E0
:1070C8000C3004AC074B2846012144F8103D06F06B
:1070D800EDFC2846694606F075FC05B030BD00BFDA
:1070E80000540040801A060073B54FF49613064604
:1070F8000D461446019304E0019B5A1E0192002B91
:1071080057D031484FF4003106F0E8FD0028F3D19C
:107118002D48012106F0D6FC4FF48053019304E07A
:10712800019B5A1E0192002B45D02748274906F09B
:10713800C0FD0028F4D024483146002206F0DAFCCD
:107148004FF48053019304E0019B5A1E0192002BD7
:1071580033D01D481E4906F0ACFD0028F4D01A486B
:10716800294606F04AFD4FF48053019303E0019B42
:107178005A1E01921BB31448164906F09AFD0028BE
:10718800F5D01148214606F038FD4FF496130193C7
:1071980003E0019B5A1E01929BB10B480E4906F071
:1071A8009DFD0028F5D00848012106F097FC002035
:1071B80008E0012006E0022004E0032002E00420A9
:1071C80000E005207CBD00BF005400400100030022
:1071D80082000700800007000400001037B54FF454
:1071E800961304460D46019305E0019B5A1E019231
:1071F800002B00F09B8056484FF4003106F06EFDDE
:107208000028F2D15248012106F05CFC4FF480536B
:10721800019305E0019B5A1E0192002B00F0888023
:107228004B484C4906F045FD0028F3D04848214614
:10723800002206F05FFC4FF48053019304E0019BA9
:107248005A1E0192002B75D04148434906F031FD82
:107258000028F4D03E48294606F0CFFC4FF480536E
:10726800019304E0019B5A1E0192002B64D0384818
:107278003A4906F033FD0028F4D03548012106F0DC
:1072880021FC4FF48053019304E0019B5A1E0192A4
:10729800002B53D02E482F4906F00BFD0028F4D0C0
:1072A8002B482146012206F025FC4FF48053019318
:1072B80004E0019B5A1E0192002B41D0244C28491E
:1072C800204606F00BFD0028F3D02046002106F0EA
:1072D80019FC20460121238B06F000FC4FF4805353
:1072E800019304E0019B5A1E0192002B2AD01848F2
:1072F8001C4906F0F3FC0028F4D0154806F07FFC82
:107308004FF480530193124A03E0019B591E0191E7
:10731800D3B113889B05F8D4012104460C4806F024
:10732800F1FB0B48104906F0F3FC0EE001240CE0D9
:1073380002240AE0032408E0042406E0052404E00B
:10734800062402E0072400E0082420463EBD00BFD2
:1073580000540040010003008200070004000010F0
:1073680002000010400000100004001013B54FF494
:1073780096130446019305E0019B5A1E0192002BC7
:1073880000F0AF8060484FF4003106F0A7FC0028F9
:10739800F2D15D48012106F095FB4FF4805301932B
:1073A80005E0019B5A1E0192002B00F09C80564874
:1073B800564906F07EFC0028F3D05348A02100224D
:1073C80006F098FB4FF48053019305E0019B5A1E89
:1073D8000192002B00F089804B484D4906F069FC6A
:1073E8000028F3D0210A484806F007FC4FF48053E0
:1073F800019304E0019B5A1E0192002B77D042486A
:10740800444906F06BFC0028F4D0E1B23E4806F08F
:10741800F4FB4FF48053019304E0019B5A1E019240
:10742800002B66D038483B4906F058FC0028F4D0B9
:107438003548012106F046FB4FF48053019304E0E0
:10744800019B5A1E0192002B55D02F482F4906F058
:1074580030FC0028F4D02C48A121012206F04AFB78
:107468004FF48053019304E0019B5A1E0192002BB4
:1074780043D0254C2849204606F030FC0028F3D09C
:107488002046002106F03EFB20460121238B06F012
:1074980025FB4FF48053019304E0019B5A1E01928F
:1074A800002B2CD018481D4906F018FC0028F4D0F1
:1074B800154806F0A4FB4FF480530193124A03E0E9
:1074C800019B591E0191E3B113889905F8D4012154
:1074D80004460D4806F016FB0B48114906F018FC47
:1074E80010E001240EE002240CE003240AE0042446
:1074F80008E0052406E0062404E0072402E0082446
:1075080000E0092420461CBD00540040010003008F
:107518008200070004000010020000104000001064
:107528000004001082B0002304E0019B01330193A2
:10753800009B01330093009B8342F6D302B070474F
:1075480037B54FF4805304460D46019304E0019B80
:107558005A1E0192002B6DD03C484FF4003106F0C2
:10756800BDFB0028F3D13948012106F0ABFA4FF4EE
:107578008053019304E0019B5A1E0192002B5BD0BB
:107588003248334906F095FB0028F4D02F48A02153
:10759800002206F0AFFA4FF48053019304E0019BF8
:1075A8005A1E0192002B49D028482A4906F081FB2F
:1075B8000028F4D0210A254806F01FFB4FF4805319
:1075C800019304E0019B5A1E0192002B38D01F48FA
:1075D800214906F06EFB0028F4D0E1B21B4806F002
:1075E8000CFB4FF48053019303E0019B5A1E019258
:1075F80043B31648184906F05CFB0028F5D0134839
:10760800294606F0FAFA4FF49613019303E0019B1A
:107618005A1E0192C3B10D48104906F05FFB0028BD
:10762800F5D00A48012106F059FA0D48FFF77AFF0C
:1076380000200AE0012008E0022006E0032004E020
:10764800042002E0052000E006203EBD0054004072
:1076580001000300820007008000070004000010FA
:10766800A0860100F7B54FF4805304460D46164630
:10767800019304E0019B5A1E0192002B74D04048EC
:107688004FF4003106F02AFB0028F3D13C480121D1
:1076980006F018FA4FF48053019304E0019B5A1E38
:1076A8000192002B62D03648364906F002FB0028CA
:1076B800F4D03348A021002206F01CFA4FF480537E
:1076C800019304E0019B5A1E0192002B50D02C48D4
:1076D8002D4906F0EEFA0028F4D0210A284806F0D1
:1076E8008CFA4FF48053019304E0019B5A1E0192D7
:1076F800002B3FD02248254906F0DBFA0028F4D0B9
:10770800E1B21F4806F079FA4FF48053019304E080
:10771800019B5A1E0192002B2ED019481B4906F0D6
:10772800C8FA0028F4D000244FF4961710E0295D19
:10773800134806F062FA019703E0019B5A1E019272
:10774800E3B10F48124906F0C9FA0028F5D0013410
:10775800E3B2B342EBD30A48012106F0BFF90D4862
:10776800FFF7E0FE00200AE0012008E0022006E022
:10777800032004E0042002E0052000E00620FEBD0E
:107788000054004001000300820007008000070049
:1077980004000010A086010013B50520012106F0A1
:1077A800F5FB184C4FF4E053009302238DF8043096
:1077B8008DF805302046002369468DF806308DF88F
:1077C800073006F03BF820460A21062206F0B6F8F4
:1077D80020460C21062206F0B1F8062220460B218D
:1077E800A4F5006406F0AAF84FF400432046694661
:1077F800009306F023F820460F21062206F09EF893
:107808001CBD00BF000802401FB50446FFF7D4F9AD
:10781800FFF73AFCFFF7FCF9FFF7BEFF01214FF431
:10782800004006F0D7FB02940F4C1023ADF802304D
:10783800204600236946ADF80430ADF80C30ADF8A9
:107848000030ADF8063006F0F4FC69464FF04020F1
:1078580006F0C3FD2046012106F073FD4FF04020DD
:10786800012106F06EFD1FBD003C0040014B186071
:10787800704700BF040E0020704710B50A4A1379FC
:10788800262B04D80949C8540133137110BD074A7F
:107898000123591ED45C0133272B5454F9D1034BCF
:1078A80083F8260010BD00BF040E0020E43D002030
:1078B800704710B504462078FFF7DFFF14F8013F42
:1078C800002BF8D110BD38B504460D46013D14F81B
:1078D800010BEDB2FFF7D1FF002DF7D138BD00BF86
:1078E800014B1878704700BF0C0E0020014B5878E8
:1078F800704700BF0C0E0020024B187880F0010082
:10790800704700BF0C0E0020024B00221A705A70FC
:10791800704700BF0C0E0020014B01221A707047FF
:107928000C0E0020014B01225A7070470C0E0020EB
:1079380082B0002304E0019B01330193009B0133D3
:107948000093009B8342F6D302B0704707B504202A
:10795800012106F01BFB01214FF4804006F046FB95
:107968004FF40073009300238DF80430034801237B
:1079780069468DF8073005F061FF0EBD000802402A
:107988000D4B07B51A680D484FF47A73B2FBF3F242
:107998000B4B013A5A600B4AF02182F8231000225F
:1079A8009A6007221A60084B084A00930121084B85
:1079B80004F072FC0EBD00BFF0020020B43E0020AF
:1079C80010E000E000ED00E00C040020F0030020CF
:1079D80058030020054B1A6812B11A68013A1A6058
:1079E800034B1A6801321A60704700BF743E0020CA
:1079F8008C3E002082B0044B0190019A1A601A68EC
:107A0800002AFCD102B07047743E0020704700BFC6
:107A180040F0BE60024B40F42020D860704700BFA1
:107A280000ED00E0C37810B503B3164B4278DB686D
:107A38008478DB43C3F30223C3F10401C9B202FA19
:107A480001F10F2242FA03F2C9B222400A430E4B57
:107A580001781201CB18D2B283F8002303780122EF
:107A6800590903F01F0302FA03F307E00378012220
:107A7800590903F01F0302FA03F32031024A42F8BE
:107A8800213010BD00ED00E000E100E021F0604190
:107A980021F07F01014B08439860704700ED00E03A
:107AA800044B1A6909B1104301E022EA0000186189
:107AB800704700BF00ED00E0044B1A6804280CBFB3
:107AC80042F0040222F004021A60704710E000E05D
:107AD800034A044B1A60044A044B1A60704700BFFB
:107AE8000000FA45B41A0020DB0FC93FB01A002085
:107AF800034B00221A60034A034B1A60E8E700BFF1
:107B0800E84400200000FA45AC19002007EE100AEE
:107B1800024BF8EEC77AC3ED007A7047AC19002023
:107B280038B510EE100A07F0E3FD0DA3D3E90023E2
:107B380007F032FE084B044618680D4607F0D8FDDA
:107B48000B4602462946204607F050FF08F006F982
:107B5800024B186038BD00BFB41A0020B01A0020CC
:107B6800182D4454FB2119402DE9F04F2DED048BBD
:107B78009D4C89B04FF00008A1469C4B38F8035043
:107B88009B4B258038F803609A4B6680186807F08D
:107B9800AFFD8DA3D3E9002307F0FEFD08F096F8AA
:107BA8006368954AC018011101F580610905090D3E
:107BB8006060C0F30B1008AF32F8203032F8212093
:107BC800616A238115FB02F0628115FB03F516FB40
:107BD80002F216FB03F607EB4103E0602561C0F3F0
:107BE800CF30C5F3CF356261A661C2F3CF32C6F399
:107BF800CF3623F8200C23F8105C23F8182C23F830
:107C0800086C7E4BA08301310B40002BE583228456
:107C1800668403DA013B63F003030133C9F82430B7
:107C2800002B40F0C5807648764A774E774D6946F6
:107C3800042309F0E1F87648764A04A9042309F0F8
:107C4800DBF87548754A02A9042309F0D5F8744A87
:107C5800744806A9042309F0CFF8B4F9283007EED0
:107C6800903AB4F92A30B8EEE79A07EE903AB4F9A8
:107C78002C30B8EEE78A07EE903AB4F92E30F8EED9
:107C8800E79A07EE903AF8EEE78A68EE087A49EE46
:107C9800097A17EE900A07F02BFD41EC100B09F05A
:107CA8003DFF51EC100B08F059F868EEA87A49EE40
:107CB800A97A306017EE900A07F01AFD41EC100B14
:107CC80009F02CFF51EC100B08F048F868EE897A9F
:107CD80058EE297A28EE288A286009EE298A17EEB4
:107CE800900A07F005FD824618EE100A8B4607F049
:107CF800FFFC4BEC10AB41EC110B09F087FE51EC8B
:107D0800100B08F02BF8484B1860286807F0F0FCB7
:107D18002FA3D3E9002307F0B1FF08B1434B2B6031
:107D280096ED000AD5ED007A80EE270A404F87EDE0
:107D3800000A09F03DFE00B9FEE73B4E3D4D3068B4
:107D480007F0D6FC24A3D3E9002307F025FD8246DB
:107D580028688B4607F0CCFC21A3D3E9002307F061
:107D68001BFD02460B465046594607F063FB07F0D9
:107D7800F5FF2860306038682F4D07F0B9FC16A36E
:107D8800D3E9002307F008FD824628688B4607F0F0
:107D9800AFFC13A3D3E9002307F0FEFC02460B4611
:107DA8005046594607F046FB07F0D8FF2860386070
:107DB80008F10208B8F5007F7FF4DFAE09B0BDEC2A
:107DC800048BBDE8F08F00BF39D6C56D305FC44065
:107DD8008DEDB5A0F7C6B03E9A9999999999B93F92
:107DE800CDCCCCCCCCCCEC3F200E0020C623002040
:107DF800001C0020B01A00209065040803000080D1
:107E080008020020480E0020F0440020E44400202E
:107E1800FC0100204A0E0020F00100204C0E00203A
:107E28004E0E0020E4010020D4440020BD378635E2
:107E3800DC440020D8440020EC440020014B93EDA2
:107E4800000A7047DC440020014B93ED000A70479C
:107E5800D4440020014B93ED000A7047EC44002005
:107E6800014B93ED000A7047D8440020014B93ED75
:107E7800000A7047F0440020014B93ED000A704758
:107E8800E4440020AFF3008010B5FEF783F800202B
:107E9800012324210246FEF7E7F8114B1C78002045
:107EA800012C05D10146FEF7B8F92046002104E06F
:107EB8000721FEF7B2F901200721FEF7AEF9632288
:107EC8001221C020FFF710F902200121FEF7A5F9C1
:107ED800FEF782FA0120BDE81040FEF772BA00BF33
:107EE800280F00200D4B1B78012B05D10C4B0D4A98
:107EF800196812688A181A600B4B1B78012B084BFB
:107F0800196805D1094A914207DD01321A607047A4
:107F1800074A914201DD01321A607047443E002051
:107F2800AC440020403E0020280F00207FD1F008FC
:107F3800FF1FA1070E4B1B78012B05D10D4B0E4AD5
:107F4800196812688A1A1A600C4B1B78012B094BA6
:107F580005D10B4A1968914208DC1A6070471A6803
:107F6800B2F57A2FDCBF4FF47A221A60704700BF4F
:107F7800443E0020AC440020403E0020280F002052
:107F880040420F002DE9F04F824657488BB0B0FBB6
:107F9800F1F00C4607F08AFB41EC100B09F004FCE9
:107FA80051EC100B07F0BAFEC307074648BF471E3F
:107FB80004FB07F007F07AFB45A3D3E9002307F099
:107FC80015FD04460D4645EC104B09F0EDFB59EC48
:107FD800108B204642464B46294607F029FACDE940
:107FE80004014946404607F099FE3BA3D3E9002324
:107FF8000990DDE9040107F04BFE00283DD100247B
:1080080001234FF01509224698462046DFF8E0B0D4
:1080180003E0234642462C46B04600FB04355D4546
:108028002ED800FB0826DDE904012DA3D3E900239F
:1080380007F02EFE30BBDDE9042300202B4907F0B2
:10804800D5FC41EC100B0390029109F0ADFB0398AD
:10805800029953EC102B8DED060B07F0E9F909F1A5
:10806800FF39CDE904015FFA89F9DDE9060107F076
:1080780055FEB9F1000FCCD104E00125002601E03E
:1080880025464646099BD9B2BAF1000F0BD13246B4
:108098002B465046FDF7E8FF012300935046514612
:1080A8003A46534609E032462B460120FDF7DCFFED
:1080B8000120009001463A460023FEF7C8F8FEF773
:1080C8008BF901200BB0BDE8F04FFEF77AB900BF7D
:1080D8000000000084D77741956479E17FFDA53DD4
:1080E800BBBDD7D9DF7CDB3D00E9A4350000F03FFC
:1080F800FFFF0F00214A224B1278012A10B51860A1
:1081080009D1204A904201DD01321A601E4A1B68DB
:1081180093420DDC0AE01D4A904201DD01321A60EB
:108128001B68B3F57A2F03DC4FF47A22144B1A60DC
:10813800134B174A1968174B174C1B68CB189342F7
:1081480023601ADC0020FFF71DFF01202168FFF7DC
:1081580019FF0A4B1C780020012C05D10146FEF7B7
:108168005CF82046002104E00721FEF756F80120BC
:108178000721BDE81040FEF750B810BD280F0020B9
:10818800AC4400207FD1F00840420F00FF1FA10738
:1081980080D1F008C4440020C8440020014B18686E
:1081A800A8E700BFA83E002008B5FEF787FC094BEA
:1081B8005A78187002435A701AB19A7801329A7034
:1081C80030B99B78034A012B02D90023537093706E
:1081D80008BD00BF500E002007B50420012105F09E
:1081E800D5FE4FF46043009301238DF80430022339
:1081F8008DF805300448002369468DF806308DF85F
:10820800073005F01BFB0EBD00080240084B1A683A
:108218004FF47A73B2FBF3F2064B013A5A60064AFE
:10822800F02182F8231000229A6007221A60704712
:10823800F002002010E000E000ED00E0034B5A6877
:1082480012B15A68013A5A60704700BF500E0020B8
:10825800024B58605A68002AFCD17047500E002023
:1082680030B585B004460D4601A85C490A220BF0DA
:10827800E3FE5B4B1B78032B10D8DFE803F0020505
:10828800080B01A8574907E001A8574904E001A8CD
:10829800564901E0564901A80BF0B8FF04AA131982
:1082A80013F80C3C5D19EDB22F2D01D80A3502E008
:1082B800392D01D90A3DEDB204AB1C194FF6FF70F8
:1082C80004F80C5CFCF7C0FD0020FCF7BFFE0DF1C4
:1082D80003050F24204623345A21002315F8012FC3
:1082E800A4B2FCF7CDFEB4F5A57FF3D164205A21E2
:1082F8002C220023FCF7C4FE0023CD205A212C2277
:10830800FCF7BEFE0020FCF79FFD354B1B78032BC6
:1083180062D8DFE803F002284B5601A931480BF078
:1083280075FF0A2200212F480CF014F9314A324B0C
:1083380012781860012A06D1304A904201DC0132D5
:108348001A602F4A06E0B0F5FA5FBCBF4FF4FA5244
:108358001A602C4A1B689342C4BF274B1A602A4BE9
:108368001A682A4B20E001A91F480BF04FFF0A2288
:1083780000211D480CF0EEF81E4A254B12781860B3
:10838800012A06D11D4A904201DC01321A601C4ABA
:1083980006E0B0F5FA5FBCBF4FF4FA521A60194A0A
:1083A8001B68934218DD1A4B1A6015E001A90F48A3
:1083B8000BF02CFF0D4800210A220CF0CBF8154BCE
:1083C80009E001A90A480BF021FF094800210A2207
:1083D8000CF0C0F8104B186005B030BD8FA9050827
:1083E800A63E0020783E00209C3E0020B14400209C
:1083F800683E0020280F0020B03E00203F420F00BA
:1084080080D1F00840420F00A83E0020AC44002074
:10841800CC440020A4440020643E002010B50D4B3D
:108428000D4C1A680D4821460BF0C8FE0C4B0D4840
:108438001A6821460BF0C2FE0B4B0C481A682146FD
:108448000BF0BCFE0A4B0B481A682146BDE81040E9
:108458000BF0B4BEB03E002099A90508783E002074
:10846800CC4400209C3E0020A4440020B1440020BD
:10847800643E0020683E00209FED010A704700BF5F
:10848800000000009FED010A704700BF00000000D7
:108498009FED010A704700BF000000007047704759
:1084A80018B1012801D1034B00E0034B1868FFF70E
:1084B80021BE00BF983E0020A83E002010B9034B03
:1084C80018687047024B1868704700BFB03E00201C
:1084D800A83E002010B9034B18687047024B186873
:1084E800704700BFCC440020983E002008B54FF4E8
:1084F8009570FEF719FA40F26523C31A584240EB0B
:10850800030008BD08B5C620FEF70EFA40F28D1329
:10851800C21A504240EB020008BD4FF4957040F279
:108528006521FEF7F3B9C62040F28D11FEF7EEB9CA
:10853800704760EEA00AB7EE007AF0EE606A70EE5F
:10854800077A40EE006A47EEA70A36EEC77A08B502
:10855800C7EE200A10EE900A07F0CAF80022084B6E
:1085680007F01AF90022074B06F064FF07F0F6FB44
:1085780007EE900AFDEEE77A17EE900A9F3008BDE5
:10858800000059400000E03F38B52DED028BF7EEB2
:10859800008AB0EE608A70EE288A10EE900A28EE03
:1085A800088A07F0A5F808EEA88A00220F4B07F002
:1085B800F3F8044618EE100A0D4607F099F802463B
:1085C8000B462046294607F011FA0022084B06F010
:1085D80031FF07F0C3FB07EE900AFDEEE77A17EECE
:1085E800900A7730BDEC028B38BD00BF00006940AF
:1085F8000000E03FF0B56A4D2DED068B95E80F00C1
:108608008DB008AE103586E80F000FCD01AC0FC451
:1086180095E807004FF6FF7384E807009F2077214D
:108628006422FAF7B6F8A020772164224FF6FF7388
:10863800FAF7AFF89E20772164224FF6FF73FAF716
:10864800A8F89F20762164224FF6FF73FAF7A1F865
:108658004FF6FF73782164229F20FAF79AF80020DA
:10866800FBF7B1FC9F2077216522FCF72FFC9F20A8
:1086780077216422FCF72AFC07AD0C36F7EE009A46
:108688000435F7EE008A95ED009A4FF49674B0EE33
:1086980068AA18EE900A07F02BF83FA3D3E9002345
:1086A80007F07AF807F05AFB08EE900A38EEE98AE4
:1086B800B0EE490AF0EE480AFFF73BFFB0EE490A70
:1086C800F0EE480A0746FFF75FFFBFB281B20F22FC
:1086D8003846FBF743FD013CDBD14FF49674F7EEC7
:1086E800008A18EE900A07F003F82BA3D3E90023B9
:1086F80007F052F807F032FB08EE900A39EEE88AE4
:10870800B0EE490AF0EE480AFFF713FFB0EE490A47
:10871800F0EE480A0746FFF737FFBFB281B20F22D3
:108728003846FBF71BFD013CDBD1B542A8D16C46AE
:1087380007AE043494ED009A4FF4C875F7EE008A3A
:1087480018EE900A06F0D4FF13A3D3E9002307F02C
:1087580023F807F003FB08EE900A38EECA8AF0EE19
:10876800490AB0EE480AFFF7E4FEB0EE480AF0EE18
:10877800490A0746FFF708FFBFB281B20022384610
:10878800FBF7ECFC013DDBD1B442D2D10DB0BDEC1E
:10879800068BF0BDAFF30080295C8FC2F528F03F4F
:1087A80090A50408121A06EE902A081AB8EEE67A7E
:1087B80006EE900AF8EEE67AC7EE277A9FED047A7D
:1087C80067EE877AFDEEE77A17EE900A704700BFEA
:1087D8000000A0438A1A06EE902A081AB8EEE67A34
:1087E80006EE900AF8EEE67AC7EE277A9FED047A4D
:1087F80067EE877AFDEEE77A17EE900A704700BFBA
:108808000000484370B506460D460024610704D5AC
:10881800A0B231462A46FBF7A1FC0134B4F5A07F8B
:10882800F4D170BD70B506460D460024600704D526
:10883800A1B230462A46FBF791FC0134C82CF5D189
:1088480070BD114B11481B781149124A0068012B61
:10885800114B09D1126808601A60104B1A68104B46
:108868001A60104B1A680CE01268D2011A600B4BA0
:108878001A680B4BD2011A600A4B1A68C0010860CB
:10888800D201094B1A607047280F0020B03E002023
:10889800A83E0020CC440020983E0020A44400209C
:1088A800403E0020843E0020C4440020014B18684C
:1088B800FFF720BCA83E002008B5FFF7C2FFBDE8BF
:1088C8000840F3E770B500210A222748274D284EB3
:1088D800284C0BF03FFE00210A22286026480BF0A6
:1088E80039FE00210A22306024480BF033FE0021B3
:1088F8000A22206022480BF02DFE224B32681860B5
:108908002B682149D31A06EE903A2368B8EEE67A26
:1089180006EE903AF8EEE67AC7EE277AFCEEE77AAA
:1089280017EE903A9AB20B80531C07EE903AB8EEC5
:10893800E77AF4EE007A67EE277A144BFCEEE76AE2
:1089480016EE901A8AB206EE902AB8EEE67A1980E8
:1089580077EEC77AF5EEC07AF1EE10FA01DD013252
:108968001A80BDE87040A7E7783E0020B03E00209E
:10897800CC440020A44400209C3E0020B1440020A8
:10898800683E0020643E00202448002084480020DF
:108998000022F0B51346202603254FF02C0C00E0EA
:1089A8002646303EF6B217460132092E10F8014B22
:1089B8000AD897FBF5F605FB16772FB9CE1801F8FC
:1089C80003C07470023301E0CC540133092AE7D1A3
:1089D8002022CA54CB1848225A707A229A70002250
:1089E800DA70F0BDF0B51F46144B1E788DB0054601
:1089F8000C4606B3A6F1040CDCF1000646EB0C06A7
:108A0800CEB90F4908A80BF0D9FB08A86946FFF7AB
:108A1800BFFF0C496A4604A80BF0D0FBBDF848001C
:108A2800FCF712FA3846FCF725FA2846214604AA2C
:108A38003346FCF743FB0DB0F0BD00BF443E0020B9
:108A48008CA00508FAA605082DE9F04F7E4B2DED00
:108A5800068B93ED008A78EE087A7C4B85B017EE8A
:108A6800900A1C6806F044FE80462046894606F0B7
:108A78003FFE68EE088A41EC100BF7EE009ACDE94C
:108A8800020108F039FE78EEA97A57EC106B17EE60
:108A9800900A06F02DFE32463B4682468B464046FB
:108AA800494606F079FE02460B465046594606F0FE
:108AB800BFFC07F053F979EEE88A09EE100AC8EE10
:108AC800898ADFED637A9DED020B68EEA78A08F0CC
:108AD80013FF404653EC102B494606F05DFE064650
:108AE80019EE100A0F4606F003FE02460B46304602
:108AF800394606F07BFF574B002206F04DFE07F083
:108B08002DF909EE100A69EE097A48EEA87AB1EE55
:108B180049AA88EEA77A504B5C60D8608AEE27AAEB
:108B280083ED008AC3ED028A83ED047A83ED05AAFA
:108B38004A4B1B78033B042B6ED8DFE803F0031283
:108B4800254E3C0018EE900A06F0D2FD044619EEB8
:108B5800100A0D4606F0CCFDCDE900014048414918
:108B68000DE017EE100A06F0C3FD04461AEE100ACF
:108B78000D4606F0BDFDCDE9000139483A492246C7
:108B88002B460BF01BFB47E018EE100A06F0B0FD71
:108B980041EC100B08F03CFF0022344B51EC100B59
:108BA80006F0FAFD07F0DAF806F0A2FD02460B46D9
:108BB8002B482F492EE018EE100A06F099FD1EA347
:108BC800D3E9002304460D46DDE9020106F0E4FD81
:108BD800CDE9000122482749D1E718EE100A06F02E
:108BE80087FD17A3D3E9002307F066F8DFED227AA3
:108BF800002818BFB0EE678A78EE297A79EEC89A0D
:108C0800C7EEA99A19EE900A06F072FD02460B46C5
:108C180013481A490BF0D2FA114C00230220CA213A
:108C28002246FCF74BFA0023237005B0BDEC068BF7
:108C3800BDE8F08FAFF30080F6285C8FC2A54C40EA
:108C4800AE47E17A14AEEF3F284500202C450020BE
:108C58000000484200004940EC470020C044002082
:108C6800FA4400209FA90508AFA90508000034C0F0
:108C7800BFA90508D1A90508A4707D3FEDA905087D
:108C88002DE9F0434FF47F708DB0FDF74DFE0027BE
:108C98001FFA80F86BE04FEAC7091FFA89F909F54E
:108CA80080691FFA89F0FEF761FB60F3070409F198
:108CB800010080B2FEF75AFB60F30F2409F10200AD
:108CC80080B2FEF753FB60F3174409F1030080B24A
:108CD800FEF74CFB60F31F6409F1040080B2FEF755
:108CE80045FB60F3070609F1050080B2FEF73EFB7D
:108CF80060F30F2609F1060080B2FEF737FB09F191
:108D0800070960F307051FFA89F0FEF72FFB60F3E8
:108D18000F25B0B206F0DAFC00221B4B06F03CFD32
:108D280007F01CF806F0E4FCCDE90001A8B206F053
:108D3800CDFC11A3D3E9002306F07AFB10A3D3E9F5
:108D4800002306F053FE07F009F806F0D1FC22468E
:108D5800CDE902010D4905A80BF030FAC1B205A80A
:108D680003F044F90120FFF773FA0137BFB2B845A1
:108D780091DA0DB0BDE8F08300000000C0FFDF40CD
:108D8800E17A14AE47C166400000F03EF8A9050834
:108D980008B50021C620FDF7B9FD4FF495700021F4
:108DA800BDE80840FDF7B2BD024B4FF6FF721A80CE
:108DB800704700BFF844002000200146C82240F256
:108DC8003F13FBF705BB07B50DF1070003F00FF9DB
:108DD8009DF807000EBD08B5FFF7F5FF0028FBD189
:108DE80008BD30B5044687B010EE100A0D4606F0EF
:108DF8007FFC02460B4601A805490BF0DFF9204627
:108E0800294601AA0023FCF759F907B030BD00BF75
:108E18000BAA050808B5084803F072FF06480221A6
:108E280004F03FF80028F9D0034803F095FF07EE57
:108E3800900AB8EE670A08BD0020014010B50C4C36
:108E480000232DED028B23809FED0A8A06E0FFF7B1
:108E5800E1FF238838EE008A013323802388182B0A
:108E6800F5D99FED050A28EE000ABDEC028B10BD6E
:108E7800103E002000000000ACC8683910B54FF45F
:108E8800C770FDF751FDDB2805D14FF4C870FDF719
:108E98004BFD84B219E041F2E104214644F201009D
:108EA800FDF734FD44F20100FDF73EFDA04214BF7A
:108EB80080244FF4007421B24FF4C870FDF726FDEA
:108EC8004FF4C770DB21FDF721FD204610BD024B92
:108ED80000221A70704700BF26480020014B01226B
:108EE8001A70704726480020014B00221A6070470C
:108EF80024450020014B1878704700BF2648002001
:108F08000030024B18BF0120187070472748002016
:108F18000D4B1A680D4B1A600D4A002313700D4A49
:108F2800012111700C4A4FF6FF7010800B4A137024
:108F38000B4B1A780B4B002A14BF052204224FF062
:108F480080401A7005F083BCA83E0020AC44002085
:108F580026480020120E0020F84400204446002035
:108F68001C0E00201D0E002070EEA10A88B030EE05
:108F7800010A08B0704770EEE10A88B030EE410A85
:108F880008B07047F0EE407A20EEA10A60EE810A40
:108F980047EEA10A88B017EE810A08B07047D0B52D
:108FA80061EEA17A41EE017A2DED048B17EE900A5D
:108FB80088B0B0EE409AF0EE609AF0EE418AB0EEDA
:108FC800618A06F095FB0022002306460F4606F04C
:108FD8004BFEE8B969EE887A49EE287A29EE088AC4
:108FE80017EE900A06F084FB32463B4606F0FEFC7C
:108FF80019EEA88A06F0B2FE044618EE100A06F02A
:1090080077FB32463B4606F0F1FC06F0A7FE01E08E
:109018000448044600EE900A00EE104A08B0BDEC81
:10902800048BD0BD0050C347F0EE407A86B020EEE6
:10903800200A67EE810A06B070472DE9F04F2DED42
:10904800028B85B0FEF7FAFE10EE105AFEF7FCFE12
:10905800284610EE104A06F04BFB8046204689460B
:1090680006F046FB41EC100B41EC180B08F044FBF2
:1090780057EC106BB0EE480AF0EE680A08F03CFCBA
:1090880032463B46404649465BEC10AB06F084FB53
:1090980006F064FE9FED138A07EE100ADFED127AE0
:1090A80057EE087A114C5B46C4ED007A52464046AA
:1090B800494606F071FB06F051FE07EE900A27EECE
:1090C800888A04AB84ED018A94E8030003E903006D
:1090D800DDED030A9DED020A05B0BDEC028BBDE88B
:1090E800F08F00BF0000F04200008C42884800204A
:1090F800F7EE007A77EEC07A20EE022A20EE210AF7
:1091080007EEA00AF0EE420A47EE810A88B008B0DE
:10911800704770B56D4B2DED068B1A786C4B94B07B
:109128000E468DED020ACDED030A22B91A68802396
:1091380092FBF3F200E01A68664C012E236C616C16
:10914800DFED659AB7EE00AA51D002D3022E60D1A6
:1091580054E0D21A07EE102ACB1AB8EEC79A07EED7
:10916800103AF8EEC77AD4ED000A89EE279A94ED02
:10917800011AD4ED021A94ED032AB0EE490AFFF75A
:10918800B7FF8DED000ACDED010A9DE8030006AB9F
:10919800D4ED040A94ED051AD4ED061A94ED072AC5
:1091A80083E80300B0EE490AFFF7A2FF8DED000A3D
:1091B800CDED010A9DE8030008AB83E80300D4ED78
:1091C8000C0A94ED0D1AD4ED0E1A94ED0F2AB0EE98
:1091D800490AFFF78DFF8DED000ACDED010ADDED9F
:1091E800068A9DED078A04AB9DE803000EE0D4EDE6
:1091F800008A94ED018A08AB103405E0D4ED028AA8
:1092080094ED038A08AB183494E8030083E803005C
:1092180003E0B0EE698AF0EE4A8ADDED030A9DEDBF
:10922800020A30EEC88A70EE688A9DED081ADDEDF4
:10923800091ACDED0C8A8DED0D8AFFF7A3FE8DED91
:10924800000ACDED010A9DE8030010AB83E8030096
:10925800DDED111A9DED101A79EEE11A3AEE411A78
:10926800B0EE680AF0EE480A8DED0E1ACDED0F1A31
:10927800FFF795FE8DED000ACDED010A9DE803008C
:109288000AAD6C4685E803008EB99DED040ADDED54
:10929800050A9DED0A1ADDED0B1AFFF773FE8DED39
:1092A800000ACDED010A9DE8030085E803000AAB3A
:1092B80093E8030014AB03E90300DDED130A9DED09
:1092C800120A14B0BDEC068B70BD00BF280F002039
:1092D800AC440020384800200000000010B5244CA1
:1092E8004FF496702168FDF72EFB61684FF4987073
:1092F800FDF729FBA1684FF49A70FDF724FBE1689C
:109308004FF49C70FDF71FFB21694FF49E70FDF729
:109318001AFB61694FF4A070FDF715FBA1694FF4C2
:10932800A270FDF710FBE1694FF4A470FDF70BFB89
:10933800216B4FF4A670FDF706FB616B4FF4A87024
:10934800FDF701FBA16B4FF4AA70FDF7FCFAE16B86
:109358004FF4AC70FDF7F7FA216C4FF4AE70FDF7DF
:10936800F2FA616C4FF4B070BDE81040FDF7EBBA4B
:109378003848002010B54FF49670FDF7FDFA224CDE
:1093880020604FF49870FDF7F7FA60604FF49A7018
:10939800FDF7F2FAA0604FF49C70FDF7EDFAE0607B
:1093A8004FF49E70FDF7E8FA20614FF4A070FDF7C6
:1093B800E3FA60614FF4A270FDF7DEFAA0614FF4A2
:1093C800A470FDF7D9FAE0614FF4A670FDF7D4FA5E
:1093D80020634FF4A870FDF7CFFA60634FF4AA70CA
:1093E800FDF7CAFAA0634FF4AC70FDF7C5FAE06365
:1093F8004FF4AE70FDF7C0FA20644FF4B070FDF77B
:10940800BBFA606410BD00BF3848002008B5FFF7FC
:109418006DF810B1BDE80840ACE708BD70B500F5BF
:109428008065A8B2FDF7A2FF294C2070681C80B2A5
:10943800FDF79CFF6070A81C80B2FDF797FFA07035
:10944800E81C80B2FDF792FFE070281D80B2FDF79E
:109458008DFF002660F30706681D80B2FDF786FFC2
:1094680060F30F26B6B207EE906AB8EE677ADFEDC2
:10947800197A194B67EE277AA81DC3ED007A80B2D6
:10948800FDF774FF0026073560F30706A8B2FDF75D
:109498006DFF60F30F26B6B2A6F5FE46FF3E07EE57
:1094A800106AF8EEC77A17EE900A06F021F906A3BB
:1094B800D3E9002306F09AFA06F050FC074B22681D
:1094C8001860074B9A6170BDCDCCCCCC0C5FC44002
:1094D8003046002000008037284500202C45002019
:1094E800EC47002013B50446002840D0244B1888C8
:1094F8000419A4B222B2002A05DB40F23F139A42B3
:10950800C8BF1C4600E00024FAF73CFEA0B24EF2A9
:109518009C71FAF749FE1A4B1C801A4B188824B222
:10952800604306F0D3F814A3D3E9002306F05EFAEB
:1095380006F014FC07EE900AFCEEE77A17EE900AA4
:10954800C00080B2FFF76AFF4FF6FF7300930E4B1F
:109558000520DC219A690023FFF744FA0B4B0C48DD
:109568001A780C4902B0BDE81040FFF76DBA02B096
:1095780010BD00BFAFF300800000000000F0734092
:10958800F844002024480020EC470020C044002074
:10959800284500202C4500202DE9F04F2F4D2DEDBA
:1095A800088B2B78022BBDB009D12D4B1A682D4B97
:1095B80042F210701A60FDF7B5FF00F018BE2A4B92
:1095C8001B78B7EE00AADFED29BA002B5ED0284E33
:1095D800284C3068C00080B2FFF720FF2278264868
:1095E8002649FFF731FA264B26499F69D3F804A08C
:1095F8000988306893ED009A79EE0A8A7AEE497AFA
:10960800D3ED029AC8EEA78A002293ED038A93ED60
:1096180004BAD3ED05AA1C4BF4EE6B8A9A60DA60A3
:109628000022F1EE10FAC8BFF0EE6B8AF4EE4A8A17
:10963800F1EE10FA48BFF0EE4A8A88421A6140F00B
:10964800DF81022129702178022902D101211975AF
:10965800DA82074B00221A60D2E100BF444600209C
:10966800A83E0020AC4400201C0E0020003C1C46F4
:1096780024450020C0440020284500202C45002017
:10968800EC47002024480020500E0020BE4B1A78DA
:10969800BE4B1F6812B9802397FBF3F7FFF7CDFC89
:1096A8008DED0A0ACDED0B0A0AAC94E80300B84B1D
:1096B80083E80300002193ED000AD3ED010AB548C1
:1096C800FFF727FD8DED0A0ACDED0B0A94E803009C
:1096D800B14B83E8030093ED018ADFEDB07AB4EE75
:1096E8006B8AF1EE10FAC8BFB0EE678ADFEDAC7A8C
:1096F800B4EE678AF1EE10FA48BFB0EE678AFDEE65
:10970800007AB4EEE78AF1EE10FAD3ED009A08DD9C
:10971800B5EE408ADFEDA37AF1EE10FA48BFB0EE5D
:10972800678A68EE088ADFEDA07AB0EE68BA09EEBB
:10973800A9BA19EE900AB5EE40BAF1EE10FA08BFD0
:10974800B0EE67BA05F0D4FF0022984B80468946F0
:1097580005F06EFE044618EE900A0D4605F0C8FFA7
:10976800224682468B462B462046294606F014F8A8
:1097780052465B4605F05EFE41EC100B08F0CEF950
:10978800002240464946894B8DED040B05F052FEF8
:1097980002460B4606F000F852465B4605F04AFEC4
:1097A80041EC100B08F0BAF9DDE9040155EC104B57
:1097B80006F0D4FA294608EE900A204606F0CEFABA
:1097C80009EE100A88EE899A794CF1EE48AACAEE99
:1097D8008BAA89EE8BBA19EE100A05F089FF64A3EB
:1097E800D3E9002306F04AFADFED727A002818BFA1
:1097F800B0EE679ADFED707A6AEEA77AB4EE4A9A0D
:10980800DFED6E8AF1EE10FA17EE900AC8BFB0EEDF
:10981800689A05F06DFFDFED6A7A4BEE4B7A4AEEF7
:10982800EA7A8046894617EE900AC4E9028905F06B
:109838005FFF49EC108B41EC110BC4E9000108F003
:10984800E5F851EC100B06F089FAB4EE4A9AF1EEFD
:1098580010FAA8BFB0EE689A7AEE497A79EE0A8AC9
:10986800584BC8EEA78A1B78DFED4C7AF4EE6B8A6A
:10987800F1EE10FAC8BFF0EE678AF4EE4A8AF1EE0C
:1098880010FAF7EE007A48BFF0EE678A022B80F0F4
:10989800004A40F0A9804C4B1B78002B00F0A480B4
:1098A8004A4B4B4C1D682C40002C03DA013C64F0F9
:1098B8000704013419EE100A05F01AFF0022454B7F
:1098C80005F06AFF06F02AFA0646504605F010FF32
:1098D80029A3D3E9002305F05FFF29A3D3E90023D7
:1098E80005F0A8FD06F01AFA3B4B3C491F6001EB56
:1098F800C403C7F307225A76C7F307429A761E773E
:109908003A0E9877C6F30726C0F307201F76DA7653
:109918005E77D877324B4FF008081B8895FBF8F82C
:109928004FEA88189D421FFA88F812D108F580601E
:1099380080B218314022FDF795FE054600B1FEE7DA
:10994800224B4FF47F70B3F90010FCF7DFFF1E4B7A
:109958001D70072C48D108F580681FFA88F0214946
:109968004022FDF77FFE00283ED0FEE7AFF30080DF
:109978002D431CEBE2361A3FCDCCCCCC0C5FC44057
:1099880000000000C0FFDF40280F0020AC4400208A
:1099980088480020384800203C460020003C1C46EF
:1099A800003C1CC6CDCC4C3D5F708930000049405E
:1099B8001048002017B7D1380AD7233D72F97F3FE6
:1099C80017B7D139443E00202648002024450020FE
:1099D800070000800000F04030460020500E0020B4
:1099E80024480020680E0020FEF740FA924C84EDCF
:1099F800020AFEF741FA84ED030AFCF753FF2061DF
:109A08008E4B1B78022B21D18D4A8E4B11681B88F7
:109A180099428D4B15DA1978012912D18B4B1B7895
:109A28005BB98B4B8B4A1868126880181860FEF770
:109A380061FB894B1868FEF70BFC814B1A680132F1
:109A48000FE002211970002313600BE0804B1A68A5
:109A5800824B1B689A4205DB7B4B02221A70784BBB
:109A680000221A60744C7E493A4634A80AF0A6FBD4
:109A7800A06805F03DFE02460B4624A879490AF085
:109A88009DFBE06805F034FE02460B4628A876499F
:109A98000AF094FB1BEE100A05F02AFECDE9060138
:109AA800DDE9062371492CA80AF088FB1AEE900A12
:109AB80005F01EFECDE90401DDE904236C4930A858
:109AC8000AF07CFB19EE900A05F012FE02460B46DE
:109AD80010A868490AF072FB18EE100A05F008FE93
:109AE8008046894642464B46634914A80AF066FBFD
:109AF80019EE100A05F0FCFDCDE90801DDE908239F
:109B08005E4918A80AF05AFB504605F0F1FD824656
:109B18008B4652465B465A491CA80AF04FFB18EE82
:109B2800900A05F0E5FD02460B4620A855490AF0C3
:109B380045FB0CA8544922690AF040FBB5EEC08ADF
:109B4800F1EE10FADFED51AA37D5384605F0BEFD23
:109B580033A3D3E9002305F01FFEF1EE487A04464B
:109B680017EE900A0D4605F0C3FD02460B46204647
:109B7800294605F011FE02460B462BA1D1E900014A
:109B880005F034FF06F0EAF89FED417A07EE900AF7
:109B9800F4EEC77AF1EE10FAC6BFC7EEAA7A3D4CCA
:109BA8003D4CF4EEEA7AF1EE10FA36DD9FED377AA5
:109BB8003A4D3B4CC7EE877A7DE01DA3D3E90023DD
:109BC8004046494605F0E8FD044638460D4605F08E
:109BD8007DFD13A3D3E9002305F0DEFD02460B4605
:109BE8002046294605F002FF06F0B8F807EE900A6D
:109BF800F4EECA7AF1EE10FA46BF67EEAA7A294C5B
:109C0800294CF4EEEA7AF1EE10FA53DD9FED1F7A53
:109C1800264D274CC7EE877A4DE0204D4BE000BF1C
:109C28001F85EB51B81E1940000000A2941A6D421E
:109C38000000000080842E41500E0020443E002089
:109C48002445002024480020444600201C0E002003
:109C5800AC440020403E0020643E0020983E002096
:109C680025AA05082FAA05083AAA050845AA05083D
:109C78004FAA050859AA050864AA05086FAA050885
:109C88007AAA050885AA050891AA050800007A4459
:109C98000024744916AA050813AA05082AAB050862
:109CA8001FAA05081CAA050819AA050851A2050833
:109CB80022AA05088C4D17EE900A05F019FD2A46D0
:109CC800CDE9000138A8894902940AF077FA884B4F
:109CD8001C68884B1D68884BAF42CCBF0026012604
:109CE800A742D8BF00269E65844B1B78013BDBB298
:109CF800012B00F26E82824B1B78072B00F26982DF
:109D0800DFE813F0080067029A0014017401C90122
:109D18002A02E4017B4B1C78002C40F05A82022076
:109D2800FBF794F94FF6FF70FBF7A4F81F20FBF739
:109D38008BF81921744A23462D20FBF7BFF94FF6FB
:109D4800FF70FBF797F82046FBF77EF80F20B42149
:109D58003A464FF6FF730094FEF744FE0F206E213B
:109D680024AA2346FBF7AAF9A0206E210DEB0002D6
:109D78002346FBF7A3F90F20382118AA2346FBF73F
:109D88009DF9A02038211CAA2346FBF797F90F203C
:109D98005C212CAA2346FBF791F9A0205C2130AA6C
:109DA8002346FBF78BF90F204A2110AA2346FBF71D
:109DB80085F9A0204A2114AA2346FBF77FF90F2032
:109DC8009B21234620AAFBF779F94C4B1B78012BE2
:109DD80005D10F20842138AA2346FBF76FF9464B9B
:109DE8001B69B3F57A7FCCBF4FF4FC604FF4784021
:109DF800FBF740F80023A0209B210CAAFBF75EF993
:109E0800424B1B78012B08D14FF4FC60FBF732F86A
:109E18004FF48C7002213E4A07E04FF6E070FBF7E2
:109E280029F83C4A4FF48C7002210023FBF746F9CD
:109E38001F20FBF71FF8CCE1DFED377A29EE279AD0
:109E480019EE100A05F054FC4BEC10AB804689461D
:109E580007F052FC404653EC102B494605F09CFC99
:109E68001DA3D3E9002305F0E5FA05F02FFF4BEC1D
:109E780010AB044607F040FD404653EC102B494612
:109E880005F08AFC02460B4615A1D1E9000105F050
:109E9800CFFA05F01BFF4FF6E07300930546002349
:109EA8000520DC213A46FEF79DFD134B9B6D53B10F
:109EB8001A4B18881A4B4FF4784619880096A2B2A4
:109EC800ABB2FAF74DFF154B1C60154B4FF6E0701F
:109ED8001D60FAF7B9FF7CE10000000000E0634074
:109EE8000000000000C05D4051A205089EAA0508B8
:109EF800B03E0020CC440020500E0020443E0020FC
:109F0800C04400201C0E0020ABAA0508280F002022
:109F1800CAAA0508CEAA05080000C842384600208B
:109F2800904800200000FA43000000005FED038A1B
:109F3800204629463A46FEF735FCF4EE689AF1EEDB
:109F480010FAC8BFF0EE689AF5EE409A5FED0A7A0B
:109F5800F1EE10FA48BFF0EE679AF4EEE89AF1EEE7
:109F680010FA04461CD8F4EEE79AF1EE10FA17DB63
:109F7800FDEEE99A002019EE902A4FF4FA71FEF7E7
:109F880029FC054656B1AA4B1888AA4B4FF6FF760E
:109F980019880096A2B2ABB2FAF7E2FEA54B1D6093
:109FA800B4EE688ADFEDA47AF1EE10FAC8BFB0EE1D
:109FB800678ADFEDA27AB4EE678AF1EE10FA48BF3D
:109FC800B0EE678AB4EEE88AF1EE10FA00F2018189
:109FD800B4EEE78AF1EE10FAC0F2FB80BDEEC88A53
:109FE800974818EE102A4FF4FA71A2E02046294645
:109FF8003A46FEF7D7FBB5EEC0BAF1EE10FA0446C2
:10A0080025DDDDE906017CA3D3E9002305F036FE52
:10A01800E8B17BA3D3E90023DDE9060105F0BCFB29
:10A0280002460B460020874905F002FA05F04EFE6D
:10A03800054656B17E4B18887E4B4FF6FF76198839
:10A048000096A2B2ABB2FAF78BFE7A4B1D60DDE93F
:10A0580004016DA3D3E9002305F02EFE002800F0CB
:10A06800B880DDE9040164A3D3E9002305F006FE06
:10A07800002800F0AE8066A3D3E90023DDE90401DF
:10A0880005F08AFB02460B4600206F4905F0D0F91F
:10A0980005F01CFE4FE0204629463A46FEF782FBB3
:10A0A8005DA3D3E900230446DDE9080105F004FEB9
:10A0B80050B19DED080B07F0ABFC002251EC100BE2
:10A0C800624B05F069FB6FE0C82570E054A3D3E943
:10A0D80000235046594605F05FFB53A3D3E90023FC
:10A0E80005F084FC05F03AFE294608EE100A3A46C7
:10A0F8002046FEF757FBDFED567A49EE677A0446AD
:10A10800FDEEE77A17EE905A56B1494B1888494B3D
:10A118004FF6FF7619880096A2B2ABB2FAF720FE86
:10A12800BDEEC88A434B18EE102A1D606FF0B300CD
:10A13800B421FEF74FFB474B9B6D054653B13C4B93
:10A148001888454B4FF4FC6619880096A2B2ABB24A
:10A15800FAF706FE404B39E0DFED407AF4EE678A05
:10A16800F1EE10FAC8BFF0EE678AF4EEE78AF1EE76
:10A1780010FA2ED83A4620462946FEF713FB044625
:10A1880018EE900A05F0B4FA41EC100B07F040FC09
:10A1980000222D4B51EC100B05F0FEFA02460B463F
:10A1A8000020284905F044F905F090FD0546294BA3
:10A1B8009B6D53B11E4B18881E4B4FF6FF761988BE
:10A1C8000096A2B2ABB2FAF7CBFD1A4B1D60184B42
:10A1D8001C60234B1B78022B09D043B14FF6FF7349
:10A1E80000930520DC213A460023FEF7FBFB3DB037
:10A1F800BDEC088BBDE8F08F9A9999999999B93F68
:10A208000000000000409F409A9999999999B9BF18
:10A218000000000000408F4089B5F81400E3693F52
:10A2280000000000008076401F85EB51B81E1940E1
:10A2380038460020904800200000FA430000FAC386
:10A248000CFEFFFF0000694000005940000054C0A8
:10A2580000004843500E0020184500200000C84266
:10A26800C04400202DE9F843461F8846B6B20025B1
:10A278000D4F12E008EB040189B23046F9F736FFBA
:10A2880029F814000A200134FDF74CF9062CF1D105
:10A2980016350136F22DB6B204D06FF0040407EB80
:10A2A8000509E7E7BDE8F883264800202DE9F04FC7
:10A2B80085B00B1A0193431E9BB20293431C441FA3
:10A2C80000F1060901F1FF3A01F1010B9BB20F46BB
:10A2D8001646A4B21FFA89F91FFA8AFA1FFA8BFBED
:10A2E80003938046204651463246F9F737FF204609
:10A2F80039463246F9F732FF204659463246F9F7D1
:10A308002DFF019B0298E518ADB229463246F9F7B0
:10A3180025FF404629463246F9F720FF01340398C5
:10A3280029463246F9F71AFFA4B20A20FDF7FAF8CF
:10A338004C45D7D105B0BDE8F08F2DE9F843461F4D
:10A348008846B6B200250E4F12E008EB040139F832
:10A35800142089B23046F9F701FF01340A20FDF7CD
:10A36800E1F8062CF1D116350136F22DB6B204D03B
:10A378006FF0040407EB0509E7E7BDE8F88300BFC1
:10A38800264800202DE9F0432DED068B70EE007A6B
:10A398008DB017EE900AB0EE408A10EE904A20EE8B
:10A3A800009A05F0A5F9064620460F4605F0A0F9E3
:10A3B800F7EE008A41EC100B41EC1A0B07F09CF900
:10A3C80079EE287A55EC104B17EE900A05F090F9C3
:10A3D8002246804689462B463046394605F0DCF948
:10A3E80002460B464046494605F022F805F0B6FC01
:10A3F800B0EE4A0AF0EE6A0A09EE900A38EEC99AF7
:10A40800DFED377A89EE299A29EE279A07F074FA50
:10A41800304653EC102B394605F0BEF9044619EEC8
:10A42800900A0D4605F064F902460B462046294677
:10A4380005F0DCFA00222B4B05F0AEF905F08EFC96
:10A44800B4EE688ADFED287A284BF1EE10FA04465C
:10A4580019EE100A08BFB0EE678A1D6805F048F9C2
:10A4680002460B4603A8224909F0A8FE204605F03B
:10A478003FF902460B4606A81E4909F09FFE78EEF2
:10A48800287A38EEC88A87EE888A18EE100A05F00E
:10A498002FF902460B4609A8174909F08FFE052037
:10A4A800014603AA0023FAF709FE0520142106AA8B
:10A4B8000023FAF703FEC820052109AA0023FAF7AA
:10A4C800FDFD4FF6E07300930520DC212A460023AA
:10A4D800FEF788FA0DB0BDEC068BBDE8F08300BF2F
:10A4E8000000484200004940A4707D3F30460020EB
:10A4F800D2AA0508A7A90508DAAA05082DE9F84F80
:10A508003F4F3B78022B2DED048B80466AD13D4CA2
:10A518003D4EE08A3D4DC00080B2FEF77FFF3A789D
:10A5280030462946FEF790FA96ED008ADFED387A34
:10A5380068EE277A2F6817EE900A05F0D9F8824658
:10A5480038468B4605F0D4F841EC100B41EC190B5A
:10A5580007F0D2F8504653EC102B594605F01CF979
:10A5680023A3D3E9002304F065FF05F0D7FBB0EE81
:10A57800490AF0EE690A064685B207F0BDF9504669
:10A5880053EC102B594605F007F90B4602461AA161
:10A59800D1E9000104F04CFF05F0C0FB237D8146A2
:10A5A8001FFA80FA2BB9B4F85C00B4F85E10FFF714
:10A5B800C4FE0023284651462375FFF753FE28465C
:10A5C80051461F22FFF772FEB0EE480A00EE907A5D
:10A5D800FFF7D8FEE38AA4F85C609844A4F81680D4
:10A5E800A4F85E90BDEC048BBDE8F88FAFF3008053
:10A5F8000000000000E063400000000000C05D4073
:10A60800C0440020500E0020284500202C45002082
:10A618000000C842174B1B78022B13B50AD1164B02
:10A628001B78022B06D1154C207808B340B2FFF7EF
:10A6380065FF1BE0124CB4F86030ADF80630BDF889
:10A6480006309BB24BB1BDF806004EF29C7180B249
:10A65800F9F7AAFD0023A4F86030074B1B78022BFA
:10A6680006D1064C94F90000FEF73CFF0023237046
:10A678001CBD00BFC044002044460020E22D00203D
:10A68800500E0020054B00201860054B1870054B34
:10A698001870054B1870FDF703BF00BF2445002054
:10A6A800444600201C0E002026480020064B10B50A
:10A6B80000241C60054B02221A702046FDF7F0FEAC
:10A6C800034B1C7010BD00BF2445002044460020E9
:10A6D8001C0E00200B4B1A680B4B1B68D31A06EE96
:10A6E800903A0A4B1B68B8EEE67A06EE903AF8EE16
:10A6F800E67AC7EE277AFCEEE77A17EE900A80B280
:10A70800704700BFCC440020B03E0020A444002085
:10A7180008B5FFF7DFFF044B1880044B1B88834202
:10A728002CBF0020012008BD24480020AC3E00209A
:10A738007047FEE7FEE7FEE7FEE7704770477047A1
:10A74800FDF77CBD10B5094CA37A4BB1084B1A68CC
:10A7580022F006021A6000F013F8204600F079FE95
:10A768004FF48020BDE8104002F0C4BDB43E002084
:10A7780010ED00E0014801F03BB800BFB43E0020F6
:10A78800364BD3F8882042F47002C3F88820344B43
:10A798001A6842F001021A6000229A60196821F0D2
:10A7A800847121F4803119602E495960196882B08A
:10A7B80021F480211960DA60009201921A6842F44B
:10A7C80080321A601A6802F400320192009A01324B
:10A7D8000092019A1AB9009AB2F5A06FF2D1204BF3
:10A7E8001B6813F4003318BF01230193019B012B4D
:10A7F8002ED11B4B1A6C42F080521A641A4A116807
:10A8080041F4804111609A689A609A6842F4004263
:10A818009A609A6842F4A0529A60144A5A601A6878
:10A8280042F080721A6019680D4A8901FBD5104BF5
:10A8380040F205611960936823F0030393609368FD
:10A8480043F002039360936803F00C03082BFAD1DA
:10A85800024B4FF000629A6002B0704700ED00E0D2
:10A8680000380240103000240070004008544007AF
:10A87800003C0240184B194A996801F00C01042960
:10A8880003D0082903D0164B19E0164B17E0596876
:10A898005A6811F4800F596814BF124B104B02F01C
:10A8A8003F02B3FBF2F30C4A5268C2F30142C1F310
:10A8B8008811013252004B43B3FBF2F3074A13608D
:10A8C800054B9A68054BC2F303129A181968127956
:10A8D80021FA02F21A60704700380240F0020020A4
:10A8E8000024F40000127A0037B51C230124002547
:10A8F80001A88DF804308DF805508DF806408DF8C4
:10A908000740FDF78FF82046214603F063FB0A490C
:10A918004CF24F334B60A3F542430B800D814D80C1
:10A928004FF0804003F0FEFE4FF080402146224663
:10A9380004F0BDFA3EBD00BF8849002038B54FF08D
:10A948008040012104F0C8FA00283FD04FF0804031
:10A9580001211F4D04F0CBFA4FF08040002103F095
:10A9680076FF2B78013B042B30D8DFE803F0030790
:10A978000B102000BDE83840F5F706BFBDE83840A9
:10A98800F5F730BFF6F77EF800232B7038BD114B72
:10A9980001221A7000242C70FEF7A0FAFEF7A4FA20
:10A9A8000D4B1878F6F754F90C4B1C7038BD094B51
:10A9B80001221A7000242C70FEF789FAFEF794FA27
:10A9C800054B1878F6F744F9044B1C7038BD00BFE6
:10A9D8001D0E002044460020C0440020120E002016
:10A9E80008B5402002F078FC30B1FAF7C5FC4020E9
:10A9F800BDE8084002F07EBC08BD0000014608B56D
:10AA0800044804F033FC0348402104F0DCFC00282F
:10AA1800F9D008BD00440040F0B589B04FF4E133E7
:10AA28000120019300232B4CADF808301E46014647
:10AA3800ADF80A30ADF80C30ADF810300C23ADF895
:10AA48000E3003F0A3FA4FF40030012103F0C2FAEC
:10AA580020680221072202F071FF072260680321A3
:10AA680002F06CFF0125022704232068059305A93D
:10AA78008DF81A608DF81B508DF818708DF81970C4
:10AA880002F0DCFE08236068059305A98DF81870AC
:10AA980002F0D4FEA06801A904F03EFB2A4640F269
:10AAA80025510D4804F076FC262307A88DF81C30A4
:10AAB8008DF81D608DF81E608DF81F50FCF7B2FFF1
:10AAC800A068294604F0A5FB044A054B1A6009B0A2
:10AAD800F0BD00BF040300200044004005AA0008A0
:10AAE800F4520020024B9868002104F092BB00BF8A
:10AAF8000403002010B5094C40F22551204604F00B
:10AB08006CFC50B1A288D2B2112A02D1044B0121A7
:10AB18001970044B19884A401A8010BD004400403F
:10AB2800160E0020B40E00207047704773B5012040
:10AB3800014603F02BFA264C4FF4D8530093022316
:10AB480003268DF804302046002369468DF8063028
:10AB58008DF807308DF8056002F070FE2046082158
:10AB68000A2202F0EBFE204609210A2202F0E6FE44
:10AB780020460B210A2202F0E1FE0A2220460C217F
:10AB880002F0DCFE01254FF48063204669460093FD
:10AB98008DF806508DF807508DF8056002F04EFECE
:10ABA8000A210A46204602F0C9FE29464FF4804091
:10ABB80003F01CFA8020294603F0F4F94FF0805086
:10ABC800294603F043FA284602F094FB7CBD00BFF7
:10ABD8000000024007B54FF4C060FCF719FF43239B
:10ABE8008DF804300322012301A88DF805308DF873
:10ABF80006208DF80730FCF715FF0EBD7823584363
:10AC08000723B0FBF3F0002301338342FCD97047DC
:10AC18004FF47A735843F1E737B50023104C01938A
:10AC280005460320FFF7EAFFEB681A69013C019229
:10AC380013D0019A002AF4DA019A42F00102019233
:10AC4800019A1A61064A1969013A019102D00199DB
:10AC5800C907F8D40320FFF7D1FF00203EBD00BF8D
:10AC6800410D030010B5C47874B900EB82000333BA
:10AC78009B10D0F8D000224603E051F8044C013272
:10AC8800046004319A42F8D1002010BD033230B577
:10AC98009210D0F8D0400B46002003E02568013020
:10ACA80043F8045C04339042F8D101EB800030BDD6
:10ACB8000122F0B50023827040220129C3708280EE
:10ACC8000CD108230370042343704FF4A073C3808E
:10ACD80002230372C1724FF0A04309E041B90C236B
:10ACE8000370062343704FF4A063C3801F4BC172E7
:10ACF80003F500620261C3604678044601461A46BD
:10AD0800002508E002F5106C02F530620A65C1F80A
:10AD180014C001353A460431B54202F12007F1D397
:10AD280003F58062426103F58862C0F8CC2006789A
:10AD380003F5A0650146002203E0C1F88C500132FA
:10AD480020350431B242F8D31946002202E0C4F893
:10AD5800CC1001320434B24201F58051F7D303F527
:10AD68006063C0F80C310020F0BD00BF0000044053
:10AD780038B5037AC2680025012B044625D1936BA8
:10AD8800417A65F3104309B143F480139363D368A0
:10AD980023F4800323F0500343F010036FF3C3033D
:10ADA8006FF3C7136FF351436FF3D343D360204658
:10ADB800FFF732FFE378012B3ED1052363F3440507
:10ADC800E36845F020059D6036E0D36843F0400312
:10ADD800D360FFF721FF237A627A032B14BF4FF465
:10ADE80034134FF43C130AB143F48013E26814207F
:10ADF8009363FFF70DFFE268217AD368032908BF40
:10AE080043F48033D360237A032B15D1156B0123C8
:10AE180063F39B656FF3D7552D2345F0805563F396
:10AE280016451563C820FFF7F3FEE36845F40005EF
:10AE38001D63C820FFF7ECFEE378012B07D1E36818
:10AE48009D68052262F3440545F020059D600020B9
:10AE580038BDC3689A6842F001029A6000207047C2
:10AE6800C3689A6822F001029A600020704707B50B
:10AE780000230193019B43F020030193019B61F39D
:10AE88008A130193019BC2681361064B1169013B48
:10AE9800019102D001998806F8D40320FFF7AEFE8D
:10AEA80000200EBD410D030007B500230193019B4F
:10AEB80043F010030193019BC2681361064B1169AB
:10AEC800013B019102D00199C906F8D40320FFF78C
:10AED80095FE00200EBD00BF410D030008B5C268F5
:10AEE800D36801296FF35D736FF39E7302D143F04A
:10AEF800005302E009B943F080433220D360FFF7E2
:10AF080087FE002008BDC368586900F0010070473B
:10AF1800C3685B6913F0010F14BF0020012070475C
:10AF2800C368586900F001007047C3685A69986996
:10AF380010407047C3685868704703691A6861F31E
:10AF480001021A607047C268002393614FF0FF3313
:10AF58005361536053610B4B9361C3789169002B24
:10AF680014BF4FF400634FF4016343F4701343F4C8
:10AF7800405343F0080321EA03010B439361002087
:10AF8800704700BF00080080F8B5D0F80C310022E7
:10AF98001A60036915461A6865F3CC221A60C37AE9
:10AFA800012B04461BD10321FFF7C7FFE36880216B
:10AFB8004FF4800261F30F0259629A62C02262F371
:10AFC8000F0561F31F454FF4A072C3F8045162F3F3
:10AFD8000F056FF31F45C3F80851C3F80C51102132
:10AFE8002046FFF744FF2046FFF75EFF2269002353
:10AFF8004FF0FF311361204653611E469161FF25D2
:10B00800D361214610E082691768C7F3076707F024
:10B018008007FFB2002F14BF4FF09047002717603A
:10B02800013316610430956062789342EBD30023B4
:10B038001D46FF2010E04A6D1668C6F3076606F045
:10B048008006F6B2002E14BF4FF090460026166018
:10B05800013315610431906062789342EBD3236920
:10B068001A6942F480721A61E278012A04D1054A09
:10B07800402161F359421A632046FFF764FF00201C
:10B08800F8BD00BF0301010003699B68C3F34103D6
:10B09800013B022B9ABF024AD05C0320704700BFD5
:10B0A800D8A5040810B5036981699C680A68C4F3C7
:10B0B8004100022802D06FF30A0202E0032060F385
:10B0C8000A020A605A6842F480725A60002010BD71
:10B0D80030B54D780B780022012D00EB830405D1A3
:10B0E80005FA03F3A46963F30F0205E0012505FAE5
:10B0F80003F3646D63F31F422368C3F3072505F068
:10B108008005EDB26DB98D6865F30A03CD78C988FD
:10B1180065F3934361F3995343F0805343F4004339
:10B1280023600369D9690A43DA61002030BD30B56C
:10B138004D780B780024012D224600EB830105D1C0
:10B1480005FA03F3896963F30F0205E0012505FA9F
:10B1580003F3496D63F31F4203696FF3CF340C6047
:10B16800D96921EA0202DA61002030BDF8B54F78CA
:10B178000B78012F00EB830349D19E694C69356830
:10B1880033692A4664F3120314B967F3DC430BE00E
:10B198008F68E419013CB4FBF7F7CC7867F3DC431C
:10B1A800012C08BF64F35E733361C378012B06D1A9
:10B1B8000B780C6900EB83039B695C610CE0CB782E
:10B1C800012B09D04B693BB103690C785E6B0127F1
:10B1D80007FA04F434435C63CB78012B07D1036985
:10B1E8009B68DB0554BF45F0005245F080520B7850
:10B1F80000EB830342F004429B691A60CB78012B71
:10B2080038D10A788B8AC968FFF72CFD32E05E6D69
:10B218004F6935688C6833692A462FB964F312037D
:10B22800012464F3DC430AE03F19013FB7FBF4F75C
:10B23800BF05BF0D67F3DC437C4364F3120333613E
:10B24800C378012B05D10B780C6900EB83035B6D88
:10B258005C61CB78012B06D14B7913B145F00052D4
:10B2680001E045F080520B7800EB830042F0044285
:10B27800436D1A600020F8BD73B54D78012D3DD19E
:10B2880083694A691E681C690094E4B242B962F392
:10B2980006048DF800409DF8024065F3C4040EE0F2
:10B2A8008D68AA4286BF4D6165F3060462F3060401
:10B2B8008DF800409DF80240012262F3C4048DF825
:10B2C8000240009A1A61C278012A05D10A780C69ED
:10B2D80000EB82029269546146F004421A60C37816
:10B2E800002B34D14B69002B31D003690A78586B95
:10B2F800012101FA02F202435A6328E00B784E69F1
:10B308008C6800EB83035B6D1A681D690095EDB2CC
:10B3180006B14C6164F306059DF802408DF80050B3
:10B32800012565F3C4048DF80240009C1C61C378B4
:10B33800012B05D10B780C6900EB83035B6D5C6115
:10B348000B7800EB830042F00442436D1A60002042
:10B358007CBD4B78012B0B7800EB83000AD1826906
:10B368001368C3F3076101F08001C9B221B143F04A
:10B37800804301E0426D136843F40013136000201A
:10B3880070474B78012B0B78C97800EB83000CBF12
:10B398008269426D02391368C9B26FF355530129A6
:10B3A80098BF43F0805313600020704703699A697F
:10B3B800D8691040000C704700EB810102694B6DA1
:10B3C8009B6850691840704703699869DB691840A1
:10B3D80080B2704782B000230093C0238DF80330F9
:10B3E8000122002362F3C4038DF8023018238DF87C
:10B3F8000030009A436D1A61C278012A06D100F51F
:10B40800B96058611A684FF080221A6002B070471C
:10B41800D0F8143110B50446D3B103699A68D2073D
:10B4280016D5827A42B1D0F80C21D0F80C116FF3FE
:10B4380041026FF300020A605A6842F001025A6042
:10B448000520FFF7E5FB23695A6822F001025A60DC
:10B4580010BD837A63B103699B68D90708D5D0F812
:10B468000C31D0F80C216FF341036FF30003136024
:10B478007047012310B5002280F8123104460346B4
:10B48800FF2104E058698160186D0132816060789D
:10B4980004338242F6D3236900221A615A61DA61C1
:10B4A8004FF0FF329A612046FFF7FEFC204610213C
:10B4B800BDE81040DBE44B78012B0B7800EB8300F0
:10B4C8000FD183691868C0F3074000F02003DBB28E
:10B4D800CBB900F00200C0B200280CBF30202020F9
:10B4E8007047436D1868C0F3074000F02003DBB2D3
:10B4F8005BB900F00200C0B200280CBF4FF4405006
:10B508004FF400507047102070474FF48050704738
:10B518004B78012B0B7810B500EB83030AD19C699B
:10B52800102A236802D1BDE8104012E7202A0CD067
:10B53800302A0FE05C6DB2F5805F236802D143F4D6
:10B5480000131BE0B2F5005F02D143F0006315E081
:10B55800B2F5405F0FD1C3F3074202F02002D2B226
:10B5680022B100234B71BDE810400AE743F0806325
:10B5780043F0802302E00AB962F3CF33236010BDA1
:10B58800F8B50446FFF794FB0122002384F8122142
:10B5980084F8133128271646194640250CE007FB86
:10B5A80003F000F58C7022182354D3805670D170A4
:10B5B8009560D1605161013362789342EFD30023E3
:10B5C8002826194640250CE006FB03F000F55C70C0
:10B5D80022182354D3805170D1709560D160516185
:10B5E800013362789342EFD32046FFF739FC2046B7
:10B5F800FFF7BEFB00212046FFF770FC2046FFF74F
:10B60800C3FC2046BDE8F840FFF723BC70B5CDB2B7
:10B618000C464FF0280601F07F0106FB010115F0EA
:10B62800800F14BF01F58C7101F55C7104F07F0483
:10B63800ED090C704D708A60CB7005B1CC80022B7F
:10B6480001D100230B71FFF743FD002070BD10B539
:10B65800CAB201F07F034FF0280404FB030312F081
:10B66800800F14BF03F58C7303F55C7301F07F0141
:10B67800D20919705A701946FFF759FD002010BDFC
:10B6880038B501F07F0528246C4304F55C74011972
:10B698004B6100238B614B70EBB20355CA60C478D1
:10B6A800012C08BF0A6113B9FFF7E6FD01E0FFF7B7
:10B6B8005DFD002038BD70B501F07F042825654385
:10B6C80005F58C7541190126E4B2CA600A610022A9
:10B6D8004E7044558A614B6114B9FFF7CDFD01E006
:10B6E800FFF744FD002070BDCAB212F0800F10B5FC
:10B6F8004FF0280306D001F07F0403FB040303F591
:10B708008C7303E003FB010303F55C73D209012486
:10B7180001F07F0119709C705A701946FFF719FEE5
:10B72800002010BDCAB212F0800F10B54FF02803E8
:10B7380006D001F07F0403FB040303F58C7303E0D8
:10B7480003FB010303F55C730024D20901F07F01B8
:10B7580019709C705A701946FFF713FE204610BDE9
:10B7680008B50B0604D501F07F01FFF780FB01E067
:10B77800FFF79AFB002008BD0369002261F30A1253
:10B7880019680A431A60704703695A6803206FF3FF
:10B7980041025A60FFF73CBA03695A68032042F035
:10B7A80002025A60FFF734BA11F0800F4FF02803F5
:10B7B80006D001F07F0103FB010101F58C7103E064
:10B7C80003FB010101F55C71FFF775BE11F0800FF5
:10B7D8004FF0280306D001F07F0103FB010101F5BA
:10B7E8008C7103E003FB010101F55C71FFF790BE6A
:10B7F8002DE9F74F0446FFF78BFB002800F03F8246
:10B808002046FFF792FB0546002800F03882C0F377
:10B81800074000F00800C0B2002861D02046FFF7BA
:10B82800C5FDA146824627464FF00008DFF86CB3F5
:10B838002E4650E01AF0010F46D05FFA88F2114602
:10B8480020460092FFF7B8FD10F0010F0546009A58
:10B8580020D07B6D01259D60E178A94207D11B6945
:10B86800D9F87813C3F31203CB1AC9F88833DBF875
:10B87800003020461B6811469847E378012B09D110
:10B88800B8F1000F06D194F81131052B02D12046EA
:10B89800FFF7A0FD05F00203DBB213B17B6D0225B3
:10B8A8009D6005F00403DBB213B17B6D04259D6038
:10B8B80005F00805EDB23DB1DBF8003020469B6885
:10B8C80098477B6D0820986008F101084FEA5A0AEA
:10B8D800043709F12809BAF1000FABD13546012028
:10B8E800C5F3074303F00403DBB2002B00F0AF807D
:10B8F8002046FFF769FD264683464FF0000801956C
:10B908009FE01BF0010F00F0978023695FFA88F928
:10B9180019695D6B04EB890225FA09F59269ED0155
:10B928009268EDB20D431540EA071CD55A6B012009
:10B9380000FA08F122EA01025A63B369974A98604B
:10B94800136805465B68204649469847E378AB424A
:10B9580009D1B8F1000F06D194F81131042B02D1A6
:10B968002046FFF737FD05F00403DBB213B1B369D6
:10B9780004259D6005F00803DBB213B1B3690825FF
:10B988009D6005F01003DBB213B1B36910259D600B
:10B9980005F02003DBB213B1B36920259D6005F0E3
:10B9A8004003DBB213B1B36940259D6005F0020383
:10B9B800DBB213B1B36902259D6025F07F0515F050
:10B9C800FF0F39D0282505FB084505F58C75C246BB
:10B9D800AB696A69C3EB020CAB689C4528BF9C46FF
:10B9E8000CF1030CB3694FEA9C0C9B696746A046AF
:10B9F80014E0AA68E9681C1B944228BF1446A3B245
:10BA080040464A46FFF72EF9EB681B19EB60AB6915
:10BA1800E71C1C19AC61B3699B69BF089BB2BB42A8
:10BA280005D9AC696B699C4201D2002BE1D1B3699D
:10BA3800802544469D60D04608F101084FEA5B0B1B
:10BA48000436BBF1000F7FF45CAF019D012005F0C7
:10BA58000203DBB213B1E36802225A61C5F307633C
:10BA680003F08003DBB2CBB1A37A43B1D4F80C3135
:10BA7800D4F80C216FF341036FF3000313602369BB
:10BA88005A6822F001025A60444B1B6820469B69A1
:10BA98009847E3684FF000425A610120C5F3072335
:10BAA80003F00803DBB2F3B13C4B1B6820465B692B
:10BAB80098472369E2689B684FF400615161A27A54
:10BAC80082B1DB070ED5D4F80C311A6842F00102B6
:10BAD8001A601A6842F003021A60314B1A6942F080
:10BAE80006021A61012005F00803DBB243B12B4BB3
:10BAF8001B682046DB689847E36808225A610120E2
:10BB080005F01003DBB2002B33D0E3689A6922F00A
:10BB180010029A611F6A282607F00F0306FB0346E6
:10BB2800C7F34343022B06F55C7602D0062B1AD1E5
:10BB38000EE047F6F0733B40ABB1C7F30A17204657
:10BB4800F1683A46FFF7A2F8F368DB19F36007E0FB
:10BB580004F5B96120460822FFF798F8C7F30A17D9
:10BB6800B369DF19B761E3689A6942F010029A6114
:10BB78000120C5F3072303F01003DBB2002B39D0F3
:10BB880023695A68002622F001025A60314620468D
:10BB9800FFF76DF923463246FF2108E0A003002095
:10BBA80000ED00E058698160186D013281606078AD
:10BBB80004338242F6D3236901274FF0FF3267F33B
:10BBC8000F069A6167F31F460F22DE615A612F2222
:10BBD8001A611A686FF30A121A602046FFF7FAFB17
:10BBE800E3684FF480525A61264B1B6820461B6954
:10BBF80098473846C5F3072303F02003DBB2EBB1BF
:10BC08002046FFF74FFAE3682046DE68FFF73CFA64
:10BC1800032806D10023A3704FF40073A3800923DF
:10BC280004E00123A3704023A380052363F38D263A
:10BC3800E3684FF40052DE6001205A61C5F3074300
:10BC480003F01003DBB24BB10E4B1B682046DB69D7
:10BC58009847E3684FF480125A610120C5F30745FD
:10BC680005F02005EDB255B1064B1B6820461B6A4E
:10BC78009847E3684FF400125A610120FFE7BDE8D6
:10BC8800FE8F00BFA003002043230B8000487047AD
:10BC98001003002038B51F4B1A68511C052A19607B
:10BCA80035D11979002201291A6030D09968B1F587
:10BCB800006F08BF9A60174B9968DC68A1421A4662
:10BCC80002D100221A7122E086BFC1F50063136118
:10BCD800C1EB0404D0F8EC3598BF14611569B3F8CA
:10BCE80039300C4C9D428AB204D95918ED1AA1601A
:10BCF800256104E06918A1600021ABB22161054902
:10BD080001240C7104498A188121FFF7D4FC002012
:10BD180038BD00BFB80E0020274A002038B52823B8
:10BD28000A4D03FB01010A4BB1F888131B6904464D
:10BD380028469847D4F8EC352046B3F8403001211E
:10BD48002A46FFF79DFC002038BD00BFDF490020D0
:10BD58008C03002070B50B7813F0600506460C467E
:10BD680025D0202D1FD1CD88B5B113F0800F48788C
:10BD780008D0214B21499B682A469847E2881F49E9
:10BD8800304625E01E4B1D4958641E4B30465D6108
:10BD98002A4600F022FB1DE0174B48789B6829468D
:10BDA8002A46984725E000F077FB022521E04B78EA
:10BDB8000A2B11D00B2B14D0062B1AD14B881B0A37
:10BDC800212B03D1CA883A2A28BF3A220E49304685
:10BDD80000F0EAFA00250CE00C49012200F0E4FA30
:10BDE80007E08B781BB9074A1D46936101E000F014
:10BDF80053FB284670BD00BF8C0300201F4A00205B
:10BE080010030020B80E002022030020D00E0020CE
:10BE180010B581210446FFF71AFC01212046FFF7DF
:10BE280016FC82212046FFF712FC024B5B689847FC
:10BE3800002010BD8C03002038B5D0F8EC3504463E
:10BE4800B3F8392081210223FFF7E0FBD4F8EC3561
:10BE58000121B3F8402020460223FFF7D7FB8221B7
:10BE6800082203232046FFF7D1FB094B02220025B5
:10BE78001A715D71074B1B689847D4F8EC35064A70
:10BE8800B3F8403020460121FFF7FAFB284638BDB9
:10BE9800D00300208C030020DF49002010B5074C98
:10BEA800606CFF2807D0064B064A9B680649526912
:10BEB8009847FF236364002010BD00BF10030020D3
:10BEC8008C030020B80E00201F4A002038B5104906
:10BED8000B79012B19D10C690CB90C7115E0D0F84C
:10BEE800EC358D68B3F839309C42AAB203D95D1994
:10BEF8008D60E41A03E0A3B22C198C6000240C6155
:10BF0800044952188121FFF7D6FB002038BD00BF35
:10BF1800B80E0020274A00200020704700207047F4
:10BF28000023F0B5084A094E1D4609E01468C75CAD
:10BF3800375501340133B4F5006F146008BF15603C
:10BF48008B42F3D10020F0BDC40E0020274A002008
:10BF5800104B114AD3F800C000232DE9F0410F4FD0
:10BF680016461D460DE0146810F8038007F8048093
:10BF78000134802C08BF2C4614603468644505D011
:10BF880001338B42EFD10020BDE8F0810220BDE8EB
:10BF9800F08100BFA8520020BC5200202852002087
:10BFA80021280FD1084B1A680A701A68120A4A70B9
:10BFB8005A888A70DA78CA701A790A715A794A7175
:10BFC8009B798B71002070478403002007B502AB72
:10BFD800012103F8010D1846FFF7A2FF0EBD00214D
:10BFE80000E00131435C002BFBD199E798E70B4B4C
:10BFF8000B491A68096891420BD00A498A5C027099
:10C008001A680132802A1A6005D100221A600120BC
:10C018007047002070470120704700BFA8520020D9
:10C02800BC52002028520020204B1A68204B1B6865
:10C038009A42F0B509D135E00133802B08BF0023BF
:10C048009A4203D11A4B1A602CE01A4CE15C002981
:10C05800F2D00A29F0D00D29EED0154C1549134D10
:10C0680023600E460023CF182268BA5CC2542268A7
:10C0780001339F18802F08BF53422F689A189742A0
:10C0880010D0B25C1AB10A2A01D00D2AEBD10022D5
:10C09800C254074A116859187F29116003D9803999
:10C0A800116000E000231846F0BD00BFBC5200201C
:10C0B800A852002028520020704700BFD0F8E4356D
:10C0C80010B51B6904469847032384F812310020F1
:10C0D80010BD08B5042380F81231D0F8E435DB68C8
:10C0E8009847002008BD08B5D0F8E035DB6903B1F2
:10C0F8009847002008BD08B5D0F8E0351B6A984776
:10C10800002008BD08B5D0F8E0355B6A98470020E4
:10C1180008BD002110B5402204460B46FFF776FA09
:10C128008021402200232046FFF770FA012384F87B
:10C138001231D4F8E435A0785B689847002010BD28
:10C1480013B56946044600F085F99DF8001001F022
:10C158001F03012B07D0022B0AD073B9204669466A
:10C1680000F026FA0FE02046694600F007FA0AE0D8
:10C178002046694600F0A2F905E021F07F01C9B226
:10C188002046FFF7B1FA00201CBD38B50446002947
:10C198003DD190F81131022B42D1D0F83421D0F89A
:10C1A80020319A4211D9C178D21A0129C0F8342114
:10C1B80004D1D0F82411CB18C0F8243192B220460B
:10C1C800D4F8241100F000F92AE0D0F83821B2FBA5
:10C1D800F3F503FB152565B99A420AD3D0F83C312B
:10C1E8009A4206D229462A4600F0EEF8C4F83C5195
:10C1F80016E0D4F8E035DB682BB194F81221032A55
:10C2080001D120469847204600F00FF908E0D0F801
:10C21800E0355B6923B190F81221032A00D19847D1
:10C22800002038BD10B5044659BB90F81131032BD6
:10C2380030D1D0F88C23D0F878339A4214D9C17809
:10C24800D21A0129C0F88C2304D1D0F87C13C9185C
:10C25800C0F87C139A4228BF1A4692B22046D4F8F6
:10C268007C1300F0CAF815E0D0F8E0351B6923B15B
:10C2780090F81221032A00D19847204600F0C6F80A
:10C2880008E0D0F8E0359B6923B190F81221032A21
:10C2980000D19847002010BD2DE9F041069F0446C3
:10C2A800164698460D46FEF741FC20462946C4F836
:10C2B800E085C4F8E475C4F8E865FFF761F9D4F8D7
:10C2C800E4351B6898472046BDE8F041FEF782BC7C
:10C2D80000207047D0F8E03510B504461B68984731
:10C2E800D4F8E4359B689847002010BD08B5D0F80D
:10C2F800E0355B689847002008BD000012230B80DA
:10C3080000487047D003002004230B800048704782
:10C31800E203002010B5044C04480A46214600F008
:10C3280075FA204610BD00BFC0520020E6AA0508D5
:10C338000A4608B50248034900F068FA014808BDF2
:10C34800F9AA0508C05200200A4608B50248034960
:10C3580000F05CFA014808BD07AB0508C052002090
:10C3680008B50A4608B9044800E00448044900F042
:10C378004DFA034808BD00BF12AB05081FAB0508FE
:10C38800C052002008B50A4608B9044800E004482D
:10C39800044900F03BFA034808BD00BF2CAB050870
:10C3A8004DAB0508C052002010B513460C46C0F826
:10C3B8003821C0F83421022280F8112100212246B8
:10C3C800FFF779F9002010BD10B50C46134600217F
:10C3D8002246FFF770F9002010BD10B513460C4631
:10C3E800C0F89023C0F88C23032280F81121002183
:10C3F8002246FFF745F9002010BD10B50C4613463C
:10C4080000212246FFF73CF9002010BD002104233B
:10C4180010B50A46044680F811310B46FFF74BF970
:10C428002046FEF7D7FF002010BD0021052310B5D8
:10C438000A46044680F811310B46FFF721F92046D9
:10C44800FEF7C8FF002010BD282303FB0100B0F849
:10C458008803704790F8C8350B7090F8C9354B7051
:10C4680090F8CB2590F8CA3503EB02234B8090F85F
:10C47800CD2590F8CC3503EB02238B8090F8CF259F
:10C4880090F8CE3503EB02239BB2CB80C0F83C3149
:10C49800012380F81131704710B591F90030002B55
:10C4A800044601DBCB880BB9802100E00021FFF7AF
:10C4B8001BF92046BDE81040FEF78CBF38B50D4685
:10C4C80004466B780979012B10D027D3032B51D15F
:10C4D80090F81231022B28D0032B47D16B889BB9D7
:10C4E80091B1802910D0FFF7FFF80DE090F81231D4
:10C4F800022B1AD0032B39D16B88002B3AD149B1C2
:10C50800802907D0FFF70EF9D4F8E03520469B685C
:10C51800294698472046FFF779FF2BE090F812311B
:10C52800022B02D0032B21D106E019B3802921D098
:10C538002046FFF7D9F81DE011F0800F4FF02803CF
:10C5480006D001F07F0103FB010393F81A2103E0F1
:10C5580003FB010191F87223074B02B101221A6013
:10C56800204605490222FFF71FFF03E0204629461F
:10C57800FFF792FF002038BDD40E002038B590F8A0
:10C588001231032B04460D460CD10B79012B09D827
:10C59800D0F8E0359B689847EB883BB92046FFF711
:10C5A80035FF03E020462946FFF776FF002038BD17
:10C5B80073B54B7804460D46092B00F21C81DFE861
:10C5C80013F0D10008011A01E4001A0172000A00F0
:10C5D8001A01C00092004B881A0A013A062A00F292
:10C5E8000A81DFE812F007001A0027000801080195
:10C5F80008010801D4F8E835A0781B680DF1060198
:10C608009847EB88402B014603D094F81231012B50
:10C618003AD10823ADF8063036E0D4F8E035A078F2
:10C628009B6A0DF106019847022343700146C4F83E
:10C63800EC0529E0DBB2052B00F2DD80DFE803F032
:10C6480003080D12171CD4F8E835A0785B6817E0CA
:10C65800D4F8E835A0789B6812E0D4F8E835A078DB
:10C66800DB680DE0D4F8E835A0781B6908E0D4F859
:10C67800E835A0785B6903E0D4F8E835A0789B69D1
:10C688000DF1060198470146BDF80630002B00F071
:10C69800B680EA88002A00F0B2809A4228BF1A467B
:10C6A800ADF806205CE08B88002B40F0A480CB8896
:10C6B800002B40F0A08094F812214B88032A00F048
:10C6C8009A8003F07F05204684F813512946FFF726
:10C6D80053F82046FFF79AFE0DB1022300E001232C
:10C6E80084F812318BE08978464E0129317100F2C5
:10C6F800828094F81231022B02D0032B7BD108E000
:10C70800002962D00121032384F8101184F8123122
:10C7180013E041B9022384F8123184F8101120463D
:10C72800FFF7E4FD51E094F81011012920464DD09F
:10C73800FFF7DCFD317984F810112046FFF7CAFDB8
:10C7480043E0CA88012A56D194F81231022B02D04C
:10C75800032B50D102E020462B4913E004F58871E1
:10C7680020460FE094F81231023B012B43D8D4F84D
:10C7780014312449002B0CBF0123032341F80C3F3B
:10C7880020460122FFF710FE39E04B88012B29D003
:10C79800022B34D18B8813F0FF0F30D121691B0A8B
:10C7A800013B4A68042B0FD8DFE803F003050709AB
:10C7B8000B00012306E0022304E0032302E0042324
:10C7C80000E0052363F306124A602046FFF71EFEC9
:10C7D80015E094F81231023B012B0CD84B88012B41
:10C7E8000DD10023C4F81431D4F8E03520469B68F5
:10C7F80029469847E9E720462946FFF74DFE0020DD
:10C808007CBD00BFD40E0020DC0E002030B5C8B1BE
:10C818000023DDB20133C41814F8014C002CF8D100
:10C828006B1C5B0013800B7003234B70022305E025
:10C83800CA545A1CD2B202338C54DBB210F8012B02
:10C84800002AF5D130BD00BF704770477047704768
:10C8580070477047704700000EB403B070470A284D
:10C8680010B5044602D10D20FFF7F9FF064A1368F8
:10C878001BB103F8014B136010BD044B1B680BB1CF
:10C888002046984710BD00BFE40E0020F452002057
:10C8980010B5044601E0FFF7E2FF14F8010B002889
:10C8A800F9D110BD2DE9F04F044685B00D464FF083
:10C8B8000A0A00E035462078002800F0C4802528C0
:10C8C80001D0013467E06078302803D1A0780123D3
:10C8D800033407E02D2802D00234002302E0A078B8
:10C8E800022303344FF0000805E00AFB080814F897
:10C8F800010BA8F13008A0F13002D2B2092AF4D90C
:10C908006C2801D04C2803D114F8010B43F0040320
:10C91800002800F09880602886BFA0F12002D2B2DB
:10C9280002464F2A3DD006D8432A2DD0442A09D0A2
:10C93800422A30D133E0552A04D0582A29D0532A24
:10C9480029D101E00A272DE02E1D2F68002500E0DF
:10C9580001357A5D002AFBD104E02020FFF77FFF34
:10C968004D4601E0980704D4454505F10109F4D383
:10C978004D463846FFF78CFF03E02020FFF76FFF96
:10C9880001354545F9D395E728782E1DFFF767FF50
:10C9980090E7102706E0FFF762FF2E468AE7022796
:10C9A80000E008272E1D442A296804D1002902DA4C
:10C9B800494243F00803002200E02A46B1FBF7FE93
:10C9C80007FB1E11CDB2092D714607D9782814BF6F
:10C9D8004FF0070C4FF0270C6544EDB230350DF8D9
:10C9E8000250551CBEF1000F02D0102DE5D10F22C8
:10C9F800190705D504A94D192D2105F8101C951CFA
:10CA080013F0010F0CBF4FF0200B4FF0300B9B07BA
:10CA18002F4604D508E05846FFF721FF4F46474503
:10CA280007F10109F7D34F46013D1DF80500FFF74F
:10CA380016FF002DF8D103E02020FFF710FF013783
:10CA48004745F9D336E705B0BDE8F08F70B5064D18
:10CA58000C462E68286001E0FFF701FF14F8010B6F
:10CA68000028F9D12E6070BDF45200200FB407B52C
:10CA780004A951F8040B0191FFF714FFBDE80E401B
:10CA880004B070470EB417B505A9084C51F8043B1B
:10CA9800206018460191FFF705FF226800231370F4
:10CAA8002360BDE81E4003B0704700BFE40E0020BD
:10CAB8000EB433B505A9074C51F8043B256820602E
:10CAC80018460191FFF7EEFE2560BDE83C4003B033
:10CAD800704700BFF452002070B51E4604461C483B
:10CAE8001546FFF7C3FF022E1FD0042E25D0012EB6
:10CAF8002AD105E0A15D1748FFF7B8FF013600E02D
:10CB08000026AE42F6DB2020FFF7A9FE002609E04A
:10CB1800A05DA0F12003DBB25E2B88BF2E20FFF7BB
:10CB28009EFE0136AE42F3DB0EE034F8021B0A48E3
:10CB3800FFF79CFF013DF8D106E054F8041B0748B5
:10CB4800FFF794FF013DF8D10A20BDE8704086E662
:10CB58006EAB050875AB05087BAB050881AB05080E
:10CB680008B501214FF4807001F07CFA4FF4807011
:10CB78000021BDE8084001F075BA43680A6823F04F
:10CB8800407323F4807313430A7943EA0223436012
:10CB9800CA680B6930B51A4384688D68084B2A4304
:10CBA800234013434A7943EA420383600B7DC26AF8
:10CBB800013B22F47002DBB242EA0353C36230BD88
:10CBC800FDF7FFC000230360037143718360C360F6
:10CBD8000361012303757047074A084B516810B574
:10CBE8000B4090E8120021438468C0682143014348
:10CBF8000B43536010BD00BF00230140E030FCFF31
:10CC08000023036043608360C3607047836811B189
:10CC180043F0010301E023F0010383607047436898
:10CC280023F4400323F400730B43436070474162CD
:10CC380082627047436823F01F030B4343607047C9
:10CC4800044B5A6810B142F4000201E022F40002D9
:10CC58005A60704700230140044B5A6810B142F4EF
:10CC6800800201E022F480025A60704700230140EC
:10CC7800092970B50CB20CD904EB44041E3CC668F3
:10CC88000725A54026EA0505A34045EA0304C46034
:10CC98000AE0066904EB44040725A54026EA0505D1
:10CCA80013FA04F42C430461062A0CD80523013A2C
:10CCB8005A43446B1F23934024EA0303914043EAF9
:10CCC8000102426370BD0C2A12B20CD802EB820238
:10CCD800233A046B1F23934024EA0303914043EA59
:10CCE8000102026370BD02EB8202413AC46A1F234B
:10CCF800934024EA0303914043EA0102C26270BDF3
:10CD0800836843F08043836070478068C0F3805035
:10CD18007047836811B143F4806301E023F48063B2
:10CD280083607047836811B143F0020301E023F088
:10CD38000203836070474368013923F4604343EA80
:10CD4800413343607047436811B143F4006301E025
:10CD580023F4006343607047C06C80B27047014B96
:10CD68001868704708230140836811B143F4807341
:10CD780001E023F4807383607047836811B143F442
:10CD8800007301E023F4007383607047044B5A6812
:10CD980010B142F4005201E022F400525A60704788
:10CDA80000230140092970B50CB20CD904EB4404E6
:10CDB8001E3CC6680725A54026EA0505A34045EAA6
:10CDC8000304C4600AE0066904EB44040725A5408F
:10CDD80026EA050513FA04F42C430461836BC3F3B4
:10CDE8000154121B0232D2B202EB82021F24944079
:10CDF80023EA040391400B43836370BD836B0139BD
:10CE080023F4401343EA01538363704782B000233D
:10CE180001930190019BCB180193019B1A6002B00A
:10CE28007047836823F470230B43836070478368DB
:10CE380023F440130B4383607047836843F48003F3
:10CE4800836070478068C0F380507047436811B1B1
:10CE580043F4806301E023F48063436070474368D0
:10CE680011B143F4805301E023F4805343607047C9
:10CE780082B0002301930190019B28335B18019332
:10CE8800019B186880B202B070470123C9B213FA37
:10CE980001F143680AB1194301E023EA0101416045
:10CEA8007047036819420CBF002001207047C9432E
:10CEB800016070474368006810EA112007D001221A
:10CEC800C9B212FA01F119420CBF002001207047C3
:10CED8006FEA112101607047036823F001030360C2
:10CEE8000023036043608360C360036121234361BF
:10CEF8002C4B98421CD02C4B984220D02B4B98425C
:10CF080025D02B4B98422AD02A4B98422FD02A4B17
:10CF1800984233D0294B984237D0294B984204D1B4
:10CF28004FF03D5243F8AC2C7047264B984203D142
:10CF38003D2243F8082C7047234B984204D14FF404
:10CF4800746243F8202C7047204B984204D14FF468
:10CF5800741243F8382C70471D4B984204D14FF097
:10CF6800746243F8502C70471A4B984203D11A4AFE
:10CF780043F8642C7047194B984203D1184A43F878
:10CF88007C2C7047174B984203D1174A43F8942CCE
:10CF98007047164B984204BF4FF03D5243F8AC2CF3
:10CFA800704700BF106002402860024040600240A5
:10CFB800586002407060024088600240A0600240F1
:10CFC800B860024010640240286402404064024095
:10CFD80058640240706402403D00002088640240AA
:10CFE800400F0020A064024000003D20B8640240C9
:10CFF8000268134B10B51340CC680A6822434C6989
:10D0080022438C692243CC6922430C6A22434C6A2E
:10D0180022438C6A22434C6B22438C6B224313437A
:10D02800036042690C6BCB6A22F007022343134367
:10D0380043610B6943604B6883608B68C36010BDB4
:10D048003F801CF00023036043608360C36003617A
:10D0580043618361C361036243628362C3620363A2
:10D06800436383637047036811B143F0010301E030
:10D0780023F0010303607047036811B143F40043D0
:10D0880001E023F4004303607047036811B143F0E3
:10D09800200301E023F020030360704741607047DC
:10D0A800406880B27047036812B143F4002301E07E
:10D0B80023F40023036001617047036811B143F44E
:10D0C800802301E023F48023036070470AB10161E3
:10D0D8007047C16070470068C0F3C040704700687F
:10D0E80000F001007047406900F0380070470A4AB4
:10D0F8000A4B10B50A4CA04288BF13468A004CBFA1
:10D108005B681B6821F0F02121F0821119420CBFE5
:10D118000020012010BD00BF0064024000600240F2
:10D128000F64024010B5084B084A094CA04288BF5A
:10D13800134611F0005F21F0F02121F0821114BF95
:10D14800D960996010BD00BF0060024000640240D1
:10D158000F6402400B0607D5436912B143F0800300
:10D1680001E023F080034361802909D001F01E010A
:10D17800036812B119430160704723EA0101016095
:10D188007047124B124A10B5124CA0428CBF14467D
:10D198001C4621F0F02323F0C3132BB1026802F0E0
:10D1A8001E0202EAD12202E0426902F080028800EF
:10D1B8004CBF6368236821F0F02121F082101840E9
:10D1C80002D0101C18BF012010BD00BF0060024033
:10D1D800006402400F64024010B5084B084A094C2D
:10D1E800A04288BF134611F0005F21F0F02121F022
:10D1F800821114BFD960996010BD00BF0060024061
:10D20800006402400F640240044B00221A605A6016
:10D218009A60DA60024A5A61704700BF003C0140D8
:10D22800FFFF7F00837910B5002B29D01A4B0168C6
:10D238001C68CA4314401C605C6822405A6002792A
:10D2480002F1804202F59E3214682143116002689F
:10D258009C68D1430C409C60DC682140D9604179CE
:10D26800102906D1996811439960D9680A43DA6090
:10D2780010BD01F1804303F59E3319680A4308E0A5
:10D288000379016803F1804303F59E331A6822EAA3
:10D2980001021A6010BD00BF003C014000230C22AF
:10D2A80003600371427183717047024B1A6902432C
:10D2B8001A617047003C0140034B5B6918420CBF80
:10D2C80000200120704700BF003C0140014B58611D
:10D2D800704700BF003C0140054B1A685B6903407A
:10D2E80004D010420CBF0020012070471846704738
:10D2F800003C0140014B5861704700BF003C0140B1
:10D308004FF0204318B943F2DB021A6003E043F2FE
:10D31800D20243F820204FF02042411C6FF07043A6
:10D3280042F8213002F5827242F82030704770B519
:10D3380084684568C368C16A026825431D43036958
:10D348001D4343691D4383691D43C3691D43036A24
:10D358001D43436A1D43836A1D43036B0D431D43ED
:10D368004FF02043082C43F8225005D153F82240AF
:10D3780044F0400443F82240436B9E691D683543DE
:10D388005E6845EA06159E6845EA0625DE6845EAB0
:10D3980006451E695B6945EA0655541C45EA03655E
:10D3A8004FF02043B1F5804F43F8245010D1836BE0
:10D3B800986919680143586841EA0011986841EA78
:10D3C800002118695B6941EA005141EA036101E003
:10D3D8006FF07041014B43F8221070BD040100A0AA
:10D3E800022242604FF480524262416B4FF4005275
:10D3F80010B5826200230F22FF2403608360C3609C
:10D40800036143618361C3610362C36203630A60AA
:10D418004A608C60CA600A614A618B61816B0A60EC
:10D428004A608C60CA600A614A618B6110BD4FF026
:10D43800204321B153F8202042F0010203E053F8C1
:10D448002010024A0A4043F820207047FEFF0F00D0
:10D4580010280CBF064B074B4FF040024FF0180145
:10D4680019605A604FF0FC329A60DA60704700BF6A
:10D47800600000A0800000A030B5836844681C43A9
:10D48800C36844F008041C4303691C43436944EA25
:10D498004324836944EA4334C36999685A68090490
:10D4A80041EA02211A68DB68114341EA0361036A11
:10D4B8009A685D68120442EA05221D68DB682A43FF
:10D4C80042EA03620368102B0CBF034B034B1C603A
:10D4D8009960DA6030BD00BF600000A0800000A045
:10D4E80010230360C269002343608360C360036143
:10D4F80043618361FC23136053609360D360026AC5
:10D50800136053609360D360704741B110280CBF1B
:10D51800074B084B1A6842F004021A60704710283B
:10D528000CBF034A034A044B11680B401360704751
:10D53800600000A0800000A0FBFF0F0041B1102890
:10D548000CBF084B084B1A6842F040021A6070473B
:10D5580010280CBF034A044A044B11680B4013609F
:10D56800704700BF600000A0800000A0BFFF0F0050
:10D57800102802D1024B58697047024B586970470E
:10D58800600000A0800000A0054B18221A6000224D
:10D598005A604FF0FC329A60DA601A61704700BF37
:10D5A800A00000A00268436842F0100242EA432249
:10D5B800836842EA4332144B10B51A60C268916816
:10D5C8005468090441EA04211468D268214341EAF5
:10D5D80002629A60026991685468090441EA042168
:10D5E8001468D268214341EA0262DA6042699168AC
:10D5F8005068090441EA00211068D268014341EAF1
:10D6080002621A6110BD00BFA00000A0C26800231A
:10D61800036043608360FC23136053609360D360AE
:10D628000269136053609360D3604269136053606A
:10D638009360D3607047054B18B11A6842F0040232
:10D6480002E01968024A0A401A607047A00000A068
:10D65800FBFF0F0062B1102801D10E4B03E0B0F5BB
:10D66800807F03D10C4B5A68114311E00B4BFAE74A
:10D67800102804D1074B5A6822EA010108E0B0F5E6
:10D68800807F0CBF044B054B5A686FEA01011140BB
:10D6980059607047600000A0800000A0A00000A0B2
:10D6A800102801D1064B04E0B0F5807F0CBF054B74
:10D6B800054B5B680B420CBF00200120704700BF80
:10D6C800600000A0800000A0A00000A0102804D1E5
:10D6D800074B5A6822EA010108E0B0F5807F0CBFC9
:10D6E800044B054B5A686FEA0101114059607047B5
:10D6F800600000A0800000A0A00000A0102801D1B8
:10D70800084B04E0B0F5807F0CBF074B074B5B6804
:10D7180013EA010004D013EAD1010CBF0020012054
:10D72800704700BF600000A0800000A0A00000A01B
:10D73800102804D1084B5A6822EAD10109E0B0F553
:10D74800807F0CBF054B064B5A684FEAD10122EA8D
:10D7580001015960704700BF600000A0800000A070
:10D76800A00000A008B52C4B984205D10120014625
:10D7780000F048FC012048E0284B984205D10220DF
:10D78800012100F03FFC02203FE0254B984205D1E3
:10D798000420012100F036FC042036E0214B984299
:10D7A80005D10820012100F02DFC08202DE01E4B9A
:10D7B800984205D11020012100F024FC102024E01B
:10D7C8001A4B984205D12020012100F01BFC202093
:10D7D8001BE0174B984205D14020012100F012FCB4
:10D7E800402012E0134B984205D18020012100F01F
:10D7F80009FC802009E0104B98420BD14FF480704F
:10D80800012100F0FFFB4FF480700021BDE80840C3
:10D8180000F0F8BB08BD00BF000002400004024051
:10D8280000080240000C02400010024000140240B0
:10D8380000180240001C0240002002402DE9F04779
:10D848000023D1F800801A464FF0010C03270CFA88
:10D8580002F404EA0805A5422ED1066817FA03F473
:10D86800E443264006600E79D0F8009006FA03FAE1
:10D87800013E4AEA0909012EC0F8009014D88668CA
:10D8880091F8059026408660866809FA03F949EA06
:10D8980006068660466826EA050545608D7946686D
:10D8A8009540ADB235434560C5682C40C460CC791D
:10D8B800C5689C402C43C46001320233102AC6D18B
:10D8C800BDE8F0874FF6FF730360002303714371CF
:10D8D8008371C371704782B04FF480330193019B09
:10D8E8000B430193019BC361C161019BC361C36980
:10D8F8000193C369019302B07047036919420CBFD1
:10D90800002001207047006980B2704743691942BE
:10D918000CBF002001207047406980B27047018326
:10D928007047418370470AB101837047418370474C
:10D938004161704743694B404361704701F00703F9
:10D94800C908083130B59B0050F821500F249C407D
:10D9580025EA040440F8214050F8214012FA03F364
:10D968001C4340F8214030BD08B5134B984207D1FD
:10D978004FF40010012100F069FB4FF4001014E08F
:10D988000E4B984207D14FF48000012100F05EFB56
:10D998004FF4800009E00A4B98420BD14FF4000085
:10D9A800012100F053FB4FF400000021BDE80840BE
:10D9B80000F04CBB08BD00BF0054004000580040B8
:10D9C800005C00407FB50446868868460D4600F036
:10D9D8006DFA02992C482B6826F03F063604B1FBF5
:10D9E800F0F0360C80B20643A680228822F00102AD
:10D9F8001204120C2280254A93420AD85B00B1FB1C
:10DA0800F3F301309BB280B22084032B98BF042328
:10DA180021E0EE884BF6FF72964205D1032253436C
:10DA2800B1FBF3F39BB206E019225343B1FBF3F3C6
:10DA38009BB243F480431A054FF4967208BF43F033
:10DA4800010350434FF47A7290FBF2F0013080B238
:10DA580043F400432084A38323886989AA889BB25E
:10DA680043F001032380238823F4816323F0020316
:10DA78001B040A431B0C13439BB223802A89AB89DE
:10DA880013439BB223817FBD40420F00A086010053
:10DA980041F288330360002383804BF6FF720381D1
:10DAA80043814FF48043C28083817047038819B152
:10DAB8009BB243F0010303E023F001031B041B0C9A
:10DAC80003807047038819B19BB243F4807303E065
:10DAD80023F480731B041B0C03807047038819B15F
:10DAE8009BB243F4007303E023F400731B041B0C84
:10DAF8000380704712B141F0010101E001F0FE011D
:10DB080001827047038819B19BB243F4806303E034
:10DB180023F480631B041B0C0380704783899BB22A
:10DB280001F0FE0123F0FE030B43838170478389D4
:10DB380019B19BB243F0010303E023F001031B0476
:10DB48001B0C83817047038819B19BB243F04003D3
:10DB580003E023F040031B041B0C03807047038879
:10DB680029B16FEA43436FEA53439BB201E05B0478
:10DB78005B0C03807047038819B99BB243F080039C
:10DB880003E023F080031B041B0C03807047B1F5EE
:10DB9800804F838B04D023F480431B041B0C02E0CA
:10DBA8009BB243F4804383837047B1F5006F0388C9
:10DBB80003D19BB243F4006303E023F400631B0426
:10DBC8001B0C03807047B1F5005F038803D19BB23B
:10DBD80043F4005303E023F400531B041B0C03809D
:10DBE8007047038819B19BB243F0100303E023F098
:10DBF80010031B041B0C0380704701827047008AC6
:10DC0800C0B27047038819B19BB243F4805303E054
:10DC180023F480531B041B0C03807047B1F5006F7D
:10DC2800038803D19BB243F4006303E023F4006349
:10DC38001B041B0C03807047038819B19BB243F087
:10DC4800200303E023F020031B041B0C0380704710
:10DC5800008BC0F307207047838819B19BB243F447
:10DC6800006303E023F400631B041B0C83807047EC
:10DC7800838819B19BB243F4805303E023F48053A3
:10DC88001B041B0C8380704782B000230193019012
:10DC9800019BCB180193019B188880B202B0704792
:10DCA80083889BB20AB1194301E023EA010181800C
:10DCB8007047838A008B9BB243EA0040084020F0FB
:10DCC8007F40431A584240EB03007047838A008B19
:10DCD8009BB243EA004020F07F40704782B00023A7
:10DCE800009301930B0F01900093009B21F07F415B
:10DCF80013B1019B143302E0019B090C1833019303
:10DD0800019B1B6819420CBF0020012002B070471C
:10DD1800C94389B2818270478388808A80B208406B
:10DD28009BB206D001F0E06113EA11410CBF00205C
:10DD380001207047C94389B2818270470A4B1A682B
:10DD480042F001021A6000229A60196821F0847179
:10DD580021F48031196005495960196821F480213E
:10DD68001960DA60704700BF0038024010300024A4
:10DD7800024B00221A701870704700BF0238024028
:10DD8800034B1A6822F0F80242EAC0021A60704790
:10DD980000380240014B1860704700BF000047423E
:10DDA800064B002201281A701A7002D0042804D1E8
:10DDB80001E01870704705221A70704770380240E9
:10DDC800014B1860704700BF800E4742014341EA8B
:10DDD800821200995B08013B42EA016141EA034172
:10DDE800014B5960704700BF00380240014B186072
:10DDF800704700BF600047428001034B40EA017151
:10DE0800C3F88410704700BF00380240014B186007
:10DE1800704700BF68004742014B1860704700BF59
:10DE28004C004742034B9A6822F0EC6202430A43D3
:10DE38009A60704700380240034B9A6822F0784293
:10DE480002430A439A60704700380240034B9A68BD
:10DE580022F0030202439A60704700BF0038024074
:10DE6800024B986800F00C00704700BF0038024071
:10DE7800034B9A6822F0F00202439A60704700BF91
:10DE880000380240034B9A6822F4E05202439A6039
:10DE9800704700BF00380240034B9A6822F4604282
:10DEA80042EAC0029A607047003802401E4B9A68E6
:10DEB80002F00C02042A10B503D0082A03D01B4B29
:10DEC80018E01B4B16E059685A6811F4800F59681E
:10DED80014BF174B154B02F03F02B3FBF2F3124A83
:10DEE8005268C2F30142C1F3881101324B43520018
:10DEF800B3FBF2F30C4903608B680E4A0468C3F362
:10DF08000313D35C34FA03F343608C68C4F38224AC
:10DF1800145D33FA04F484608968C1F34231525CB9
:10DF2800D340C36010BD00BF003802400024F40095
:10DF380000127A002804002000F44073B3F5407FF3
:10DF4800084B08D1996820F0704221F4F81122F4A6
:10DF580040720A439A601A6F000542EA1050186727
:10DF6800704700BF00380240014B1860704700BF7F
:10DF78003C0E4742014B1860704700BF400E4742B5
:10DF8800014B1860704700BF5C014742044B1A6B95
:10DF980009B1104301E022EA00001863704700BF8E
:10DFA80000380240044B5A6B09B1104301E022EAE1
:10DFB80000005863704700BF00380240044B9A6B5A
:10DFC80009B1104301E022EA00009863704700BFDE
:10DFD80000380240044B1A6C09B1104301E022EAF0
:10DFE80000001864704700BF00380240044B5A6CA8
:10DFF80009B1104301E022EA00005864704700BFED
:10E0080000380240044B1A6909B1104301E022EAC2
:10E0180000001861704700BF00380240044B5A697D
:10E0280009B1104301E022EA00005861704700BFBF
:10E0380000380240044B9A6909B1104301E022EA12
:10E0480000009861704700BF00380240044B1A6A0C
:10E0580009B1104301E022EA00001862704700BFCE
:10E0680000380240044B5A6A09B1104301E022EA21
:10E0780000005862704700BF00380240044B1A6D18
:10E0880009B1104301E022EA00001865704700BF9B
:10E0980000380240044B5A6D09B1104301E022EAEE
:10E0A80000005865704700BF00380240044B9A6D65
:10E0B80009B1104301E022EA00009865704700BFEB
:10E0C80000380240044B1A6E09B1104301E022EAFD
:10E0D80000001866704700BF00380240044B5A6EB3
:10E0E80009B1104301E022EA00005866704700BFFA
:10E0F80000380240044B1A7809B1104301E022EAC3
:10E1080000001870704700BF0D3802404309012B0A
:10E11800074A01D1136803E0022B0CBF136F536F3A
:10E1280000F01F0033FA00F000F00100704700BF54
:10E138000038024007B5002301933120FFF7E6FFBE
:10E14800019B01330193019BB3F5A06F01D0002817
:10E15800F3D03120FFF7DAFF003018BF01200EBDE1
:10E16800024B5A6F42F080725A677047003802407B
:10E17800034BDB6818420CBF00200120704700BF2A
:10E1880000380240014B1870704700BF0E3802403B
:10E1980008B5154B98420BD101214FF48050FFF779
:10E1A80061FF4FF480500021BDE80840FFF75ABFD7
:10E1B8000E4B984207D14FF480400121FFF746FFEC
:10E1C8004FF4804009E00A4B98420BD14FF40040CD
:10E1D8000121FFF73BFF4FF400400021BDE8084054
:10E1E800FFF734BF08BD00BF0030014000380040D1
:10E1F800003C00400B88028810B54C8823438C886B
:10E208002343CC8823430C8923434C8923438C899B
:10E218002343CC8902F44152234313439BB2038026
:10E22800838B23F400631B041B0C83830B8A0382F8
:10E2380010BD838B23F47B6323F00F031B041B0C9B
:10E248008383022303848B68F0B5858B022BADB2E0
:10E2580038D0294A8E889468002E14BF02260126D9
:10E26800240203D5946824F400049460D2F884400E
:10E27800D2F884705268DFF884C002F03F02BCFB19
:10E28800F2F2C4F388145443C7F30272B4FBF2F4F5
:10E29800CA88B2F5007F4FF00A0201D1240A02E0D1
:10E2A8007601B4FBF6F46243B2FBF3F305330A22BA
:10E2B8009BB2B3FBF2F303F001021202C3F34F0364
:10E2C80092B200E000229C1EA4B2FE2C28BF0022BD
:10E2D800CC8828BF0223134323439BB203840B88B3
:10E2E8004A882B4343F4006313438A8813438A897B
:10E2F80013439BB28383F0BD0038024000127A00BA
:10E308000023038043808380C3800381438183810A
:10E31800C3810723038270470023022203804380BE
:10E328008380C380826083817047038819B19BB260
:10E3380043F0400303E023F040031B041B0C03805D
:10E348007047838B19B19BB243F4806303E023F4D5
:10E3580080631B041B0C83837047038823F40063CA
:10E368001B041B0C038003889BB20B43038070477C
:10E37800B1F5804F038803D19BB243F4804303E097
:10E3880023F480431B041B0C038070474FF6FF6384
:10E398009942038803D09BB243F4807303E023F4CB
:10E3A80080731B041B0C03807047838819B19BB2D0
:10E3B80043F0040303E023F004031B041B0C8380D5
:10E3C8007047838819B19BB243F0100303E023F030
:10E3D80010031B041B0C83807047838B23F47B631F
:10E3E80023F00F031B041B0C8383022303840B8875
:10E3F800828BB3F5007F10B592B205D0002B0CBF0D
:10E408004FF48073002301E04FF480734C8822435B
:10E418008C88898942F4006222430A4392B21343EA
:10E42800838310BD808980B27047818170470388DB
:10E4380019B19BB243F4005303E023F400531B04C7
:10E448001B0C0380704703889BB243F480530380FE
:10E458007047012902D0008B80B27047808A80B251
:10E468007047008A80B2704783889BB20AB119430B
:10E4780001E023EA010181807047090901238B40EB
:10E488009BB21AB1828892B2134303E0828892B297
:10E4980022EA030383807047038919420CBF0020D6
:10E4A80001207047C94389B20181704710B584883B
:10E4B8000089012301F00F0280B213FA02F2104022
:10E4C800A4B205D009098B401C420CBF00200120D2
:10E4D80010BD01F00F0101238B40DB439BB2038188
:10E4E800704700BF08B501214FF48040FFF7BAFD1F
:10E4F8004FF480400021BDE80840FFF7B3BD014B51
:10E50800186070470038014001F0030289080A4B7F
:10E51800023130B5920053F821500F24944025EA77
:10E52800040443F8214053F8214010FA02F214433E
:10E5380043F8214030BD00BF00380140014B18604E
:10E54800704700BFDC002742014B1860704700BFCE
:10E5580000042742024B186AC0F30020704700BF2E
:10E568000038014030B5048C24F001042404240C44
:10E578000484058B048CADB2A4B225F0F3051543D1
:10E5880024F00A0445EA031544F00104ADB20C4333
:10E598000583048430BD30B5048C24F010042404B1
:10E5A800240C0484048B058C24F44074ADB2240537
:10E5B800240D25F0A00544EA022445F0100544EA9C
:10E5C800033445EA0115A4B2ADB20483058430BD15
:10E5D80008B5474B984205D101200146FFF742FD97
:10E5E80001203DE0B0F1804F05D101200146FFF741
:10E5F8002DFD012076E03F4B984205D102200121F4
:10E60800FFF724FD02206DE03B4B984205D1042022
:10E618000121FFF71BFD042064E0384B984205D127
:10E6280008200121FFF712FD08205BE0344B9842D7
:10E6380005D110200121FFF709FD102052E0314BD0
:10E64800984205D120200121FFF700FD202049E054
:10E658002D4B984209D102200121FFF703FD02202A
:10E668000021BDE80840FFF7FDBC284B984207D1C0
:10E678004FF480300121FFF7F5FC4FF48030EFE7CD
:10E68800234B984207D14FF400300121FFF7EAFCF1
:10E698004FF40030E4E71F4B984207D14FF4802035
:10E6A8000121FFF7DFFC4FF48020D9E71A4B98428D
:10E6B80005D140200121FFF7C9FC402012E0174B8B
:10E6C800984205D180200121FFF7C0FC802009E095
:10E6D800134B98420BD14FF480700121FFF7B6FC21
:10E6E8004FF480700021BDE80840FFF7AFBC08BDBB
:10E6F800000001400004004000080040000C0040F9
:10E708000010004000140040000401400040014097
:10E71800004401400048014000180040001C00402F
:10E72800002000401C4A038890429BB212D002F598
:10E73800806290420ED0B0F1804F0BD0A2F58032AB
:10E74800904207D002F58062904203D002F58062C1
:10E75800904203D14A8823F0700313430F4A904232
:10E7680008D002F58062904204D023F440730A89ED
:10E778009BB2134303804B68C3620B880385064B27
:10E78800984203D003F58063984201D18B7A0386BF
:10E7980001238382704700BF000001400010004041
:10E7A8004FF0FF334360002303800381438083726B
:10E7B8007047018582827047038823F070031B0429
:10E7C8001B0C0B430380704741627047C16270475E
:10E7D800406A7047008D80B27047038819B19BB2B8
:10E7E80043F0020303E023F002031B041B0C038025
:10E7F8007047038819B19BB243F0040303E023F088
:10E8080004031B041B0C03807047038819B19BB2D7
:10E8180043F0800303E023F080031B041B0C0380F8
:10E828007047038823F008031B041B0C038003882C
:10E838009BB20B4303807047038823F440731B0487
:10E848001B0C038003889BB20B430380704703882B
:10E8580019B19BB243F0010303E023F001031B0449
:10E868001B0C03807047038C23F001031B041B0C53
:10E87800038470B5038C8488028B0D884E8822F03F
:10E8880073021204120C2A438D8923F002031B041D
:10E8980035431B0CADB22B430E4DA842A4B203D096
:10E8A80005F58065A8420ED1CD894E8A23F008036C
:10E8B8002B438D8823F004032B430D8A354324F41E
:10E8C8004074ADB22C43848002838A684263038417
:10E8D80070BD00BF00000140038C23F010031B042F
:10E8E8001B0C0384038C828830B5048B0D8824F4B8
:10E8F800E6442404240C23F0200344EA05241B04E2
:10E908008D891B0C43EA05134D8843EA0513134D03
:10E91800A84292B2A4B29BB203D005F58065A84282
:10E9280015D1CD8923F080039BB243EA05134FF636
:10E93800BF751D408B8845EA03130D8A22F4406297
:10E9480042EA85024D8A42EA85029BB292B28280EF
:10E958008A6804838263038430BD00BF00000140DD
:10E96800038C23F480731B041B0C0384038C8288A0
:10E9780030B5848B0D8824F073042404240C23F40C
:10E9880000731B042C438D891B0C43EA05234D8817
:10E9980043EA0523124DA84292B29BB203D005F573
:10E9A8008065A84215D1CD8923F400639BB243EA60
:10E9B80005234FF6FF351D408B8845EA03230D8A52
:10E9C80022F4405242EA05124D8A42EA05129BB2ED
:10E9D80092B282808A688483C263038430BD00BF98
:10E9E80000000140038C23F480531B041B0C038498
:10E9F800038C30B58488828B0D8822F4E642120499
:10EA0800120C23F4005342EA05221B048D891B0CC7
:10EA180043EA05334D8843EA05330B4DA842A4B2B7
:10EA280092B29BB203D005F58065A84205D10D8A44
:10EA380024F4804444EA8514A4B2848082838A68DA
:10EA48000264038430BD00BF00000140002303803E
:10EA58004380838083608381C381038243827047BC
:10EA680030B5058C0124ADB28C4025EA040400F1D0
:10EA78001803048409B1082907D149084FF68F7093
:10EA8800CC582040C850C8580AE00439C1F34E0198
:10EA980048F6FF70CC582040C8501202C85892B2AD
:10EAA8000243CA5030BD4163704781637047C163F8
:10EAB800704701647047038B23F070031B041B0C21
:10EAC8000B4303837047038B23F4E0431B041B0CA5
:10EAD80043EA01239BB203837047838B23F07003BF
:10EAE8001B041B0C0B4383837047838B23F4E04385
:10EAF8001B041B0C43EA01239BB283837047038BDF
:10EB080023F008031B041B0C0B4303837047038B80
:10EB180023F400631B041B0C43EA01239BB2038309
:10EB28007047838B23F008031B041B0C0B43838360
:10EB38007047838B23F400631B041B0C43EA0123F7
:10EB48009BB283837047038B23F004031B041B0CC5
:10EB58000B4303837047038B23F480631B041B0C54
:10EB680043EA01239BB203837047838B23F004039A
:10EB78001B041B0C0B4383837047838B23F4806334
:10EB88001B041B0C43EA01239BB283837047038B4E
:10EB980023F080031B041B0C0B4303837047038B78
:10EBA80009025B0441EA53439BB203837047838B9A
:10EBB80023F080031B041B0C0B4383837047838B58
:10EBC80009025B0441EA53439BB283837047038C79
:10EBD80023F002031B041B0C0B4303847047038CB4
:10EBE80023F008031B041B0C0B4303847047038C9E
:10EBF80023F020031B041B0C43EA01139BB203847C
:10EC08007047038C23F080031B041B0C43EA011399
:10EC18009BB203847047038C23F400731B041B0C02
:10EC280043EA01239BB203847047038C23F40063F7
:10EC38001B041B0C43EA01239BB203847047038C1B
:10EC480023F400531B041B0C43EA01339BB20384D7
:10EC5800704710B5048C01238B40A4B224EA030347
:10EC68000384038C12FA01F10B439BB2038410BD99
:10EC780010B5048C04238B40A4B224EA0303038454
:10EC8800038C12FA01F10B439BB2038410BD0023DD
:10EC98000122038043808280C38003817047406BD8
:10ECA8007047806B7047C06B7047006C7047038B70
:10ECB80023F00C031B041B0C0383038B9BB20B4335
:10ECC80003837047038B23F440631B041B0C0383EB
:10ECD800038B9BB243EA01239BB203837047F8B5C9
:10ECE8000C464988A288B4F800E023890546002923
:10ECF8000CBF02270027012A14BF01260226BEF1F5
:10ED0800000F10D1FFF72EFC2846E188FFF7CFFF50
:10ED18002846394632462389FFF73DFCE1882846D4
:10ED2800BDE8F840CEE7FFF736FC2846E188FFF754
:10ED3800C9FF2846394632462389FFF713FCE18884
:10ED48002846BDE8F840B2E7838B23F00C031B0488
:10ED58001B0C8383838B9BB20B4383837047838B0A
:10ED680023F440631B041B0C8383838B9BB243EA0D
:10ED780001239BB283837047F8B50D460B88AA8898
:10ED8800498804463BB92B89FFF7ECFBE988204604
:10ED9800BDE8F8408BE7042B07D12B89FFF7FBFB75
:10EDA800E9882046BDE8F8408CE7082BB5F808C08C
:10EDB800078C1DD127F480773F043F0C0784868B8E
:10EDC800038CB6B29BB226F0F30623F4206346EA1E
:10EDD8000C1C43EA01211FFA8CFC89B24CEA02029E
:10EDE80041F4807182830184E988BDE8F840ABE78B
:10EDF80027F480573F043F0C0784868B038C26F446
:10EE0800407623F4005336055B04360D5B0C46EA66
:10EE1800022243EA013342EA0C329BB2E98892B2F9
:10EE280043F4805382830384BDE8F84097E74A8817
:10EE38000B8813438A881343CA8813430A891343E8
:10EE48004A8913438A8913439BB2A0F84430704718
:10EE58000023038043808380C380038143818381AF
:10EE68007047B0F8443029B16FEA43436FEA53431F
:10EE78009BB201E05B045B0CA0F8443070478388C8
:10EE880019B19BB243F0040303E023F004031B040D
:10EE98001B0C83807047838819B19BB243F0010330
:10EEA80003E023F001031B041B0C83807047838954
:10EEB8009BB20AB1194301E023EA0101818170473D
:10EEC80081827047038A19420CBF002001207047D5
:10EED800C94389B201827047038A828911EA030013
:10EEE80092B203D011420CBF002001207047C943E1
:10EEF80089B2018270470A43A0F848207047838985
:10EF08009BB20AB1194301E023EA010181817047EC
:10EF1800838819B19BB243F0080303E023F0080388
:10EF28001B041B0C83807047038923F007031B0411
:10EF38001B0C03817047038923F070031B041B0C0F
:10EF48000B43038103899BB243F007030381704796
:10EF580038B50D4611460122602D044602D1FFF74F
:10EF68001AFB01E0FFF7FEFA238923F070031B0464
:10EF78001B0C1D43258123899BB243F00703238182
:10EF880038BD038923F070031B041B0C0B4303815A
:10EF98007047838823F070031B041B0C83808388CD
:10EFA8009BB20B4383807047038923F007031B043C
:10EFB8001B0C038103899BB20B43038170470389B0
:10EFC80023F080031B041B0C038103899BB20B43B2
:10EFD8000381704710B50489E4B20C43144344EA32
:10EFE8000324A4B2048110BD10B50446FFF7F2FF54
:10EFF80023899BB243F48043238110BD10B5044696
:10F00800FFF7E8FF238923F077031B041B0C43F069
:10F018007703238110BD70B50489068B058C26F40F
:10F028004076ADB226F0030624F00704360425F036
:10F0380022052404360C1543240C46F4807645EA50
:10F048000315214346F00106ADB20181068305840C
:10F0580070BD838819B19BB243F0800303E023F0AD
:10F0680080031B041B0C83807047A0F85010704766
:10F0780008B5234B984205D110200121FEF7F2FF75
:10F08800102037E01F4B984207D14FF40030012180
:10F09800FEF7DCFF4FF4003009E01B4B98420BD120
:10F0A8004FF480200121FEF7D1FF4FF4802000218A
:10F0B800BDE80840FEF7CABF144B984207D14FF489
:10F0C80000200121FEF7C2FF4FF40020EFE7104BAC
:10F0D800984207D14FF480100121FEF7B7FF4FF493
:10F0E8008010E4E70B4B984209D120200121FEF75C
:10F0F800B9FF20200021BDE80840FEF7B3BF08BDD6
:10F10800001001400044004000480040004C00400E
:10F118000050004000140140038ACA889BB223F4BF
:10F12800405330B513430D46038283890989AA8861
:10F1380023F4B0530A43698923F00C031B040A43E0
:10F148001B0C92B213438381838AAA899BB223F44E
:10F158004073134385B0838204466846FEF7A6FED3
:10F168001A4B9C4203D003F580639C4201D1039B58
:10F1780000E0029BA28912B2002A4FF019012A6806
:10F1880001FB03F101DA520000E092006423B1FBB5
:10F19800F2F1B1FBF3F21201100903FB1011A0897F
:10F1A80000B2002806DAC9003231B1FBF3F303F0EC
:10F1B800070305E009013231B1FBF3F303F00F0354
:10F1C8001A4392B2228105B030BD00BF0010014041
:10F1D8004FF4165303600C2200238380C3800381FD
:10F1E8004281838170470B88028A10B54C8823437B
:10F1F8008C88C988234392B20B4322F470629BB275
:10F208001343038210BD0023038043808380C3809F
:10F218007047838919B19BB243F4005303E023F488
:10F2280000531B041B0C83817047038B03F47F433B
:10F238000383038B9BB20B4303837047838929B1F4
:10F248006FEA43436FEA53439BB201E05B045B0CF4
:10F2580083817047838A19B19BB243F4006303E04A
:10F2680023F400631B041B0C83827047C905C90D76
:10F27800818070478088C005C00D7047038A23F0DD
:10F288000F031B041B0C0382038A9BB20B430382EC
:10F298007047838919B19BB243F0020303E023F05E
:10F2A80002031B041B0C83817047838923F40063CA
:10F2B8001B041B0C838183899BB20B43838170479A
:10F2C800038A23F020031B041B0C0382038A9BB2CE
:10F2D8000B4303827047038A19B19BB243F48043FE
:10F2E80003E023F480431B041B0C038270478389CB
:10F2F8009BB243F0010383817047838A19B19BB2A3
:10F3080043F0080303E023F008031B041B0C83826B
:10F318007047038BDBB20383038B9BB243EA012361
:10F3280003837047838A19B19BB243F0200303E03B
:10F3380023F020031B041B0C83827047838A19B1B6
:10F348009BB243F0100303E023F010031B041B0CD3
:10F3580083827047838A23F004031B041B0C838277
:10F36800838A9BB20B4383827047838A19B19BB20D
:10F3780043F0020303E023F002031B041B0C838207
:10F388007047838A9BB20AB1194301E023EA01015D
:10F3980081827047C1F3421310B501F01F010124A7
:10F3A80014FA01F1A34201D10C3004E0022B01D17F
:10F3B800103000E0143003680AB1194301E023EA71
:10F3C8000101016010BD038819420CBF0020012013
:10F3D8007047C94389B201807047012210B501F016
:10F3E8001F03C1F342149A40012C01D1838903E021
:10F3F800022C0CBF038A838A9BB21340028892B204
:10F4080043B1090A012313FA01F111420CBF00208C
:10F41800012010BD184610BD090A01238B40DB43AB
:10F428009BB20380704700BF81F0004102E000BF3B
:10F4380083F0004330B54FEA41044FEA430594EAAC
:10F44800050F08BF90EA020F1FBF54EA000C55EAE7
:10F45800020C7FEA645C7FEA655C00F0E2804FEAB8
:10F468005454D4EB5555B8BF6D420CDD2C4480EA9A
:10F47800020281EA030382EA000083EA010180EACA
:10F48800020281EA0303362D88BF30BD11F0004F18
:10F498004FEA01314FF4801C4CEA113102D040424E
:10F4A80061EB410113F0004F4FEA03334CEA133389
:10F4B80002D0524263EB430394EA050F00F0A780A1
:10F4C800A4F10104D5F1200E0DDB02FA0EFC22FA9C
:10F4D80005F2801841F1000103FA0EF2801843FA90
:10F4E80005F359410EE0A5F120050EF1200E012A81
:10F4F80003FA0EFC28BF4CF0020C43FA05F3C018BF
:10F5080051EBE37101F0004507D54FF0000EDCF137
:10F51800000C7EEB00006EEB0101B1F5801F1BD3E0
:10F52800B1F5001F0CD349085FEA30004FEA3C0CE4
:10F5380004F101044FEA445212F5800F80F09A80DA
:10F54800BCF1004F08BF5FEA500C50F1000041EBDE
:10F55800045141EA050130BD5FEA4C0C404141EBE2
:10F56800010111F4801FA4F10104E9D191F0000F09
:10F5780004BF01460020B1FA81F308BF2033A3F18C
:10F588000B03B3F120020CDA0C3208DD02F1140C83
:10F59800C2F10C0201FA0CF021FA02F10CE002F1BE
:10F5A8001402D8BFC2F1200C01FA02F120FA0CFCB7
:10F5B800DCBF41EA0C019040E41AA2BF01EB045100
:10F5C800294330BD6FEA04041F3C1CDA0C340EDCFE
:10F5D80004F11404C4F1200220FA04F001FA02F341
:10F5E80040EA030021FA04F345EA030130BDC4F1FF
:10F5F8000C04C4F1200220FA02F001FA04F340EAF4
:10F608000300294630BD21FA04F0294630BD94F0A4
:10F61800000F83F4801306BF81F480110134013D8B
:10F628004EE77FEA645C18BF7FEA655C29D094EAFC
:10F63800050F08BF90EA020F05D054EA000C04BF7A
:10F648001946104630BD91EA030F1EBF0021002065
:10F6580030BD5FEA545C05D14000494128BF41F004
:10F66800004130BD14F580043CBF01F5801130BD68
:10F6780001F0004545F0FE4141F470014FF00000F3
:10F6880030BD7FEA645C1ABF194610467FEA655CA4
:10F698001CBF0B46024650EA013406BF52EA033546
:10F6A80091EA030F41F4002130BD00BF90F0000F34
:10F6B80004BF0021704730B54FF4806404F1320470
:10F6C8004FF000054FF0000150E700BF90F0000F29
:10F6D80004BF0021704730B54FF4806404F1320450
:10F6E80010F0004548BF40424FF000013EE700BF20
:10F6F80042004FEAE2014FEA31014FEA02701FBFB0
:10F7080012F07F4393F07F4F81F06051704792F081
:10F71800000F14BF93F07F4F704730B54FF46074FB
:10F7280001F0004521F0004120E700BF50EA010246
:10F7380008BF704730B54FF000050AE050EA0102F3
:10F7480008BF704730B511F0004502D5404261EB63
:10F7580041014FF4806404F132045FEA915C3FF4A4
:10F76800DCAE4FF003025FEADC0C18BF03325FEA3D
:10F77800DC0C18BF033202EBDC02C2F1200300FAF2
:10F7880003FC20FA02F001FA03FE40EA0E0021FA17
:10F7980002F11444C1E600BF70B54FF0FF0C4CF401
:10F7A800E06C1CEA11541DBF1CEA135594EA0C0FB7
:10F7B80095EA0C0F00F0DEF82C4481EA030621EAF2
:10F7C8004C5123EA4C5350EA013518BF52EA03352D
:10F7D80041F4801143F4801338D0A0FB02CE4FF0DF
:10F7E8000005E1FB02E506F00042E0FB03E54FF00F
:10F7F8000006E1FB03569CF0000F18BF4EF0010E07
:10F80800A4F1FF04B6F5007F64F5407404D25FEA02
:10F818004E0E6D4146EB060642EAC62141EA5551B5
:10F828004FEAC52040EA5E504FEACE2EB4F1FD0CF7
:10F8380088BFBCF5E06F1ED8BEF1004F08BF5FEA75
:10F84800500E50F1000041EB045170BD06F0004627
:10F8580046EA010140EA020081EA0301B4EB5C04D4
:10F86800C2BFD4EB0C0541EA045170BD41F48011CC
:10F878004FF0000E013C00F3AB8014F1360FDEBFF1
:10F88800002001F0004170BDC4F10004203C35DACD
:10F898000C341BDC04F11404C4F1200500FA05F350
:10F8A80020FA04F001FA05F240EA020001F00042F1
:10F8B80021F0004110EBD37021FA04F642EB060167
:10F8C8005EEA430E08BF20EAD37070BDC4F10C0491
:10F8D800C4F1200500FA04F320FA05F001FA04F255
:10F8E80040EA020001F0004110EBD37041F1000141
:10F8F8005EEA430E08BF20EAD37070BDC4F120054C
:10F9080000FA05F24EEA020E20FA04F301FA05F2B3
:10F9180043EA020321FA04F001F0004121FA04F25B
:10F9280020EA020000EBD3705EEA430E08BF20EA2B
:10F93800D37070BD94F0000F0FD101F00046400065
:10F9480041EB010111F4801F08BF013CF7D041EAE7
:10F95800060195F0000F18BF704703F000465200EB
:10F9680043EB030313F4801F08BF013DF7D043EABC
:10F978000603704794EA0C0F0CEA135518BF95EA72
:10F988000C0F0CD050EA410618BF52EA4306D1D1F9
:10F9980081EA030101F000414FF0000070BD50EA18
:10F9A800410606BF1046194652EA430619D094EAA2
:10F9B8000C0F02D150EA013613D195EA0C0F05D18C
:10F9C80052EA03361CBF104619460AD181EA0301E0
:10F9D80001F0004141F0FE4141F470014FF0000098
:10F9E80070BD41F0FE4141F4780170BD70B54FF033
:10F9F800FF0C4CF4E06C1CEA11541DBF1CEA1355B3
:10FA080094EA0C0F95EA0C0F00F0A7F8A4EB050494
:10FA180081EA030E52EA03354FEA013100F088808B
:10FA28004FEA03334FF0805545EA131343EA126354
:10FA38004FEA022245EA111545EA10654FEA002609
:10FA48000EF000419D4208BF964244F1FD0404F5C2
:10FA5800407402D25B084FEA3202B61A65EB03051E
:10FA68005B084FEA32024FF480104FF4002CB6EBDB
:10FA7800020E75EB030E22BFB61A754640EA0C005B
:10FA88005B084FEA3202B6EB020E75EB030E22BF9B
:10FA9800B61A754640EA5C005B084FEA3202B6EBDC
:10FAA800020E75EB030E22BFB61A754640EA9C009B
:10FAB8005B084FEA3202B6EB020E75EB030E22BF6B
:10FAC800B61A754640EADC0055EA060E18D04FEA29
:10FAD800051545EA16754FEA06164FEAC30343EAC9
:10FAE80052734FEAC2025FEA1C1CC0D111F4801F96
:10FAF8000BD141EA00014FF000004FF0004CB6E78F
:10FB080011F4801F04BF01430020B4F1FD0C88BF2D
:10FB1800BCF5E06F3FF6AFAEB5EB030C04BFB6EB38
:10FB2800020C5FEA500C50F1000041EB045170BD2B
:10FB38000EF0004E4EEA113114EB5C04C2BFD4EB58
:10FB48000C0541EA045170BD41F480114FF0000EDC
:10FB5800013C90E645EA060E8DE60CEA135594EA58
:10FB68000C0F08BF95EA0C0F3FF43BAF94EA0C0F5B
:10FB78000AD150EA01347FF434AF95EA0C0F7FF4D0
:10FB880025AF104619462CE795EA0C0F06D152EA24
:10FB980003353FF4FDAE1046194622E750EA410608
:10FBA80018BF52EA43067FF4C5AE50EA41047FF419
:10FBB8000DAF52EA43057FF4EBAE12E74FF0FF3C7E
:10FBC80006E000BF4FF0010C02E000BF4FF0010C4F
:10FBD8004DF804CD4FEA410C7FEA6C5C4FEA430CC8
:10FBE80018BF7FEA6C5C1BD001B050EA410C0CBF17
:10FBF80052EA430C91EA030F02BF90EA020F002079
:10FC0800704710F1000F91EA030F58BF994208BFDF
:10FC180090422CBFD8176FEAE37040F0010070479C
:10FC28004FEA410C7FEA6C5C02D150EA013C07D1F3
:10FC38004FEA430C7FEA6C5CD6D152EA033CD3D03E
:10FC48005DF8040B704700BF8446104662468C4638
:10FC58001946634600E000BF01B5FFF7B7FF00286B
:10FC680048BF10F1000F01BD4DF808EDFFF7F4FF94
:10FC78000CBF012000205DF808FB00BF4DF808ED1F
:10FC8800FFF7EAFF34BF012000205DF808FB00BF42
:10FC98004DF808EDFFF7E0FF94BF012000205DF864
:10FCA80008FB00BF4DF808EDFFF7CEFF94BF012019
:10FCB80000205DF808FB00BF4DF808EDFFF7C4FF12
:10FCC80034BF012000205DF808FB00BF4FEA410265
:10FCD80012F5001215D211D56FF47873B3EB625296
:10FCE80012D94FEAC12343F0004343EA505311F0BD
:10FCF800004F23FA02F018BF404270474FF000004F
:10FD0800704750EA013005D111F0004008BF6FF08C
:10FD1800004070474FF00000704700BF4A0011D202
:10FD280012F5001211D20DD56FF47873B3EB62524D
:10FD38000ED44FEAC12343F0004343EA505323FA59
:10FD480002F070474FF00000704750EA013002D1CE
:10FD58004FF0FF3070474FF0000070474FEA410204
:10FD6800B2F1E04324BFB3F5001CDCF1FE5C0DD911
:10FD780001F0004C4FEAC0024CEA5070B2F1004F5B
:10FD880040EB830008BF20F00100704711F0804F5E
:10FD980021D113F13872BCBF01F00040704741F423
:10FDA80080114FEA5252C2F11802C2F1200C10FA27
:10FDB8000CF320FA02F018BF40F001004FEAC1230B
:10FDC8004FEAD32303FA0CFC40EA0C0023FA02F3AF
:10FDD8004FEA4303CCE77FEA625307D150EA013385
:10FDE8001EBF4FF0FE4040F44000704701F0004055
:10FDF80040F0FE4040F40000704700BF4BB942B9E4
:10FE0800002908BF002802D04FF0FF31084600F053
:10FE180037B882B0EC462DE9005000F01BF8DDF849
:10FE280004E002B00CBC7047F8B5144606460F460D
:10FE38001D4600F027F804FB01F300FB0535A4FB81
:10FE48000023EB18069CB21A67EB0303C4E90023EE
:10FE5800F8BD00BFF8B5144606460F461D4600F02B
:10FE680075F900FB05F5A0FB042304FB0155EB180D
:10FE7800069CB21A67EB0303C4E90023F8BD00BF70
:10FE8800704700BF00292DE9F0071D46C0F29E808B
:10FE98000024002DC0F2958007460D4616469C4664
:10FEA800002B3ED18A4254D9B2FA82F343B1C3F14E
:10FEB800200620FA06F501FA03F19A4029439840F2
:10FEC800160CB1FBF6F597B206FB15114FEA104C6C
:10FED80007FB05F34CEA01418B4209D9891805F162
:10FEE800FF3C80F015818B4240F21281023D891857
:10FEF800C3EB010CBCFBF6F306FB13C180B207FB96
:10FF080003F740EA0140874207D9591E821880F05A
:10FF18000581974240F20281023B43EA05420023F1
:10FF280003E08B420AD900231A461046194614B139
:10FF3800404261EB4101BDE8F0077047B3FA83F333
:10FF4800002B40F087808C4501D38242ECD80122F7
:10FF5800EBE712B90123B3FBF2F2B2FA82F6002EF4
:10FF68003AD1891A150C1FFA82FC0123B1FBF5F767
:10FF780005FB17114FEA10480CFB07F648EA014148
:10FF88008E4207D9891807F1FF3802D28E4200F253
:10FF9800DA804746891BB1FBF5F605FB161180B2DE
:10FFA8000CFB06FC40EA0140844507D9711E821803
:10FFB80080F0B080944540F2AD80023E46EA0742A8
:10FFC800B3E7E443524263EB430365E7404261EB26
:10FFD80041014FF0FF345CE7B240C6F1200521FA39
:10FFE80005F320FA05F701FA06F9150CB3FBF5F845
:08FFF80047EA09091FFA82FC27
:020000040801F1
:1000000005FB18374FEA19410CFB08F341EA074793
:10001000B040BB420AD9BF1808F1FF3180F095808B
:10002000BB4240F29280A8F10208BF18FE1AB6FB4C
:10003000F5F305FB13611FFA89F90CFB03F649EA96
:1000400001418E4206D95F1E891878D28E4276D938
:10005000023B8918891B43EA08438BE7C3F1200759
:1000600026FA07F80CFA03F248EA020C21FA07F123
:1000700005FA03FA4FEA1C4920FA07F5B1FBF9F833
:1000800045EA0A0509FB18172A0C1FFA8CFA0AFB25
:1000900008F142EA0747B94206FA03F609D917EB15
:1000A0000C0708F1FF324ED2B9424CD9A8F1020830
:1000B00067447F1AB7FBF9F209FB1271ADB20AFB74
:1000C00002FA45EA01418A4507D9551E11EB0C0198
:1000D00037D28A4535D9023A614442EA08424FEAAA
:1000E000124C1FFA86F808FB0CF7360C95B208FB89
:1000F00005F806FB057505EB184506FB0CFCAF4241
:1001000088BF0CF5803CCAEB01010CEB1546B142EF
:1001100012D309D000230CE76546EDE60E4646EA09
:10012000074206E70B46FCE61FFA88F800FA03F3DD
:1001300008EB0545AB42EDD2013A0023F9E63B4618
:1001400088E72A46C9E79046B3E788466EE7023F4C
:10015000891823E72DE9F00F144605460E46002BBB
:100160003FD18A424AD9B2FA82F343B1C3F12000A7
:1001700025FA00F201FA03F69C4016439D40210C3B
:10018000B6FBF1F22F0CA0B201FB126C00FB02F3E4
:1001900047EA0C46B34208D9571E361980F0FF8053
:1001A000B34240F2FC80023A3619F61AB6FBF1F37C
:1001B00001FB1361ADB200FB03F045EA0141884247
:1001C00007D95E1E091980F0EC80884240F2E98070
:1001D000023B43EA0242002310461946BDE8F00FF5
:1001E00070478B4243D8B3FA83F4002C42D18B4240
:1001F000234601D382423BD80122EDE712B9012305
:10020000B3FBF2F4B4FA84F2002A40F08A80091BAE
:10021000260CA7B20123B1FBF6F006FB10114FEA42
:10022000154C07FB00F24CEA01418A4207D9091933
:1002300000F1FF3C02D28A4200F2D3806046C2EB5A
:10024000010CBCFBF6F206FB12C1ADB207FB02F7D4
:1002500045EA0145AF4207D9511E2C1980F0A38011
:10026000A74240F2A080023A42EA0042B4E70023EB
:100270001A46B1E7C4F1200722FA07F603FA04F39D
:10028000334321FA07FA4FEA134C01FA04FB20FA30
:1002900007F141EA0B0BBAFBFCF70CFB17A61FFAA0
:1002A00083F84FEA1B4508FB07F945EA0645A945CF
:1002B00002FA04FA04D97A1EED18C0F088801746B5
:1002C000C9EB0505B5FBFCF60CFB16521FFA8BFBC0
:1002D00008FB06F84BEA0241884503D9721EC9188B
:1002E00070D3164646EA0742170C1FFA8AFC0CFB2D
:1002F00007F695B24FEA1A430CFB05FC03FB0565B4
:1003000005EB1C4503FB07F3AE4288BF03F58033C2
:10031000C8EB010103EB1543994250D347D00023AA
:100320005AE79440C2F12008260C20FA08F721FA77
:1003300008F501FA02F9B5FBF6F847EA090906FBE8
:100340001855A7B24FEA194C4CEA054C07FB08F3C5
:10035000634500FA02F509D91CEB040C08F1FF32E1
:100360003DD263453BD9A8F10208A444C3EB0C027B
:10037000B2FBF6F306FB13201FFA89F907FB03F221
:1003800049EA00418A4206D9581E091925D28A42F3
:1003900023D9023B0919891A43EA08433BE73A4645
:1003A00003E7334615E70A4642EA004214E71FFA1C
:1003B0008CF100FA04F001EB0545A842AFD2013AF6
:1003C000002309E788458CD9023EC9188AE7A94568
:1003D0007FF675AF023FED1872E70346DBE7904604
:1003E000C4E7023809192AE7002103E00A4B5B58E9
:1003F0004350043109480A4B42189A42F6D3094A3D
:1004000002E0002342F8043B074B9A42F9D3FAF783
:10041000BBF900F00DF8704784B00508000000201B
:10042000FC0C0020000D0020FC520020FEE7000024
:10043000B54BF7B54FF4FA661E60B44AB44BB54FEE
:100440001A60B54AB54B1A60B54B42F210721A6089
:10045000B44B64241C6001233B70F8F73CFDB24BA5
:1004600000251D70F7F7D6FEF5F7C2FFF5F7CCFFB4
:10047000F5F7DAFFF6F7E6FD2046F7F75DFAF6F74F
:1004800007FE2046F7F758FAF7F7AAFEF7F700FD40
:10049000F7F760FA2046F7F74FFAFAF7C1FA204665
:1004A000F7F74AFA4FF4FA50F7F7B2F92046F7F7A0
:1004B00043FAF6F71FFD2046F7F73EFA2846F7F70E
:1004C0001BFB9A48F7F738FAF4F7D8FA2046F7F703
:1004D00033FA974B03F1100229468DE82400284691
:1004E0005A681B68F4F7DCF83046F7F725FA284617
:1004F000F4F7AEFC4FF6FF70F4F7C0FC0321322096
:100500008C4A2B46F4F7DEFD96208B4A8C212B4635
:10051000F4F7D8FD9620A021884A2B46F4F7D2FDA7
:10052000874A2B469620B421F4F7CCFDF8F78AFCD5
:100530005021DC20F8F759FC3046F7F7FDF9814AE5
:100540002B46DC212846F4F7BDFD7F48F7F7F4F988
:100550002046F7F7F1F9F6F765FA2046F7F7ECF9D8
:100560009FED7A0AF7F7E0FA2046F7F7E5F9F7F793
:100570000BFAF5F76FF82046F7F7DEF9142001467D
:10058000F5F7BEFF2846F6F711F82046F7F7D4F93D
:10059000F6F792F92046F7F7CFF9F6F74BFD20462C
:1005A000F7F7CAF9F6F78EFA00B13D70F6F796FA4A
:1005B00008B1F8F7F1FBF1F751F8F5F701F808B9D0
:1005C000634803E0634B644800221A70F1F761F856
:1005D000F5F76AFCF8F739F9F8F76CF9F8F71AFF4C
:1005E000F7F720FFF8F7FBFBFAF782F9F8F74AFC78
:1005F0005A4B5B4C574E802814BF4FF480504FF439
:1006000080601880454B1A68414B1B68D31A06EE70
:10061000903A434B1B68B8EEE67A06EE903AF8EE55
:10062000E67A504BC7EE277A2546FCEEE77A17EEBE
:10063000902A1A804C4B1868F7F760FDF6F764FAB9
:100640003378012B21D1494B1A786AB100221A70F4
:10065000474B1868474B1B68C018474B1860F7F7A3
:100660004DFD4B20F7F7F8FD444B1A786AB1002294
:100670001A703F4B18683F4B1B68C01A3E4B1860FE
:10068000F7F73CFD4B20F7F7E7FDF7F791FDF2F7A1
:10069000F5FFF9F7C3FF23781BB100232370F1F7AF
:1006A0005FFC6B781BB100236370F1F7E5F8344F02
:1006B0003B881BB2012B05D1A3780BB9F8F770FF6B
:1006C00000233B80E3783BB10020E070F3F7BAFEF3
:1006D0002C4B1878F0F7C0FA237943B1F8F7B2FB46
:1006E000F0209621F8F781FB2748F6F71FFF274FE8
:1006F0003846FBF780FC0028A0D03B78112B9DD119
:10070000F8F7C2FA9AE700BF843E0020E0673500A0
:10071000B03E0020280F002080C3C901CC44002037
:10072000A4440020643E00204446002000127A00C9
:1007300078880108EDA8050807A9050813A9050888
:100740001FA9050828A90508002D31010000FA4459
:1007500058110020443E002044130020AC3E0020ED
:10076000100E002024480020A83E0020E02D00208C
:10077000AC440020403E0020483E0020E32D0020F5
:10078000F40D0020C044002040420F004C3E0020E9
:1007900010B4314C0180B1F5807F44608270C37029
:1007A00052D00DD9B1F5806F39D017D9B1F5006F9E
:1007B0002ED0B1F5805F24D0FF2040B210BC70472E
:1007C00020293AD014D9402930D08029F4D12349A6
:1007D0004FF02012C26081600020EEE7B1F5007F8B
:1007E000EAD11F4B4FF00811C16083600020E4E79D
:1007F0001029E1D11B494FF00122C2608160002025
:10080000DBE7194B4FF00111C16083600020D4E792
:10081000164A4FF00213C36082600020CDE71449EE
:100820004FF00412C26081600020C6E7114B4FF008
:100830004011C16083600020BFE70F4A4FF0801372
:10084000C36082600020B8E70C4A4FF01013C36009
:1008500082600020B1E700BF5CA704089A970508F2
:100860006A9705085A9905085C9705085E97050878
:1008700062970508DA9705085A9805087A970508D7
:100880002DE9F00FB2B02E9030932E9B00882E9C55
:100890005B68309FA4682D90451E03EB4506BF089A
:1008A000209328942C952F911F921E96319700F03B
:1008B0003A814FEA900A4FEACA0B00F003002F99E1
:1008C000299003F1080504EB0B00CDF884A0CDF8C6
:1008D000A8B019951A921B97189617912B90179AF2
:1008E000189E13883380B2F802C0A6F802C094881C
:1008F000B480D788F78008361896219F199E083251
:10090000179256F8041C56F8082C4FF0000A4FF0C6
:10091000000B002F00F06982CDE904ABCDE906ABF6
:10092000CDE902ABCDE900AB289CBC46029BDDF8CB
:100930000C902568C2FBC5394FF0000848EA030A4D
:10094000CB46CDE902AB049BDDF814B0C1FBC53B3F
:10095000CDF824B0CDF82080DDE908ABC1EA020073
:100960004AEA030ACDE904AB069BDDF81CB0326805
:10097000C0FBD53BCDF82CB0CDF82880DDE90AAB23
:10098000C2EA01074AEA030ACDE906AB9DE801087D
:10099000C7FBD50BCDF834B0CDF83080DDE90CAB1A
:1009A0004AEA000A63680298CDE900AB0834DDF832
:1009B0000CB0C1FBC30BCDF83CB0CDF83880DDE9FD
:1009C0000EAB4AEA000ACDE902AB71680498DDF883
:1009D00014B0C2FBC30BCDF844B0CDF84080DDE9C4
:1009E00010AB4AEA000ACDE904AB0698DDF81CB06A
:1009F000C7FBD30BCDF84CB0CDF84880DDE912AB86
:100A0000C1EA02054AEA000ACDE906AB9DE8010801
:100A1000C5FBD30BCDF854B0CDF85080DDE914AB55
:100A200008364AEA000ABCF1010CCDE900AB7FF4BC
:100A30007DAF2A9D19982B9B2E18299F002F35D00A
:100A40001868039F029BC2FBC03700241D971C94AB
:100A5000DDE91C4544EA0304CDE90245049B059DFC
:100A6000C1FBC035002723952297DDE9224544EAE2
:100A70000304CDE90445C1EA0203079D069AC3FBBE
:100A8000D02525952497DDE9244544EA02043368FE
:100A9000C3EA0101CDE9064553465D46C1FBD035A9
:100AA00027952697DDE926AB4AEA030A069A029CB7
:100AB0000499039D079FD30B059AE60BC90B46EAE1
:100AC000454043EA474441EA424604F30F0500F338
:100AD0000F0C199BCCEA054706F30F001A9D1B9ECD
:100AE0002F604FEADA3A08334AEA4B4B0BF30F0414
:100AF000C0EA04426A600835711E19931A951B9169
:100B00007FF4EDAE319A2F9E1E991F9BDDF880B0C9
:100B1000D00037180D182F970BEB000A1F181E95E1
:100B20001F97CDF880A0DDF8C0C01CF0030BCDF8F6
:100B300020B000F086802D9BDDF8BC80CDF808B099
:100B40005808DDF880A0DDF8A0B00690CDF8108040
:100B5000049A1E9E32F8025B069826F8025B049205
:100B6000BAF80270BBF80230BAF80020BBF80040B7
:100B70001E9617FB03F112FB04F6451E4FEAE177C0
:100B800011EB06082B4605F0010047EBE6790AF168
:100B900004020BF10401002D3BD0A8B1B2F800C053
:100BA000BBF80470548848881CFB07F518EB050750
:100BB00049EBE57614FB00F917EB090846EBE979F8
:100BC00004320431013B24D00F88B2F800C05688AB
:100BD00048888C8895881CFB07FC18EB0C0816FBD2
:100BE00000F7D088CE8849EBEC7C15FB04F518EBB8
:100BF00007084CEBE77918EB050710FB06FC49EBFF
:100C0000E57417EB0C0844EBEC7908320831023B31
:100C1000DAD11F9A02994FEAD83545EA494404F3DC
:100C20000F0322F8023B4F1E0AF1020A1F9202979D
:100C30008ED1DDF880A0DDF820B00AEB4B0ACDF8AC
:100C400080A02C9E2E98B50840683FD0209F47EA90
:100C5000000212F0030F00F1080307F1080214BFAD
:100C6000002101219F4298BF904294BF0026012697
:100C7000314277D097E84200016001216C1EA94201
:100C8000466004EA010419D044B192E812001960E8
:100C900002215C6008320833A9420FD092E850006C
:100CA0001C605E60966802F1080BD2689E6002319B
:100CB000DA601033A9420BF10802EFD1DDF880C0F1
:100CC000ED000CEB050B4019CDF880B02C9C14F016
:100CD000030343D05A085400002A00F08E80209D60
:100CE00040EA050717F0030F209F14BF00250125D8
:100CF000011D3E1D012B94BF002505F001058F420B
:100D000098BFB04294BF002101210D4275D03968CF
:100D10009200BF18A342016020971044C4EB030166
:100D20001CD0209B013933F8024B0A4620F8024BB5
:100D300001F0010192B129B133F8021B013A20F808
:100D4000021B0BD01C46014634F802CB21F802CB23
:100D50005D88A31C4580881C023AF3D132B0BDE8FF
:100D6000F00F7047B7F800C0A0F800C07C8844803E
:100D7000BE888680691EFE880C46BA4601F00101D5
:100D8000C680002C9AD089B1B2F800B0A3F800B0A8
:100D900051885980B2F804C0A3F804C0B2F806B074
:100DA0000832A3F806B00833013C87D016881E80AD
:100DB00051885980B2F804B0A3F804B0B2F806C064
:100DC000A3F806C016891E8103F1080B5189ABF800
:100DD00002109389ABF80430D6891032023C0BF133
:100DE0000803ABF80660E1D168E7289BCDE904ABC6
:100DF000CDE906ABCDE902AB1FE6194691E700BF8E
:100E00002DE9F00F9CB006780F900F9C40880F9D45
:100E1000A4686D681990B3FBF6FA471E4FEA5A08AA
:100E200004EB4709AAEB480340460A940D951A972C
:100E3000CDF86C800C911492CDF82C901193002871
:100E400000F0B5811746199A199CCDF84880910891
:100E5000CA00159104F00303A9181792169310976E
:100E60001891760075084FEA450C002D00F03B8480
:100E70000B9FDDF8308047EA080010F0030F14BF25
:100E80000021012108F10404381D012E94BF002126
:100E900001F00101804598BFA74294BF4FF00009BF
:100EA0004FF0010911EA090F00F01D84BB46D8F884
:100EB000002001236F1EAB42CBF8002007EA030796
:100EC0002146024614D237B1246802230431021DA0
:100ED000AB4204600CD20C46104654F8047B40F838
:100EE000047B496802335160211D021DAB42F2D3DD
:100EF000DDF83080DDF82CB04FEA4C05664508EB94
:100F000005020BEB0503CCEB06001DD0013832F8CF
:100F100002CB014623F802CB00F00100A1B128B1B9
:100F200032F8029B013923F8029B0DD014461F466C
:100F300034F8029B27F8029BB2F802A0A21CA3F887
:100F400002A0BB1C0239F1D10C9ADDF83CC00B9811
:100F50009CF80080710053180A9E0C93159BCDF8E5
:100F60004C80451806EB48020B950E92002B00F0C2
:100F7000B18300240025CDE90445CDE9024507935E
:100F80000D9913460A9AB3F804A0B2F806B0CDF84A
:100F900004A0B3F806A00E881588CDF820B0CDF8CF
:100FA00024A0DDE902AB15FB06F51AEB050A4BEBB5
:100FB000E57BCDE902AB1F884888B2F802C0B3F8E0
:100FC0000290B2F804808C88CDF81880DDE904AB7B
:100FD00016FB07F61AEB060A4BEBE67BDDE9026728
:100FE0001CFB00F5761910FB09F047EBE5771AEBCF
:100FF000000A4BEBE07BCDE902ABDDF818B0DDF881
:1010000004C0B1F80680099D1BFB04F016EB000A32
:1010100047EBE07BDDE9026714FB0CF4361947EB84
:10102000E477089C14FB08F00831083208331AEB07
:10103000000418FB05F84BEBE075079816EB080A5F
:1010400047EBE87B0138CDE90245CDE904AB0790D9
:1010500099D1179E0E9C0A9B1899A7199A190E9759
:10106000169F002F73D00E9B31F8020B32F8024B03
:1010700033F8026BDDE90289DDE904AB14FB00F40F
:101080007D1E10FB06F618EB040849EBE4791AEB19
:10109000060A4BEBE67B2F4605F00100CDE90289FD
:1010A000CDE904AB002D52D0002873D031F8024BAB
:1010B00032F8020B33F8025B10FB04F614FB05F068
:1010C000DDE90245DDE90489A41945EBE67518EB75
:1010D000000849EBE079013FCDE90245CDE90489FB
:1010E00035D0C246CB46DDE902890D461446049749
:1010F000214628461A4630F8026B31F8027B32F856
:1011000002CB6D8864885B8817FB06F718EB07082D
:1011100016FB0CF649EBE7791AEB060714FB05FA08
:101120004BEBE67B15FB03FC8C1C931C0499851C84
:1011300018EB0A0849EBEA7917EB0C0A4BEBEC7B4E
:101140008A1ECDE902890492D2D1CDE904AB029D79
:1011500003990498DDF828A0059BEA0B109D42EA4C
:101160004148129908F30F09A5F80090DDF84C905A
:10117000C70B0AEB8908281D4A1E47EA4346CDF8EB
:10118000288006F30F0410906C8012920AD00F9CF6
:10119000267866E6DDE904AB0D4614460497DDE9E2
:1011A0000289A5E7149F1B9B07EB83061496119FEA
:1011B000002F00F0A681DDF864B0DDF86480DDF872
:1011C00034C04FEA9B09CDF81C904FEAC90908F0DA
:1011D000030A0CEB090BCDF82090CDF810A0CDF848
:1011E00024B0DDF83CC09CF8006075084FEA450C5F
:1011F000002D00F07E820C990B980B9F40EA0104B1
:1012000014F0030F14BF002201220C1D0430012E24
:1012100094BF002202F00102814298BFA74294BF0E
:10122000002301231A4200F06482BA4601230F68AA
:10123000691EAB42CAF80070024601EA0307214664
:1012400014D237B127680223211D021DAB4207606B
:101250000CD20C46104654F8047B40F8047B4968D5
:1012600002335160211D021DAB42F2D3DDF83090F4
:10127000DDF82C804FEA4C05664509EB050208EBCA
:101280000503CCEB06001DD0013832F802BB014645
:1012900023F802BB00F00100A1B128B132F8025BD3
:1012A000013923F8025B0DD014461F4634F802AB17
:1012B00027F802ABB2F802C0A21CA3F802C0BB1C04
:1012C0000239F1D1DDF82CA0DDF830B007987600B6
:1012D0000AEB060C0BEB0608CDF82CC0CDF83080DD
:1012E000002800F0F0810A9ADDF834805788B2F8BF
:1012F00000A0DDF828909488B9F80690B8F8062088
:1013000084460D9841880588B8F8040017FB01F65B
:101310001AFB05F3B3461BEB03014FEAE67714FB18
:1013200000F047EBE3750F180A9B19FB02F145EB40
:10133000E0750CF1FF3617EB010AB14606F001002B
:1013400008F1080203F1080345EBE17B002E00F0F1
:10135000858048B3DDF834C01E88BCF80840588842
:10136000518897889D88B2F80680B3F806C016FBAE
:1013700004F41AEB040A10FB01F14BEBE4761AEBD0
:10138000010415FB07FB46EBE17014EB0B011CFBA2
:1013900008F640EBEB740832083311EB060A44EB15
:1013A000E67BB9F1010959D0CDE902ABCB46B3F8E0
:1013B0000080B3F808901688CDF8389018FB06F630
:1013C000DDE902895D88548898889188B2F806C062
:1013D000DF88B2F808A015FB04F418EB060810FB30
:1013E00001F149EBE67918EB040817FB0CF749EB20
:1013F000E47918EB010849EBE17918EB070849EBB0
:10140000E779CDE90289DDF838905D8954899889BA
:101410009189B2F80EC0DE8919FB0AF7DDE902896D
:1014200015FB04F418EB070810FB01F149EBE77911
:1014300018EB040849EBE47916FB0CF618EB0104F1
:1014400049EBE17510321033A01945EBE671BBF1A1
:10145000020BCDE90201AAD182468B460DF120088C
:1014600098E816006318049D9DB332F802CB33F858
:10147000026B16FB0CF4013D1AEB040A294605F039
:1014800001004BEBE47B25B358B132F8028B33F803
:10149000020B10FB08F71AEB070A4BEBE77B691E00
:1014A00017D01446184634F8025B30F8027B528895
:1014B0005B8817FB05F81AEB08064BEBE87713FB84
:1014C00002FBA21C831C16EB0B0A47EBEB7B0239D9
:1014D000E7D10F9DDDF8508095F800C00A9A119E63
:1014E0004FEADA3343EA4B4404F30F0028F8020BC7
:1014F00002EB4C07711E0A97CDF8508011917FF4D2
:1015000070AE1A9E0F9CB508A06842D00A9F47EAA9
:10151000000616F0030F07F1080200F1080314BFDC
:10152000002101219F4298BF904294BF4FF0000AD2
:101530004FF0010A11EA0A0F7FD097E842000160DC
:1015400001216C1EA942466004EA010419D044B18D
:1015500092E81200196002215C6008320833A94247
:101560000FD092E850001C605E60966802F108049B
:10157000D2689E600231DA601033A94204F1080299
:10158000EFD1DDF828A0ED000AEB05094019CDF8F0
:101590002890DDF868A01AF003034AD05A085400D6
:1015A000002A00F0A480DDF828B040EA0B0515F011
:1015B000030F14BF002501250BF10406011D012BAB
:1015C00094BF002505F001058B4598BFB04294BF3C
:1015D0004FF0000C4FF0010C15EA0C0F00F0878063
:1015E000DBF8001092009344A3420160CDF828B0CC
:1015F0001044C4EB03011CD00A9B013933F8024BA1
:101600000A4620F8024B01F0010192B129B133F8EA
:10161000021B013A20F8021B0BD01C46014634F88D
:1016200002CB21F802CB5D88A31C4580881C023ABE
:10163000F3D11CB0BDE8F00F7047B7F80090A0F8E8
:1016400000907C884480BE888680691EFE880C4697
:10165000B84601F00101C680002C92D091B11188EA
:101660001980B2F802C0A3F802C0B2F804A0A3F82F
:1016700004A0B2F806900832A3F806900833013CA3
:101680003FF47FAF11881980B2F802C0A3F802C0FE
:10169000B2F80490A3F80490B2F806A0A3F806A04C
:1016A00016891E8103F1080C5189ACF80210938948
:1016B000ACF80430D6891032023C0CF10803ACF8C7
:1016C0000660DFD15DE70D9A0A9B4FF0000A4FF0EC
:1016D000000BC8E600260027CDE904670A9A0D9999
:1016E000CDE90267BCE430460B9B0C9A0EE4194628
:1016F00082E730460B9B0C9AC6E500BF0000000055
:1017000000B553EC102B42F2FB1223F00043C3F65A
:10171000E972934285B026DD4FF6FF72C7F6EF728D
:1017200093420BDD51EC100B02460B46FDF784FE95
:1017300002460B4643EC102B05B000BD684600F096
:10174000EBFB00F0030001289DED000B9DED021B5B
:101750001AD0022810D0F8B900F0FEFE53EC102B7E
:1017600010461946E4E79FED101B00F0F5FE53EC20
:10177000102B10461946DBE700F0EEFE53EC102B61
:10178000104603F10041D3E701F022FC53EC102B8B
:10179000104603F10041CBE7012001F019FC53ECA6
:1017A000102B10461946C3E700000000000000009F
:1017B0002DE9F04759EC108BC9F30A56A6F57E7453
:1017C000073C132C4D46CA46474626DC002C4FDB0F
:1017D0004FF6FF76C0F20F0646FA04F606EA090550
:1017E00055EA080517D044A3D3E9002351EC100BA8
:1017F000FDF724FE00220023FEF762FA00284AD0FB
:10180000B9F1000F6EDB2AEA060A4FF000085346D2
:10181000424643EC102BBDE8F087332C0CDDB4F5C9
:10182000806FF8D151EC100B3A460B46FDF706FEDF
:1018300041EC100BBDE8F087A6F58265033D4FF043
:10184000FF3323FA05F515EA080FE4D02AA3D3E9FC
:10185000002351EC100BFDF7F1FD00220023FEF7F1
:101860002FFAC0B1B9F1000F1CDB28EA050813E01C
:1018700021A3D3E9002351EC100BFDF7DFFD00227B
:101880000023FEF71DFA38B1B9F1000F1BDB4FF052
:101890000008C24600E0CA465346424643EC102BBD
:1018A000BDE8F087142C09D0C6F5866303334FF0EA
:1018B000010808FA03F818EB0708D6D30AF1010A61
:1018C00028EA0508E8E729F0004848EA07084FF049
:1018D000000AD045CBF6F07A08BFCA4618BF4FF0D1
:1018E0000008D9E74FF4801343FA04F409EB040A23
:1018F00089E700BFAFF300809C7500883CE4377E29
:1019000000B553EC102B42F2FB1223F00043C3F658
:10191000E972934285B027DD4FF6FF72C7F6EF728A
:1019200093420BDD51EC100B02460B46FDF784FD94
:1019300002460B4643EC102B05B000BD684600F094
:10194000EBFA00F0030001289DED000B9DED021B5A
:101950001DD0022812D008BB012001F039FB53EC46
:10196000102B10461946E3E700209FED111B01F0F4
:101970002FFB53EC102B10461946D9E7012001F03C
:1019800027FB53EC102B104603F10041D0E700F089
:10199000E3FD53EC102B10461946C9E700F0DCFDBF
:1019A00053EC102B104603F10041C1E7AFF3008068
:1019B000000000000000000010EE103A0BB90220F9
:1019C0007047B3F1004FFAD0A3F500016FF0014268
:1019D000914201D80420704703F1FF419142F9D9A7
:1019E0004FF6FE72591EC0F27F02914201D80320C9
:1019F000704703F1004101399142F8D9B3F1FF4F2B
:101A000005D013F5000F14BF0020012070470120FE
:101A1000704700BF00F0E4B8D0B52DED048BB0EEF8
:101A2000408AF0EE608A3C4C8AB000F0D9F994F913
:101A30000030B0EE409AF0EE609A013335D0B0EE4F
:101A4000480AF0EE680A01F04DFD00282DD051EC57
:101A5000180B00220023FEF71FF930B32F4B247818
:101A60000193002308938DED028B8DED048B002CE8
:101A700023D000270026CFF6F07751EC180B002278
:101A80000023CDE90667FEF7F3F8002825D00223EE
:101A90009C42009336D0684601F05CFD002831D0AE
:101AA000089B002B27D19DED069BB0EE490AF0EE76
:101AB000690A0AB0BDEC048BD0BD4FF6FF774FF03A
:101AC0006046CCF2EF7751EC180B00220023CDE9F1
:101AD0000667FEF7CDF80028D9D10123022C009328
:101AE00015D0684601F036FD88B10D4801F034FD8F
:101AF0008DED060BD4E701F0EDFF089B9DED069BF5
:101B00000360D2E701F0E6FF22230360C8E701F09B
:101B1000E1FF21230360E8E73804002088AB0508D3
:101B2000E8AD050810B52DED048BB0EE408AF0EE5F
:101B3000608A294C8AB000F02BFC94F90030B0EE9A
:101B4000409AF0EE609A01332BD0B0EE480AF0EEE6
:101B5000680A01F0C7FC20B351EC180B00220023E7
:101B6000FEF790F8E8B11D4B247801930123009310
:101B7000002308938DED048B8DED028BCCB10020FA
:101B8000002102460B46FDF735FF022CCDE9060188
:101B900015D101F09FFF21230360089BABB99DED98
:101BA000069BB0EE490AF0EE690A0AB0BDEC048B60
:101BB00010BD0022002343EC172B8DED067B6846F9
:101BC00001F0C8FC0028E8D1E3E701F083FF089B9F
:101BD0009DED069B0360E4E73804002090AB050808
:101BE000F8B5B0EE407AF0EE607A53EC112B544227
:101BF00010461D46002125F00047044353EC102BEE
